:020000024000BC
:100000006FD0425B00000000001801180028012892
:100010000228032800290129022903290429052986
:10002000062907290829002A012A022A032A042A64
:10003000052AA62AD4E10600F24204006804002042
:10004000EA040020EA030020B80300205003002047
:10005000FA2900208A430400AC440400424704000B
:100060005C4804004A420400F8410400B402002045
:1000700054020020184D040064080020604304006E
:100080001E4A04008A7B0600707D0600D67D0600AD
:100090005658060090580600D8870500A67C050033
:1000A000607606004C4A0400545F060014FC04000D
:1000B000A2FC040000FD04001C5504005A55040075
:1000C000D053040022BE040008B904001C2B0020F9
:1000D00046CA040098CD0400AAAB04004CAB04004F
:1000E00018AF0400F6AB04002AAB0400A2AB040076
:1000F000E0AA040078AC0400D0AC040080AC04009A
:1001000084AC040012AD0400D8AC040008AD0400B7
:10011000EAB10400EEB1040074AC04007CAC04004D
:1001200010AD0400ECB10400BEAD04004AB30400FD
:1001300046DB0400B8DB0400F2DB040068C0040006
:100140007EC00400B8C00400C2A00400C8A204001D
:1001500090A30400BC720400066D0400C096040065
:10016000826D040076920400D6BA06000CB3060035
:1001700012B806008ACF060054CE0600ACD20600A4
:1001800068D20600A4D20600F8D30600C8A1060073
:1001900088D30600E6C506000CC606002CC606007D
:1001A00068D4060048CC0600E0CB0600D8D4060090
:1001B0004CA40600E4A4060004A50600B6A40600AC
:1001C000E05F05006A4A0500E64D0500A64B050004
:1001D000F8550500AC3D0020F8750600FCA10600AE
:1001E000A64E0400A6590600345F06002C600600E7
:1001F0003A6E0600C26E06002070060022C404009B
:10020000E25E0500A05605003A4805004E5905007B
:100210001A4A05002A0A00207E5A0600D2D2060099
:100220006CD20600A0D206009CD20600C246040092
:10023000A0C10400DAD20600B062060076630600B0
:10024000DE6306007AB80600D6D2060020D3060088
:10025000287C050024D3060042200020082000202E
:100260005AB80600F0B9060028D306007CD3060071
:1002700080D30600DED2060018D306001CD3060089
:1002800084D30600985F0500000000000000000015
:10029000000000000000000000000000000000005E
:1002A000000000000000000000000000000000004E
:1002B000000000000000000000000000000000003E
:1002C00097470000938787F21747000013070776C8
:1002D0006373F700828023A007009107D5BF97477B
:1002E0000000938727E317E706E013072757974691
:1002F00000009386A6EF63F3F60082801043110797
:0603000090C39107CDBF80
:100308004111B7E700E022C480433707200006C642
:10031800798C23A0E7180F10000011C199E5B7E701
:1003280000E023A08710014579A80D05334505088D
:10033800130740037199B34705086366A702174579
:1003480000000325A5EA9746000083A6A6E9639165
:10035800A602174700000327270C71D3C207DD8DBB
:10036800054502976DBF174500000325E5E7E1BF86
:100378007A2131EF5A21636CF704B306F74021481C
:10038800174600001306C6036375D80283280500C4
:1003980003586600938687001D8FAA966117DAA214
:1003A80023A016012393060014C15EA1130788FF3A
:1003B8007AA27A226EA12105B307F7407EA2B7E799
:1003C80000E023A08710B240224441018280084106
:1003D800BDBFB7E700E08C433707200023A0E7182C
:1003E800F98D0F10000001E523A0B7108280174394
:1003F80000000323A3DF9748000083A8A8DE9A879C
:10040800814663FE170903A80700636DF508636B4F
:10041800A808138787006364E508F22321670507A6
:100428006319E600174600001306B6EA1822050706
:1004380018A2174500001305A5F8D2237A212393A3
:1004480007003297334707087AA163856702174385
:100458000000032363D9630FF30003D36600631B13
:100468000300DE2223A0060121073E962106D2A220
:100478007AA1B6879843630417039746000083A6BA
:10048800A6D6630ED700762399EAD62352231843BB
:10049800A106B296D6A398C37E21A1077EA1B7E78D
:1004A80000E099B7BE86C287A9BFAA871747000090
:1004B8000327C7D3174600000326C6D2B305B540A5
:1004C8006314E6003E8529A8930687001843E3E9EC
:1004D800D7FEE3F7E7FE2E85E3E4D5FEE3F2E5FE7B
:1004E800828023AC05FE1C4199E30CC182803E87C3
:1004F80083A787FFEDFF232CB7FE8280411126C218
:10050800B7E400E04AC003A90400B707200006C604
:1005180022C43379F90023A0F4180F10000009E56C
:1005280023A0241101452DA09565938505D0C98D7B
:100538002A842105B3C5050833450508D1336DD193
:10054800FD572320050042A17CA123A024112105E9
:10055800B240224492440249410182804111B7E7E6
:1005680000E04AC003A9070026C23707200006C6D4
:1005780022C4AA843379E90023A0E7180F100000E9
:100588009747000083A7C7C60144014695E311C8F1
:10059800A285174500001305A5C5974004E0E7802C
:1005A80080EEA1652685974004E0E78040441DA0C1
:1005B80003C7E7FF631B970215CCA2851745000008
:1005C800130505C3974004E0E780E0EBA1652685A5
:1005D800EF20206DB24022852244B7E700E023A037
:1005E8002711924402494101828011E03E8683A787
:1005F80087FF69BF3E84E5BF37E700E01C43B706C5
:1006080020002320D718F58F0F10000019C191C1C1
:1006180011E637E700E02320F71082802E960F704E
:10062800B650D5BF37E700E01C43B70620002320AB
:10063800D718F58F0F10000019C1014785E137E77A
:1006480000E02320F7108280B386E50003A80600A7
:10065800B306E5007D1623A00601110775F6C5B798
:1006680037E700E01C43B70620002320D718F58F92
:100678000F10000001C53307C50011E637E700E099
:100688002320F71082800505A30FB5FEE31DE5FEC4
:10069800F5B7B7E600E09C42370620002A87F18FBD
:1006A80023A0C6180F1000000145B306A7008386D3
:1006B800060091E637E700E02320F7108280050561
:1006C800EDB70111B7E700E026CA84434AC83707E7
:1006D800200006CE22CC2A892E86F98C23A0E71882
:1006E8000F1000009305F00432C633450608093997
:1006F8002A8401C53246CA850137F2402285624400
:10070800B7E700E023A097104249D24405618280F0
:1007180037E700E01C43B70620002320D718F58FE1
:100728000F10000001C599C1014711EA37E700E041
:100738002320F710054582800507E309E6FE330804
:10074800E500B386E500034808009422E306D8FED6
:1007580037E700E02320F7100145828037E700E003
:100768001C43B70620002320D718F58F0F10000070
:100778001307F6FFBA952A966317C50037E700E016
:100788002320F71082809821FD150505A30FE5FEAB
:10079800E5B737E700E01C43B70620002320D71849
:1007A800F58F0F10000001C53307C50019E637E7BC
:1007B80000E02320F7100145828014210505E39805
:1007C800B6FEE31CE5FE37E700E02320F7100545F9
:1007D8008280797126D2974400009384E4A222D4BF
:1007E800804006D64AD04ECE52CC56CA5AC85EC6AB
:1007F80062C455C437C9C901814B174B0000130B9C
:100808002BA01309F937174A0000130AEABD974AC3
:100818000000938AEABA974900009389E9C13E200B
:1008280091EF5C4463990B009CC0032CC4002285A3
:100838004D36628489A823A6FB00C5BF83270B0019
:1008480082971C443307F5406376F50003A78900B7
:100858001D8F2A976368E9062E200820EF20604440
:100868005C405844A9CB0C4417460000032646BDFB
:10087800AE97BE8663E4B70063E4C700B386C7409B
:1008880014C4A28B3A8441FC17470000032747B4DD
:10089800894763E6E7009747000023AB07B2B250E9
:1008A800225492540259F249624AD24A424BB24BFC
:1008B800224C4561828063940B0098C0BDB723A683
:1008C800EB00A5B703274A021DCB63EDA7023385CA
:1008D800A7401C2099EF03479A0183A68900611756
:1008E800B307A7003E8563E4E70063E4D7003385D8
:1008F800D74083A70A016374F50023A8AA00A28B36
:10090800404451B703A78900BA97D1B7011126CA45
:1009180006CE97440000938424B222CC4AC84EC61F
:1009280052C49C288844DDC3B7E700E003A9070048
:100938003707200023A0E7183379E9000F100000DB
:10094800174700000347478B19CB23A02711F24014
:100958006244D2444249B249224A0561828017471B
:100968000000130727DF8357C70AB1CB9C44032431
:10097800870A6306F40497490000938969A403A7CA
:1009880009012285630DF702174A0000130A4A87F6
:1009980083270A008297636EA40C83270A00098CB8
:1009A800829783A7090198443354F40AB307A40033
:1009B8003E8563E4870063E4E7003385E740B7E7F3
:1009C80000E023A027119C44639DA7021744000060
:1009D8001304049F18489747000083A76782631D84
:1009E800A70882979444374736FE130707C83697F7
:1009F800B307A7003E8563E4E70063E4D7003385C7
:100A0800D740174400001304E4F75C5C99CB974681
:100A1800000083A6E6919C463707CDFF7D17F98F26
:100A28009CC611E1884485475CD09747000083A79E
:100A3800E79D829715E15C5C99CF5C5089CF976000
:100A480006E0E78080A3975006E0E780A02197475B
:100A5800000023AB07F4B53B5C5CE38A07EE17475D
:100A680000000327E78C1C47B7063300D58F1CC747
:100A7800F9BD9C443E9415B7829714489844B387AF
:100A8800A6003E8563E4D700E3EDE7F63385E7404B
:100A98008DBF9737000023AFA77411C58547173757
:100AA8000000230BF7748280AA8799E51747000096
:100AB8000347879909C7F1BF11476369B70017470B
:100AC800000013072796B3C5E5209CC1828097379D
:100AD800000083A7277285C3411106C682979737FE
:100AE800000083C7677189E79737000023A4077060
:100AF800B240410182809737000083C7E76F91E7D2
:100B08009737000023A8076E82808280411122C493
:100B180026C206C64AC0974400009384A4E683C749
:100B28003402174400001304E48FB9C717440000C7
:100B380013040489173900001309496D03270900B4
:100B48001C2014300146B3A5E7208E21A5CD11C283
:100B58001CA00820636FD5069747000023820786EC
:100B68009737000083A7C769C5EFB2402244924473
:100B780002494101828082971C40F5FF9747000097
:100B880083C7878C85E3DC48858B89CFD84C994708
:100B9800631EF7009747000023A007E0EF10F01846
:100BA8005C4482971C44D9D3829749B7D84C9D4757
:100BB800E31AF7FE9747000023A007DEEF10F016B0
:100BC8001C48C5B7850793F7F70F0546E3EDD7F639
:100BD80041B73327E5200E2323100700973700007D
:100BE800239D07609737000083A7C761B347F520A7
:100BF8009C4382971C20832609001737000003575F
:100C0800C75F3377E540B3A6D7209222518F9AA2C7
:100C180099C385071CA018201C30E368F7F42DBF82
:100C28009747000083A7C7811CC8653683C734026D
:100C38008DFF83C7140299CBDC4C89EB97470000E2
:100C4800A38207D6975006E0E78000219737000077
:100C580083A7C77B99DB1C4889DB183083260900EA
:100C6800814763C9E702D84C9147E3E0E7F097472B
:100C7800000083C767AC918BE39907EE97370000B4
:100C880083C78757E39307EE2244B2409244024950
:100C98004101ADB933A6D7201222E31806EC850727
:100CA800C9B7B7C700401387C7201443139626490E
:100CB80010C301000100938787261735000003251C
:100CC800E5719C436A0514C393C7F7FF99835D8D4B
:100CD80082809737000083A7E75391C38287130563
:100CE800F00F82809737000023A6A752828017460C
:100CF80000001306A6A197460000938626A3DC36BB
:100D0800383E4C4ABA97FD8B33D7F5001CB2DCB697
:100D1800058B0DE7943A13050002B3F7D702814615
:100D280033D8E548630908006394D70018B2828075
:100D3800850693F6F60F0507E314A7FE828097470A
:100D4800000083A767C5C1E741114AC09737000073
:100D580083A7074B06C622C426C2829717490000FC
:100D68001309C99C83278900638DA7046363F5046D
:100D78001D8D9744000093846499BC2C135455002E
:100D88006361F404AD37BC2C0327890093965700A0
:100D980036971D8C2324E900E376F4FE224488303C
:100DA800B2409244024981454101173305E067008A
:100DB800E369173700000327A768B307F7403E9594
:100DC8004DBFB24022449244024941018280828050
:100DD800011126CA9737000083A7874206CE22CC86
:100DE8004AC84EC652C4829797440000938404941C
:100DF8009844AA870145630DF70463E3E706998FD2
:100E0800174900001309899093F9F70113D4570083
:100E18008347A901636AF402173A0000130ACA61FA
:100E2800F9350347A9018C4403268A009317570014
:100E3800AE97198CBE8663E4B70063E4C700B38637
:100E4800C74094C4E37EE4FC1315540033653501B0
:100E5800F2406244D2444249B249224A0561828042
:100E68009736000083A6C65D3387E640BA9749BF28
:100E7800411122C4174400001304C4B01C4426C204
:100E880006C6858B9744000083A4049391EBEF304A
:100E980080062244B2402685924441016F10907E1C
:100EA80098289747000023A307AE8947E301F7FE78
:100EB8000146930550020145EF10301A8145177518
:100EC80005E01305A5E5CD36014681450545EF103A
:100ED800607E5C44858BC5DFB24022449244410168
:100EE80082809747000083A7E79063930718011152
:100EF80022CC2A84094506CE26CA4AC84EC6EF30F7
:100F0800A007973900009389A94103A60900930710
:100F18008007173900001309A93F7CD297370000D2
:100F2800238C072C832709009734000093844440BE
:100F3800B7053300D8572285719B13671700D8D798
:100F480098431377F7CF98C398431377F7CF13676E
:100F5800072098C398401447CD8E14C7B7060300DE
:100F68009386862534CA5457F59A54D7984334241F
:100F7800137707F893F6F607558F98C3EF20E00725
:100F880083A60900370500827D15DC4293E7170028
:100F9800DCC203260900030784065C569375F70331
:100FA800E605E98FCD8F5CD69305A0039C4063D5F9
:100FB800E508F84FB70500074D8FF8CFB7C7898EFA
:100FC800938767ED1CC6B7575500938757555CC282
:100FD8008347A40683444406DD8C894717470000ED
:100FE8002320F79C9747000023A4079A7C44BCDE83
:100FF8009737000083C7474599C7FC52FDFF9747BD
:10100800000023A5079818289D478145172500004B
:101018001305E53E6306F70017050000130585E58F
:10102800613410386244F2404249B249A685D2443C
:10103800014505616F1000689305200263DAE50039
:10104800F84FB70500F9FD156D8FB7050005ADB769
:10105800B70500F96945FD156357E500F84F6D8F31
:10106800B705000391BFF84F6D8F13178729B1B7E4
:101078008280973700009387E76DE853054754252A
:101088006390E60203C747079147631AF700011107
:1010980006CE2AC6EF10D05A3245F240056191B506
:1010A800828083278511E5CB411122C406C65825C5
:1010B8008345E5049437D2272A841377C70F1395FD
:1010C800466063F7C50663510506882793F6F60759
:1010D80094B70546936627006314C5009366170006
:1010E80054A4D8430907D8C3032504114CB82E8645
:1010F800CC430905EFF04FD0832784115438D843E7
:101108003697D8C3DA27158FDAA789473CBC034737
:1011180064039737000083C7472E6369F706B24018
:1011280022440145410182801367170058A46DBF0E
:101138009376F60F635505028827854513662700C1
:101148006314B5001366170050A454B8A3840700AD
:1011580085473CBC832784119C43D5FBC9B71367DB
:10116800170058A454B8A384070003250411CC43DE
:101178000905EFF06FC8832784115438D843369790
:10118800D8C3DA27158FDAA78D47E1B75C2493E730
:1011980007015CA469B705458280411197370000B3
:1011A80083A7471522C406C6858B2A84C5E74165EF
:1011B800130525F5979005E0E780408441CD3C254F
:1011C8003EA583270412ADE32320A4122322A412F0
:1011D80085472311F404232005007C2854415EA58B
:1011E800583418A5054718B5138517021737000096
:1011F8000327077D15811C437D151375F50F9CC2C8
:101208005C43DCC21C479CC65C47DCC61C4B9CCAC2
:101218005C4BDCCA1C4F9CCE5C4FDCCE0DC1938668
:10122800060213070702C1BF8327441288C38357E6
:1012380024042322A4128507B3C7070859BF173708
:101248000000130727511E2785071EA7B240224416
:10125800410182805C2423090400054593C74700A7
:101268005CA4EDB7142D854763EED70A1C3D2A8789
:101278000145DDEB5C2713F507013C2B99CB834631
:1012880067039737000083C7571763ECF60001E53B
:10129800828059E582808357271E0357671EBA97B5
:1012A80021A08357271E75F90145BDCF9387C71223
:1012B8001735000003550519B3B5A70237460F00C7
:1012C800411113060624814622C426C206C67D544F
:1012D8003385A70297C006E0E780006197340000D5
:1012E80083C41412AA949737000083A7E74F03A773
:1012F80007099C433354E40AFDFB9737000083A792
:1013080027F0829781476364A400B307A440B240E2
:10131800224433B597001345150092444101828059
:101328008147A5BF014582808280173700000327C7
:1013380027FF3C5BFDFF01000100828039C90111D4
:101348006C0022CC06CE2A84EF20D00715C9FD57A1
:10135800630DF502B2479735000083C5750A63EB44
:10136800B700034594026244F240B385B740056173
:101378006F10D017173700000327870CBA97D5B717
:101388006244F24005616F202047F24062440561E3
:1013980082808280797152CC173A0000130A8A3B06
:1013A80026D283244A0906D622D44AD04ECED5C89E
:1013B800973700009387075DD44F15476386E60487
:1013C800DC532A8989CF975006E0E780000B9750B5
:1013D80006E0E78020899737000023A7075CFD59BE
:1013E8006C002685EF20007E0DE917250000130507
:1013F800E540EFF00FEA9737000083A767F2370759
:10140800100098C70547B8DB0D45B25022549254D6
:101418000259F249624A4561828063743501324457
:10142800AA898440D5FCFD571305F00FE38FF9FC1A
:10143800914763F187029307B4FF2320F90023241F
:10144800FA0A99E79737000083A787FF2320F90056
:10145800014565BF9737000083A787FEED17A29760
:10146800E9BF09455DB7797126D206D622D44AD09C
:101478004ECE52CC56CA5AC85EC68347550303445B
:101488007513AA843E941374F40F9307400263F60D
:1014980087001304B4FD1374F40F03A9841383A9FC
:1014A800C413A38B841222864A85CE8597C006E092
:1014B800E780C03E058915E503CBD412014A814A6D
:1014C800337B6403930B500252864A85CE8597C0BE
:1014D80006E0E780A03C05890DC563916A03137493
:1014E800FA0F238B8412B250225492540259F249B3
:1014F800624AD24A424BB24B45618280850A939A2E
:101508004A60050AE3127AFDE9BF83278509035675
:101518000504797193D60701BD8EB3C60608358ECA
:1015280093575640898B135776485D8F93573640AB
:10153800918B5D8F93571640A18B5D8F9317160083
:10154800C18B5D8F9317360093F707025D8F931752
:10155800560093F707045D8F9317760093F7F70FFC
:1015680022D45D8F2A849357D6001355B60011896B
:10157800898B93558600C98F1355F6002582C98F2C
:10158800218AD18F13961500418AD18F1396350081
:1015980013760602D18F1396550013760604D18F61
:1015A800139675001376F60FD18FA207C5455D8F88
:1015B8003307B70226D24AD04ECE03298413832993
:1015C800C4135AC806D652CC56CA369733470708AA
:1015D80013565740098A93577748D18F1356374087
:1015E800118AD18F13561740218AD18F13161700ED
:1015F800418AD18F1316370013760602D18F13163E
:10160800570013760604D18F131677001376F60F5A
:10161800D18F1358B7001356D70013784800098A9A
:1016280013558700336606011358F7002583336680
:101638000601218B518F13161500418A518F1316FD
:10164800350013760602518F1316550013760604DB
:10165800518F131675001376F60F518F2207D98F05
:10166800B387B7025EC6B697B3C7070813D5574006
:10167800098913D77748498F13D537401189498F7E
:1016880013D517402189498F139517004189498F30
:101698001395370013750502498F13955700137575
:1016A8000504498F139577001375F50F598D13D8D5
:1016B800B70013D7D70013784800098B13D68700D3
:1016C8003367070113D8F700A58333670701A18B98
:1016D800D98F13171600418BD98F1317360013773C
:1016E8000702D98F13175600137707041E06D98FE0
:1016F8001376F60FD18FA2073367F5003307B702C9
:10170800130650024A85CE853697B98EB3C40608AB
:1017180033F6C402137BF60F97C006E0E780001883
:10172800058905E9834AD412014A930B5002B38A0A
:101738009A02814493DA0A0126864A85CE8597C0A3
:1017480006E0E780A01505890DC563914A0313FBE0
:10175800F40F230B6413B250225492540259F249E5
:10176800624AD24A424BB24B45618280050A137ADB
:10177800FA0F8504E39274FDE9BF8327C508035671
:101788008508797193D60701BD8EB3C60608358ED4
:1017980093575640898B135776485D8F9357364039
:1017A800918B5D8F93571640A18B5D8F9317160011
:1017B800C18B5D8F9317360093F707025D8F9317E0
:1017C800560093F707045D8F9317760093F7F70F8A
:1017D80022D45D8F2A849357D6001355B6001189F9
:1017E800898B93558600C98F1355F6002582C98FBA
:1017F800218AD18F13961500418AD18F139635000F
:1018080013760602D18F1396550013760604D18FEE
:10181800139675001376F60FD18FA207C5455D8F15
:101828003307B70226D24AD04ECE0329040A8329A9
:10183800440A5AC806D652CC56CA369733470708C0
:1018480013565740098A93577748D18F1356374014
:10185800118AD18F13561740218AD18F131617007A
:10186800418AD18F1316370013760602D18F1316CB
:10187800570013760604D18F131677001376F60FE8
:10188800D18F1358B7001356D70013784800098A28
:1018980013558700336606011358F700258333660E
:1018A8000601218B518F13161500418A518F13168B
:1018B800350013760602518F131655001376060469
:1018C800518F131675001376F60F518F2207D98F93
:1018D800B387B7025EC6B697B3C7070813D5574094
:1018E800098913D77748498F13D537401189498F0C
:1018F80013D517402189498F139517004189498FBE
:101908001395370013750502498F13955700137502
:101918000504498F139577001375F50F598D13D862
:10192800B70013D7D70013784800098B13D6870060
:101938003367070113D8F700A58333670701A18B25
:10194800D98F13171600418BD98F131736001377C9
:101958000702D98F13175600137707041E06D98F6D
:101968001376F60FD18FA2073367F5003307B70256
:10197800130650024A85CE853697B98EB3C4060839
:1019880033F6C402137BF60F97C006E0E78000F138
:10199800058905E9834A1408014A930B5002B38A62
:1019A8009A02814493DA0A0126864A85CE8597C031
:1019B80006E0E780A0EE05890DC563914A0313FB95
:1019C800F40F230F6407B250225492540259F2497B
:1019D800624AD24A424BB24B45618280050A137A69
:1019E800FA0F8504E39274FDE9BF8327450903567E
:1019F8008508797193D60701BD8EB3C60608358E62
:101A080093575640898B135776485D8F93573640C6
:101A1800918B5D8F93571640A18B5D8F931716009E
:101A2800C18B5D8F9317360093F707025D8F93176D
:101A3800560093F707045D8F9317760093F7F70F17
:101A480022D45D8F2A849357D6001355B600118986
:101A5800898B93558600C98F1355F6002582C98F47
:101A6800218AD18F13961500418AD18F139635009C
:101A780013760602D18F1396550013760604D18F7C
:101A8800139675001376F60FD18FA207C5455D8FA3
:101A98003307B70226D24AD04ECE0329040B832936
:101AA800440B5AC806D652CC56CA3697334707084D
:101AB80013565740098A93577748D18F13563740A2
:101AC800118AD18F13561740218AD18F1316170008
:101AD800418AD18F1316370013760602D18F131659
:101AE800570013760604D18F131677001376F60F76
:101AF800D18F1358B7001356D70013784800098AB6
:101B080013558700336606011358F700258333669B
:101B18000601218B518F13161500418A518F131618
:101B2800350013760602518F1316550013760604F6
:101B3800518F131675001376F60F518F2207D98F20
:101B4800B387B7025EC6B697B3C7070813D5574021
:101B5800098913D77748498F13D537401189498F99
:101B680013D517402189498F139517004189498F4B
:101B78001395370013750502498F13955700137590
:101B88000504498F139577001375F50F598D13D8F0
:101B9800B70013D7D70013784800098B13D68700EE
:101BA8003367070113D8F700A58333670701A18BB3
:101BB800D98F13171600418BD98F13173600137757
:101BC8000702D98F13175600137707041E06D98FFB
:101BD8001376F60FD18FA2073367F5003307B702E4
:101BE800130650024A85CE853697B98EB3C40608C7
:101BF80033F6C402137BF60F97C006E0E78000CAED
:101C0800058905E9834AF408014A930B5002B38A0F
:101C18009A02814493DA0A0126864A85CE8597C0BE
:101C280006E0E780A0C705890DC563914A0313FB49
:101C3800F40F230F6407B250225492540259F24908
:101C4800624AD24A424BB24B45618280050A137AF6
:101C5800FA0F8504E39274FDE9BF411126C206C656
:101C680022C44AC09734000083A444B46389041092
:101C780003A4C40AAA86054525C43C241307700A90
:101C88006392E70858301C34172900001309C97AF1
:101C980003268900B387E7020357C900B387E70221
:101CA8001307003293870719B3D7E70203A744093C
:101CB8003E97BA846364F7006364C700B304C740FF
:101CC8009727000083A7C75384C28297B387A4408D
:101CD80063F5A40003278900BA9789EB1305F00F71
:101CE800B24022449244024941018280583093060E
:101CF800204E3307D702E3F3E7FE930780FA3CA4AC
:101D08000145F9BF1307800AE39AE7FC972700000B
:101D180083A7074F82972A893545EF20E025AD47ED
:101D280017370000232EF7C658301C34172600003A
:101D380013068670B387E7025A261046B387E70270
:101D48001307003293870719B3D7E70203A744099B
:101D58003E97BA866364F7006364C700B306C7405A
:101D6800E31ED9F617D505E0130585D6EFE07FD237
:101D78009727000083A7C75A0947F8D785B70545AD
:101D880085B7397156D2973A0000938AAABF83A7BC
:101D98000A033707080026DA06DE22DC4AD84ED6C0
:101DA80052D45AD05ECE62CC66CA6AC86EC6F98F63
:101DB8009734000083A4849F638A071C83A9C40AFC
:101DC80083C7990003A4C90092073E942820B1470D
:101DD80005053305F5025E203E9533450508EFE01D
:101DE800EFF1AA8C630F051A130DC5002324A50172
:101DF80034203146370B0300B386C6022313040090
:101E08000149172A0000130AAA51972B0000938B47
:101E18002B50972D0000938DAD51130B8B15054C4E
:101E2800EA9654C483C679009307D00783250A002D
:101E3800B386F602C1679CC5370833008606B4D15D
:101E480083A60B0090421376F6CF90C29042137689
:101E5800F6CF1366062090C203A50D001045336621
:101E6800060110C503A6090023A8650593055002BD
:101E780090C672205444B2962324DD0014300146E3
:101E8800CA96A301DD0003C504089736000023ADF8
:101E980006AEEF00901C83260A00CC46139615491F
:101EA800D0C60F10000083260A003706020090C62D
:101EB8001306000823A8CA0003A60B0010421356F5
:101EC8007648631E860B1306E018F0D2CCC6173688
:101ED8000000232306AC17360000232706AA23A0F8
:101EE8008601A125EF20200183A64A00858AD9CA48
:101EF800EA85268597E005E0E780A0C70DE9034657
:101F08005D0049C276204E20B29663DDB606B4283D
:101F1800AC4803258D00918E8906B695EFE0CFED8C
:101F280023020D0003465D007620B29676A00326B4
:101F38000A00310D3452FDFE342005091379F90FDA
:101F4800E362D9EE9C246685A381FC001C20A38251
:101F58000C002383DC002382FC006254F250D2542C
:101F68004259B259225A925A025BF24B624CD24CF5
:101F7800424DB24D2161172305E0670023D91306AE
:101F8800E01AA1B7FD562302DD0055B797270000D8
:101F980083A70739FC5791C7854717270000230DEA
:101FA800F724F2506254D2544259B259225A925AE2
:101FB800025BF24B624CD24C424DB24D21618280A1
:101FC800797122D426D22E84AA84414697C506E088
:101FD800938545CD0A8506D6972004E0E780003E24
:101FE800414697C506E09385E5CB0808972004E0AD
:101FF800E780C03C3C3010088A85DC875C20268559
:102008005C875C30DC86973006E0E780C07F03475A
:10201800F1011C200145631EF7000347E1011C3054
:1020280001456318F7000345D1013C201D8D133588
:102038001500B2502254925445618280011122CC7D
:1020480026CA4AC84EC606CEAA841724000003240E
:10205800A47C13092500854905C09C303830858B40
:102068006304F700405CCDBF1946930544004A85D8
:10207800EFE00FEAE31835FFF24022856244D244CC
:102088004249B24905618280411122C426C24AC030
:1020980006C6172400000324247893042500054964
:1020A80001E8B240228522449244024941018280DB
:1020B800A6851305A4022937E30525FF405CCDB7A3
:1020C800411122C426C24AC006C6172400000324B0
:1020D800A47493042500054901E8B24022852244EE
:1020E8009244024941018280A6851305A401C93D95
:1020F800E30525FF405CCDB7011126CA644122CC17
:102108004AC84EC652C406CE2A841D49930965059D
:10211800054A3C4463E4F4000545A1A05834DC209A
:1021280063192705034784026304F7008440D5B781
:10213800D83083475405E31BF7FE19469305640519
:1021480013856400EFE0CFDC8547E311F5FED82462
:1021580083479402E31CF7FCFA243E34E318F7FCA7
:102168000145F2406244D2444249B249224A0561DB
:102178008280E31DF7FAD83083475405E318F7FA4D
:102188001946CE8513856400EFE08FD8E31045FB30
:10219800C1BF411122C406C626C24AC01724000086
:1021A8000324C4625DC88347840B1307700A6393D2
:1021B800E7080347140E8347A40B172900001309E7
:1021C800A92783268900B387E7020357C900B38785
:1021D800E7021307003293870719B3D7E7020327EB
:1021E800440A3E97BA846364F7006364D700B30473
:1021F800D7409727000083A7A70004C18297B38719
:10220800A44063F5A40003278900BA9785CB034748
:10221800140E9306204E3307D70263F1E7029307A3
:1022280080FA230CF40A0145B24022449244024940
:10223800410182801307800A639EE700172506E0A4
:102248001305E576EFE0FF849727000083A7470D85
:102258000947F8D71305F00FC1BF0545F1B70111BC
:1022680022CC26CA06CE2AC42EC617240000032470
:10227800245A854419E001450DA09C841830858BAB
:102288006304F7000044FDB719469305A100130540
:102298002400EFE0EFC7E31795FEF2406244D24412
:1022A80005618280EFE0BF8273000000000000003B
:1022B80097220000938242F40383020023800200E5
:1022C800630F0300F32510342EC097050000938593
:1022D800A5FD73901534EF0080617300203086DC13
:1022E800EF00E060E6508280000041114AC01729E3
:1022F80000001309E9010327090026C206C61C5F6E
:1023080022C4972400009384640093D76748C1C708
:10231800930700061CDF172400001304A466184C5A
:10232800930700086317F7009C409C4393F7070442
:102338001CCC1C4093F7070499CB9727000083A770
:1023480027EC829748D81C4093F7F7FB1CC01C4029
:1023580093F7070299CF1C4017270000032747FC73
:10236800B706080093F7F7FD1CC05C5414C786072E
:102378007CD71C4893F7070499EF85475CC8370753
:1023880002009727000083A7A7F998C71307000C36
:1023980018C81854F8D383270900985F135747487B
:1023A80005C3985F1367070198DF9727000083A785
:1023B80027F723A20706854717270000232CF75C79
:1023C8009C40D8431357174819C7D843759BD8C39F
:1023D800D843799BD8C3B240224492440249410170
:1023E8008280213773002030972700009387875910
:1023F8003707040088DB698F11CF172700000327F0
:1024080027F2FD5634D797260000938666FBD84EF0
:102418000507D8CE137785000DC398479726000087
:1024280083A606EF1367170098C71307000898CB11
:10243800D856719B13671700D8D61377150011CF9C
:10244800D8439726000083A6A6EC13671700D8C3C5
:10245800D856719B13671700D8D6137765000DC33C
:102468001377450059C798431367170098C39726F1
:10247800000083A6E6E9D856719B13671700D8D6E3
:102488004167698F0DC39726000083C6E633C18A6A
:10249800172700001307072CB5C28346470793E6A2
:1024A8000602230AD70637070200698F11CF984B17
:1024B8001377070819C3054798CB9727000083A708
:1024C80027E63707020098C7B70708007D8D0DC1BA
:1024D800172700000347572F058B9727000093877E
:1024E80067271DCB03C7570713672700A38AE7068B
:1024F8008280D84713671700D8C795BF8346470718
:102508000946BD8A6388C600834647070D46BD8ACB
:10251800E39BC6F8914671B703C75707118B69DB70
:1025280003C7570713678700D1B79726000083A60C
:1025380026DF172700001307E7441C43858B91E724
:102548005C43858B99E3FC52EDFB9727000023A59C
:102558000744828097260000938686DB2A87884274
:102568001C5D93D75748C1EB81C51C59BD839CA1FD
:1025780015C69C42945BC60693D7660163D60600CF
:1025880093E707C0B3C707088316060093975760F9
:10259800A9CABE968947B3C6F60216A297270000B5
:1025A80083A707D8BC4B083393D757488DCF29C585
:1025B8009726000083A6863E93F6060493079500A7
:1025C80009459DCABA979C230547194593F6F7060E
:1025D8006394E60201459397476063DF0700394536
:1025E80082801EA265BF2A9748331375F5077D15AB
:1025F8003335A0008280054582809727000083A795
:10260800A7D199CB944BD04B9842518F98C2944301
:102618009C479842D98F9CC217260000130646D0C3
:10262800054818429726000083A686CE9727000003
:10263800938747356314050503A80600136808083F
:1026480023A0060183C62702B3C5D5205447938526
:10265800A50C13981649232607010F1000001842ED
:1026680037060200860510C71306000890CB6CD306
:1026780054C797270000238FA7C882808842137504
:10268800F5F788C283C62702B3E5D520544793855A
:10269800E50E1395164948C70F1000001842370673
:1026A8000200860510C71306000890CB6CD354C7E8
:1026B8000945C1B7411122C4AA8706C626C22E857C
:1026C800172400001304C4C5B285CDEB1C40F85391
:1026D8007DFF3707020098C79727000023A8072A1D
:1026E80097240000938444D0DC5085C7B7E700E006
:1026F8003707200023A0E728B7F700E0938707D023
:10270800984B6D9B98CB984B1367870398CB7300B6
:102718005010E5359727000083A787BF9843131704
:10272800772998C3D857719BD8D79727000023A536
:1027380007269727000023A907241C40094798C3A8
:10274800DC5099CB37F700E0832707D193E7870060
:102758002328F7D0730050101440172700001307E0
:1027680067221C47858B91E75C47858B99E3FC5270
:10277800EDFBB24022449244410182800D476390B0
:10278800E7069727000023A307209727000023A127
:10279800072097240000938424C5DC5085C7B7E739
:1027A80000E03707200023A0E728B7F700E0938769
:1027B80007D0984B6D9B98CB984B1367870398CBA2
:1027C800730050101D3D9727000083A767B49843F6
:1027D8001317772998C3D857719BD8D795B705474A
:1027E800E39CE7F697260000938606C0DC5285C76F
:1027F800B7E700E03707200023A0E728B7F700E095
:10280800938707D0984B6D9B98CB984B136787039A
:1028180098CB730050101C40D04713171649D8C7DF
:102828000F1000001C403707020098C71307000864
:102838009725000023A0E51617270000032747ADBA
:1028480018431357774819C71307E018F8D3D0C7A8
:10285800DC52C5BD1307E01AD5BF9727000083A730
:10286800A7AB89CFD44303A88700984233670701F1
:1028780098C2D447DC4B9842D98F9CC2054797270A
:10288800000083A7E7A895056310E504984313673C
:10289800070898C3984F137707C01367A71398CFF3
:1028A80013078007B8BB939735009387C70317278B
:1028B80000001307270D1CD797270000238CA7A417
:1028C80019C2060610D78280984309451377F7F78F
:1028D80098C3984F137707C01367271398CF130728
:1028E800F007B8BB939745009387C703C9B79727E5
:1028F800000083A7E7A28847D847798D01C988C710
:102908009727000083A787A191C382878280896760
:10291800172700000327C7A0938707F47CD39726BF
:10292800000083A6E6A083A7060993D7A74991C705
:1029380083A7060993D7974999E37C53EDF78280DB
:10294800411106C622C426C24AC063030510AD471A
:102958002A8463EAA70C1304F5FF1374F40F138594
:10296800F5FF01469305F00F1375F50FFD35972414
:1029780000009384E49B98401729000013094999A3
:10298800136404045C571374F40717050000130557
:10299800250DF59B5CD7032709001C4393F707F81F
:1029A800C18F1CC3B7477671938797121CC7B75757
:1029B80055009387575517240000130464965CC389
:1029C80018409727000023AF07FA5C43F99B5CC3C4
:1029D800A547172700002325F7FCEFE08F8B14404D
:1029E8009727000023AA07FA9727000023AE07F8C5
:1029F8000327090085479CC21C433706330001455D
:102A080093F7F7CF1CC31C4393F7F7CF93E707203F
:102A18001CC398401C47D18F1CC7B7070300938776
:102A28008715BCCA05A0B1476307F5029307600282
:102A380063E5A7001304E5FF0DB793077002494546
:102A4800E30FF4F0B24022449244024941018280EB
:102A58001304500229B71304600211B717270000A6
:102A6800032787F2058B972700009387A7CE01CF0E
:102A7800172700000327C789185F1357574801E72E
:102A88009A2705079AA703C68703EC33C8234DBDC9
:102A9800411122C406C626C24AC02E849DCD13F910
:102AA80015008147414763040904131745003E9701
:102AB800B1463307D7029714000083A46475B3178F
:102AC800F02833C90708BA949C40C840829723A0CD
:102AD800040023A2040033448900B2402285224422
:102AE8009244024941018280B356F448DDFE8507CD
:102AF800E39CE7FECDB7011126CA06CE22CC4AC810
:102B08004EC6AE84B1C593F7150001444147A1CF25
:102B180093174500A2973147B387E702971900003A
:102B28009389096F03A909003E998327090081C782
:102B380003254900829731473307E40283A7090038
:102B4800BA979C478DC733148028B3470408BD8CB7
:102B5800F24062444249B2492685D24405618280E6
:102B6800B3D68448D5F60504E31CE4FECDB723208C
:102B7800090023220900C1BFAA87171500000325F1
:102B8800A56811E182803A216315B7001821E30B8B
:102B9800F7FE4845FDB77971B7E700E022D48043D6
:102BA80052CC06D626D24AD04ECE56CA5AC85EC68F
:102BB80062C43A8A37072000798C23A0E7180F10DF
:102BC800000005E123A087100945B2502254925411
:102BD8000259F249624AD24A424BB24B224C4561F1
:102BE80082809717000083A7A761B6892A89AE8AD1
:102BF800328B971B0000938BAB61829703A70B0066
:102C08008144B146C147338CD40233068701104250
:102C180041E2C165938505F04145EFD06FEE19EDAE
:102C28009717000083A7477F81C781451145829781
:102C3800B7E700E023A087102D4541BF1717000014
:102C48001307875C1C43A1E308C323000500B317DF
:102C580090283EA183A70B002326050023246501A5
:102C680023224501E29723A0270123A2570123A489
:102C780047016384090023809900B7E700E023A097
:102C88008710014599B73E87DC47F5FF48C775BFF0
:102C98008504E39AF4F6B7E700E023A087102145FE
:102CA8002DB7B7E700E09843B706200023A0D71850
:102CB800758F0F1000009716000083C67670637337
:102CC800D5029716000083A666543325D520162111
:102CD800D58D0EA19716000023AC066E23A0E71031
:102CE8000145828023A0E7100D4582800111B7E7D6
:102CF80000E022CC80433707200006CE26CA4AC807
:102D0800798C23A0E7180F100000BD4763E9A704DA
:102D180031473307E5029717000083A7674FBA9733
:102D28009C4395CF3315A0282E89B3450508014546
:102D38002EC69935AA8409C9B2450145972004E0F1
:102D4800E780608F23A42401B7E700E023A0871061
:102D58000145F2406244D244424905618280B7E7A6
:102D680000E023A087100945EDB79726000083C629
:102D7800A6999717000083A7275201476394E60096
:102D8800014582808E23138687026394A5003E85C1
:102D9800828005071377F70FB287CDB79727000012
:102DA80083C79796AA868507171500000325854FC0
:102DB800014712216307D60005071905E36BF7FEE3
:102DC800014582802A87171500000325254E11E149
:102DD80082801C45B227636BC70003584500B306C1
:102DE800C8006355D7008146639406010841C5B7FA
:102DF80003D3A700938807016316E30091C192A14A
:102E08003E8582808506C687B3C60608F1BF972629
:102E1800000083C6668F9717000083A7E74B01471A
:102E28006394E60001458280AE231386C70363944A
:102E3800A5003E85828005071377F70FB287CDB7C7
:102E4800411122C406C697270000238F079617143E
:102E580000000324644905C06C390145B315B02846
:102E6800B3C50508972004E0E78000CA9307102738
:102E78003305F50202942244B240814501454101DF
:102E88006FD09FC2411106C6383D19C7342563105B
:102E9800D704B24041016DB73C2DE5DF3825E30A80
:102EA800F7FE3CA5814517E5FFFF1305C51CEFD0CC
:102EB800BFBF9717000083C7275999C79717000006
:102EC80083A707465147F8D3B240410182803C2D81
:102ED80089C7E398F6FC38A5F1B7C5FEEDBF4111E7
:102EE8004AC0172900001309E9A98327890022C4C9
:102EF80026C206C6972400009384C485858BE050BB
:102F08009DCB9727000023A307A883C74407C18B3D
:102F180085CFEF00507E83C7440793F70702E5DFAC
:102F280083C74407228593F7F70C238AF406974052
:102F380005E0E78040FCEF00107C22852244B24087
:102F4800924402494101EDBD83C75407858B91CB5B
:102F5800EF00707A8D47230EF406BC5822858297BD
:102F6800D9BF83C744071547BD8B6395E7048347DB
:102F7800B406034534060146930550025D8DEFF013
:102F8800DF8D014681450545EFF0CFF28327C90063
:102F9800858BD5D322859727000023AB079E9740C2
:102FA80005E0E78000DD41F9B2402244924402493D
:102FB8004101828083C744071947BD8BE39DE7F62B
:102FC8008347B406034534060146930550025D8DD8
:102FD800EFF0BF88014681450545EFF0AFED832747
:102FE800C900858BA9DB22859727000023A2079AB1
:102FF800974005E0E78020B17DB7411122C426C281
:1030080006C67C2578452A84BD8B1CA91CA31D47B0
:103018006445639BE7340547B8A08347F5058D46AB
:103028006395D7185E2DCDE37C491147B18B638D2D
:10303800E70831476398E700034715068347F50714
:103048006304F7088547BCB01946930564031385E4
:103058004400EFD06FDABC20990793F7F70FBCA0B4
:10306800034704061377070401CFB8301367070432
:10307800B8B07844BA975838B8B3BC208507BCA014
:103088009717000023820774BC2013F7F70305077E
:1030980018B80347E4051A07D98FBCA0834754031F
:1030A800858B91E70347440389476317F700784402
:1030B8001C2393E707041CA37C44183898B3B24038
:1030C8002244924441018280A147BCB08357C40680
:1030D8009715000093850568171600001306462407
:1030E800DCA08357C406034714067444A18312075F
:1030F800BD8BD98FDCB2B4208547890693F6F60FCD
:10310800B4A0171700000347276C631EF706183C86
:103118009387E6008E07231AF4069387C708B387B8
:10312800E702794510420948238A0507C1650CC69C
:10313800938707FBB3C7070893877716B3C7A70218
:1031480033C70708B387A70286073CD2BC3093E78A
:103158000701BCB07C44B6978346240693E6060470
:10316800B4B3B4207C44B697D8A3B4207C4421835C
:103178007D8BB697834634069606558FD8B3BC2008
:103188008D07BCA011B71042F94738520583335751
:10319800F7023C5268528583FD8BAA977CD28D47F3
:1031A800238AF5063347070855B71946639DC712A2
:1031B8005E2DC1E393056503B8B013854400EFD0D5
:1031C800AFC3BC201385A4009907BCA0BC3093E70B
:1031D8002700BCB083475403898B95CF0C58BC2972
:1031E8009DCB1946D105EFD02FC178441C2393E716
:1031F80007F81CA3BC20990793F7F70FBCA0034757
:10320800040613770704E30D07E6B430784493E621
:103218000604B4B085B58347D40391C778441C230A
:1032280093E707F81CA319469305E403EFD0CFBC36
:10323800D1B7A147BCB08357C506DCA08357C506E4
:10324800034615066C45A1831206BD8BD18FDCB1F0
:10325800B020171500001305E54F9715000093855A
:10326800250C09061376F60FB0A09717000083C740
:10327800A7556398E704183C9307E6008E07231ABE
:10328800F4069387C708B387E70279488946230A73
:10329800D5069441C1658CC6938707FBB3C7070859
:1032A80093877716B3C7070333C70708B38707039E
:1032B8008607BCD2BC3093E70701BCB07C44B29708
:1032C80061BD8C41B851F94705833357F702BC51AA
:1032D80003A845068583FD8BC297FCD1230AD50632
:1032E80033470708C1BFA147BCB08357C506DCA058
:1032F8008357C506034615066C45A1831206BD8B88
:10330800D18FDCB1B020171500001305A5440906BC
:103318001376F60FB0A09717000083C7E74A9715F2
:10332800000083A5E5FFE39FE7F8183C9307E60054
:103338008E07231AF4069387C708B387E702F9466E
:103348000948230A0507416588C5938707FBB3C762
:10335800070893877716B3C7D70233C70708B38719
:10336800D7028607BCD1B9B70547639EE706B147C0
:103378001CB983475503898BA1CB0C59BC29A9C714
:103388001946D10513858400EFD00FA778441C2374
:1033980093E707F81CA368441946930564030905D5
:1033A800EFD08FA511679717000083A7A747F98F5C
:1033B800E38607CE7C24B98BE39207CE78441C239E
:1033C80093E707021CA3D9B98347D40389C79C2074
:1033D80093E707F89CA0684419469305E403210580
:1033E800EFD08FA14DBF522D0C559307660093F770
:1033F800F7031CB913858400E5B7011126CA971491
:103408000000938424589C4422CC06CE1714000054
:1034180013044434858B6850D9C32AC69717000013
:1034280023A60756EF00302D034744078947324546
:103438006307F700034744078D47631EF702971693
:10344800000083A6E6EDBC520357450785831307A2
:10345800C71263F2E702BC528583B1C391470347A1
:103468004407E31EF7FE6244F240D2440561174365
:1034780005E06700A3D1382D3C3D09CF3425630909
:10348800D7026388F60238A56244F240D244056147
:103498006FD03FA599CF382509EF3CA5F5B72AC6C7
:1034A800EF00702562443245F240D244056149BAC2
:1034B800EDF7DC4CEDF70347440789476307F7004E
:1034C800034744078D47E31CF7FC9147034744072C
:1034D800E31EF7FE49BF63000532011122CC06CE78
:1034E80026CA4AC84EC652C456C2582585472A8499
:1034F8006318F72C971700009387C748D44F1547D0
:10350800638AE600D44F0D476386E600D84FAD477F
:103518006312F7026C386244F240D2444249B2491D
:10352800224A924A01450561B315B028B3C505087A
:103538006FF02FF716311307006497140000938477
:1035480064213347D7029C20E8D0850793F7F70F0B
:103558009CA063CAE700972004E0E780E0A09717E3
:1035680000002389071E78249D47631FF7048347BB
:103578009406B1C38356040763ECF6020C24930740
:1035880030041CAC1305300493F6F60F014697700F
:1035980006E0E78020BA22856244F240D2444249DC
:1035A800B249224A924A0561174305E06700036E53
:1035B80085062318D406930530020545972004E0B4
:1035C800E78060932301A4060549238A2407183C51
:1035D8008D47631CF70E971004E0E78040FC0D89C7
:1035E800630F051463162517930760023CA493071D
:1035F80050023CAC9307700278243CBC85476302B8
:10360800F70889659385F57013051027171A0000C8
:10361800130A8AE283497401972004E0E780209026
:103628000E30835ACA002A8913060064B3855503ED
:10363800814613850532B335B50097A006E0E780CB
:10364800A02AAA84B335590337460F001306062467
:1036580081463305590397A006E0E780E0288327D1
:103668000A00AA948297B307950003278A00BE85AB
:1036780063E4A70063E4E700B385E7404E85EFF015
:10368800EFE683475403898BE9CB8347C403F1C72B
:103698000C58E1C5BC25F1C38947230AF402194631
:1036A800B10513056403EFC03FF50347C407894715
:1036B80063E9E70A22856244F240D2444249B249AA
:1036C800224A924A05616FD0DF8189467C346315AE
:1036D800D70213F7170019CB898B1307500291EB08
:1036E8009307700238A43CAC814739B713076002CE
:1036F800C5BF93076002FDB799CF93F6170013076C
:10370800500291E6898B13B717001307670238A494
:10371800230D0400D1BF3C2C130740026368F70057
:10372800930750023CAC3C2C3CA47DBF850793F723
:10373800F70F3CAC13077002E364F7FEEDB713070D
:103748007002930750023CAC38A4930760026DB531
:103758001307500293077002FDB78547230AF40246
:10376800A9B70327C40A9716000083A666A93C27B1
:10377800ADC31C375833971400009384E4CB9044AE
:10378800B387E702DA24B387E70213070032938787
:103798000719B3D7E702032744093E973A896364B8
:1037A800F7006364C7003309C7408296B307A9408E
:1037B8006374A9009844BA9703576407E3FCE7EEDB
:1037C800F2406244D2444249B249224A924A0561CF
:1037D800828083248409829663E9A400835764075E
:1037E8003385A440E378F5ECE1BF9717000083A781
:1037F80027C5BE94E5B7828001114EC6971900000F
:10380800938949F522CC03A4C9094AC817190000AD
:10381800130989C20357C90026CA83546408832739
:10382800040906CEB384E40237470F009306F72352
:103838001307072452C456C25AC0B694B3D4E4023C
:1038480063E09704171A0000130A8A9BB384974011
:1038580083270A00829763E9A4023385A440634959
:10386800050283570404A30F040085072310F404FA
:1038780083470414639E07102285EFD0DFBE21AA78
:1038880003278900BA977DBF83278900BE94F1B7C3
:1038980083270A008297032784086366E50A198D3F
:1038A8007E3C0357C9008E07B387E702130700322F
:1038B80093870719B3D7E70263ECA708B74A0F0045
:1038C800138BFA23938A0A24835704048507231049
:1038D800F4048347041481E72285EFD0DFB82285FA
:1038E800975005E0E78000246317052403260409A0
:1038F8000327C408832689003297BA876364C70000
:103908006364D700B307D740783C0356C90023281F
:10391800F408050778BC035764083307C7025A97A9
:1039280033575703B384E74063F5E700998EB384B0
:10393800F60083270A00829763E6A4043385A4402F
:10394800E34405F839BF83278900998F3E9589BFDD
:10395800A1452285975005E0E780E014A305A4025D
:103968009717000083A747AB6387071C6244F240A0
:10397800D2444249B249224A924A024B89451545E6
:103988000561828783278900A6973385A7404DBFA5
:103998002285EFD09FB72285975005E0E7808018F1
:1039A800631B05180355C90083576408B7460F0001
:1039B8001386F623B387A7029386062403270409F0
:1039C800230B0402832A8900B297B3D7D702636E08
:1039D800F716B307F7408326C4082324F408014BDD
:1039E800B387E600BE8463E4D70063E45701B38479
:1039F80057411E3023289408A1CB835604045A301B
:103A080037460F0056B03387E640B387E7023A30AF
:103A18001306062481468145BA97B3C7070833853C
:103A2800A7023EB097A006E0E78000EC11CD2695EE
:103A3800B3349500A695AA876314BB006364550147
:103A4800B30755412328F40883270A008297AA84DC
:103A580083270A008297E30D95FE83270A008324B3
:103A68008408829763E8A40E3385A4406301051097
:103A7800035AC90083576408B7440F001387F42317
:103A8800B387470393840424BA97B3D797021717C9
:103A980000000347F796BA9763EBA70CB335950276
:103AA800835A2402528681463305950297A006E080
:103AB800E78080E33389AA0033854A0337460F003D
:103AC800130606248146814597A006E0E780C0E1F9
:103AD80015C1B337950252868146B385B402338542
:103AE800A402BE9597A006E0E78000E0B38AAA404A
:103AF800231154033545492123AE890838348547B5
:103B0800631EF704930700FD7CA481451705000098
:103B18000325457FEFC05FF995471717000023215C
:103B2800F7E8370710009707000083A7677F98C753
:103B3800060923A82707F2406244D2444249B24901
:103B4800224A924A024B05618280B3065701B38725
:103B5800F64051B583278900BE9439B7930710FC06
:103B68007CA48145170500000325457965B797179B
:103B7800000023AF07C6834709019DC3170500004E
:103B88000325C576EFD00F96624483274900F2409B
:103B9800D2444249B249224A924A024B056182877D
:103BA800834594026244F240D2444249B249224ACF
:103BB800924A024B01450561B315B028B3C5050803
:103BC8006FF02F8E011122CC26CA4EC606CE4AC8E7
:103BD80052C456C25AC038358547832405092A84F9
:103BE800AE896314F70C83570508835AC503171A5F
:103BF8000000130A6A84035BCA0063FE571914297C
:103C0800639BE61803278511631707180327450ADE
:103C18006313071874351D47639FE6162A3DB38A58
:103C2800FA409307204E33055503032944093746C4
:103C38000F001306062481463305F5029707000096
:103C480083C7077C33592503B335AB023E99334903
:103C58000908231324093305AB0297A006E0E7807F
:103C6800A0C8B307950033B5A7002E9503278A008F
:103C7800BE8419E163E4E700B384E740B30769034E
:103C880037470F009306F7231307072423A099004B
:103C9800B697B3D7E702D69763E4F4009D8C31A0BA
:103CA80003278A00B307F740BE94170900001309D9
:103CB80029558327090023A09900829763E2A4105D
:103CC8003385A440635D050A83270900170B0000AC
:103CD800130B8B76829703A709006369E50E198D8C
:103CE8007E3C0357CB008E07B387E70213070032E9
:103CF80093870719B3D7E70263EFA70C374A0F007A
:103D0800930AFA23130A0A24835704048507231005
:103D1800F4048347041481E72285EFD0CFF4228589
:103D2800975005E0E78000E061E5832604098327D2
:103D3800C40803278B00B697BE8463E4D70063E406
:103D4800E700B384E7407C3C8356CB0023289408E3
:103D580085077CBC83576408B387D702D697B3D747
:103D6800470363E6F40A9D8C8327090023A0990082
:103D7800829763E1A40A3385A440E34705F89707CF
:103D8800000083C7F76763E6A7069717000023A11B
:103D980087A60145B9A88357640837470F009306DB
:103DA800F723B387670313070724B697B3D7E70248
:103DB800E3F6F4EE03278A002697B304F740F5B537
:103DC8009707000083A7C767BE94DDBD83278B00D4
:103DD800998F3E9531B7A1452285975005E0E78038
:103DE80080CCA305A4029707000083A7E76281EFB0
:103DF8007D55F2406244D2444249B249224A924A2D
:103E0800024B05618280894515458297D5B71D8F7C
:103E1800BA9499BF83278B00BE94B1BF970700005F
:103E280083A7074F98433706CEFF7D161377F7CF42
:103E38001367071098C3170700000327674F144735
:103E4800370803001375F51FF18E14C79706000095
:103E580083A6064D23A8060523A40700904B93F5D7
:103E6800F507130888151366F60390CB904313667D
:103E7800060890C3F04F137606E0498EF0CF23ACC6
:103E8800070423A007065057759A50D79043137616
:103E980006F84D8E90C31306401FF0D21716000087
:103EA800232C06AE17160000232006AE054690C246
:103EB8009043B70533001376F6CF90C3904313763B
:103EC800F6CF1366062090C310474D8E10C723A85F
:103ED8000605D8531317F728D8D32547F05201C63B
:103EE800B04FE37DC7FED8531317F748D8D3A8536C
:103EF80013354500828097060000938666429C42EF
:103F0800B84B1377F78FB8CB98431367870098C3DC
:103F18009C4393D7374889C701000100010001007D
:103F2800170700000327C73E1C4393F7F7CF93E713
:103F380007101CC3170600000326863F1C463707D8
:103F4800CEFF7D17F98F1CC69C4237070300B8CBFC
:103F58009707000083A7473C99CBD44390479842E2
:103F6800518F98C2944BDC4B9842D98F9CC29717BB
:103F7800000023A707A282809707000083A7473A7B
:103F88009C438D8BF9C74111B7E700E04AC003A9EC
:103F9800070026C23707200006C622C4AA84337940
:103FA800E90023A0E7180F100000171400001304FD
:103FB800649D584C8D47631AF7009707000083A744
:103FC800E775014681454545829719476393E4049F
:103FD8008347140289CB8347040263969700971797
:103FE8000000A381079C584CA1476315F70093076D
:103FF80080101EB09707000023800720ED3DB240D7
:104008002244B7E700E023A0271192440249410166
:1040180082809D47639BF40083471402E9D70347D6
:1040280004028D47E311F7FC5DBF544C6389E60039
:10403800584C6306F700584CA147E31DF7FA83472D
:104048001402CDFB5C4C2300F4028547A300F40264
:1040580055B78280411122C42A84354506C6293FB6
:1040680049CCAD4763E987067D141374F40F9707AD
:10407800000083A7E72B984BB70600C1FD16137401
:10408800F403758F6204418F98CB984B9706000014
:1040980083C6C636717693F6F6031306F60FA206A4
:1040A800718F558F98CBF84FB706F9FFFD16136738
:1040B8004700F8CF984B0145758F1317172998CBF0
:1040C800370702001307874F98C7B1471717000033
:1040D8002328F78C39A8B1476304F40293076002D8
:1040E80063E48700791451B7930770024945E300E8
:1040F800F4F8B2402244410182801304500285BF83
:0841080013046002ADB70000D2
:104110002A8309CA83830500230073007D160503E3
:1041200085056DFA82809707FC1F83A7A7E1170713
:10413000FC1F0327A7E001456313F7008280F623E5
:1041400099E2D62336959C43C5BF1707FC1F13077A
:1041500027FF1C435A23411193860711E117BA9791
:1041600085651706FC1F232FD6DC1706FC1F2327A7
:10417000F6DC06C69D051356370063F4E50013060A
:1041800000203387C6009705FC1F23ABE5DA6116D4
:1041900098C2D2A2239306001CC3998FE1175EA395
:1041A000231307004937B2409707FC1F2399A7F64E
:1041B000410182809707FC1F83A7C7D81707FC1F00
:1041C0000327C7D701456313F7008280F62381E6F2
:1041D000D6233375D50A9C43FDB7184183A785FFC5
:1041E0006319B7001CC1FD5723AC05FE238FF5FEF4
:1041F0008280232CF6FEC5BF411122C437E400E0C3
:1042000026C204403707200006C6F98C2320E41894
:104210000F10000009E9232094101545B2402244F4
:104220009244410182800347E5FF9307F00F630644
:10423000F700232094101145D5B797C0FB1FE780E6
:1042400000EF014523209410D1BF41114AC037E946
:1042500000E022C403240900B707200006C626C2D6
:104260007D8C2320F9180F10000089E52320891088
:10427000154515A0AA849707FC1F83C7F7E92E856B
:1042800063F5F400894763EE9700BD37B7E700E0B8
:1042900023A087100D45B2402244924402494101B7
:1042A000828083A785FF99E703C7E5FF9307F00F97
:1042B0006308F7009137B7E700E023A087104DBFF0
:1042C000238F95FE1705FC1F130505C897C0FB1F1C
:1042D000E780E0F6A165268597E0FB1FE780207266
:1042E00001452320891045BF9707FC1F23AE07C453
:1042F00082804111B7E700E026C2844337072000DF
:1043000006C622C4F98C23A0E7180F1000009707F7
:10431000FC1F83A7E7E41704FC1F130424BA91C70A
:1043200082971C40AA971CC031A09707FC1F83A747
:10433000A7C2FDF70840B74703009387D73F33056F
:10434000F502B7A72600938737ECB2403E9508C028
:104350002244B7E700E023A09710924441018280F5
:10436000411122C406C69707FC1F83A7A7BE1704E6
:10437000FC1F130464DA89C782975C48AA975CC85B
:104380004848B240224441018280B7E700E09843A8
:10439000B706200023A0D718758F0F1000009706CE
:1043A000FC1F83C676D76370D5029706FC1F83A6D1
:1043B00066BB3325D5201621B3F5B6400EA123A048
:1043C000E7100145828023A0E7100D4582807971B6
:1043D000B7E700E026D284433707200006D622D470
:1043E0004AD04ECE52CCF98C23A0E7180F10000013
:1043F000930705FF93F7F70F7D476363F70A31478C
:104400003307E5029707FC1F83A707B6BA979C43BB
:10441000C1CB135445003D893315A028AE89B3455F
:10442000050822852EC697E0FB1FE780A04A2A894F
:1044300039C9B2452285170AFC1F130A6AD5B1375C
:104440009707FC1F83A747B182978357CA002A8426
:1044500081463387370313060064B3B73703130568
:104460000732B335E500BE95EF90421DB3078500D6
:1044700083268A003E8763E4A70063E4D70033877E
:10448000D7402324E900B7E700E023A097100145B7
:10449000B250225492540259F249624A45618280D4
:1044A000B7E700E023A097100945DDB7797122D462
:1044B00037E400E04AD003290400B707200006D6FD
:1044C00026D24ECE52CC56CA5AC85EC63379F900AF
:1044D0002320F4180F1000009707FC1F83C7D7C3D1
:1044E0006378F500970BFC1F83AB0BA763970B005A
:1044F000B7E700E023A0271199A0970AFC1F938A31
:104500002AC903AB8A00B74736FE938707C83E9B8C
:1045100083D7CA002E8AAA84B385C702B28981468E
:10452000B3B7C70213850532B335B500130600646F
:10453000BE95EF90A2106370AB02232024110145B9
:10454000B250225492540259F249624AD24A424B22
:10455000B24B45618280829B83D7CA002A841306AE
:104560000064B38537038146B3B73703138505323B
:10457000B335B500BE95EF90620CB307850003A775
:104580008A003E8463E4A70063E4E7003384E740E5
:10459000D285268597E0FB1FE780C03301C900C59F
:1045A000B7E700E023A02711054559BF93E504F0C4
:1045B0004145B3C5050897C0FB1FE78020AA11E954
:1045C0009707FC1F83A7C7BA85D7A6851145829791
:1045D00005B71707FC1F1307A7981C4389EF08C3EB
:1045E00085472326050000C52311450104A11CB100
:1045F0002322050075B73E87DC47F5FF48C7CDB7D6
:104600007971B7E700E026D284433707200006D649
:1046100022D44AD04ECE52CC56CA5AC85EC662C4C4
:1046200066C2F98C23A0E7180F10000035C12A8953
:104630002E8AB28AB6894144B14C170BFC1F130B6A
:10464000AB92130C0003B30B940383270B00DE978C
:104650009C43B9EF135544409375F4005686137587
:10466000F50FB315B028B3C50508893531C18327C7
:104670000B00DE9723A0270123A2470163840900D2
:1046800023808900B7E700E023A09710014521A00F
:1046900023A097100945B250225492540259F2496E
:1046A000624AD24A424BB24B224C924C45618280C4
:1046B0000504E31A84F9B7E700E023A09710214529
:1046C000D9BF011122CC37E400E026CA04404AC811
:1046D0004EC652C406CEB70720002A892E8AB28958
:1046E000FD8C2320F4180F100000C933D2854A85B1
:1046F00097E0FB1FE780001E01ED23209410214569
:10470000F2406244D2444249B249224A0561828061
:104710009707FC1F83D787A8B38537032A89130619
:1047200000648146B3B7370313850532B335B5004E
:10473000BE95EF80B2702322A9002320941001457A
:10474000C1B7011126CAB7E400E04AC803A90400B2
:1047500022CC4EC6B707200006CE52C4AA892E84AA
:104760003379F90023A0F4180F10000097E0FB1F25
:10477000E7804016170AFC1F130A0A9A1DE1A2855A
:104780004E85213183470A006382370523A0241117
:104790001945F2406244D2444249B249224A056175
:1047A000828023110500A2854E85C53683470A0005
:1047B0006386370123A024110145E1BF17F7FB1FD2
:1047C000130727791E23C18F1EA3EDB797F7FB1F91
:1047D000938727789A23598C82A34DBF01114AC829
:1047E00037E900E022CC03240900B707200006CEF9
:1047F00026CA4EC67D8C2320F9180F10000093079F
:10480000F00263E7A704B144B304950297F9FB1FD4
:104810009389897583A70900A6979C4395CB9375C7
:10482000F5001181B315B028B3C50508193F83A75A
:1048300009000145A69723A0070023A20700232013
:104840008910F2406244D2444249B24905618280F3
:10485000B7E700E023A087100945E5B74111B7E7A6
:1048600000E026C2844306C622C437072000F98C24
:1048700023A0E7180F10000097E0FB1FE7808005DA
:1048800019E90145B2402244B7E700E023A09710A0
:10489000924441018280004597F7FB1F83A7C76BB5
:1048A00082979707FC1F9387A78E6367A402984798
:1048B000B74636FE938606C83305A4403697E372A2
:1048C000E5FC13070064B335E502D22781463305C2
:1048D000E502EF80B2567DB798473A94C9BF4111BF
:1048E00006C697F7FB1F23A7A7660295B240970756
:1048F000FC1F23AFA782014541018280411151462F
:1049000081451705FC1F1305658706C622C426C20C
:1049100097F7FB1F23A6076497F7FB1F23AC0762DB
:1049200097F7FB1F23AA076297F7FB1F23820762F3
:1049300097F7FB1F23AC076097C0FB1FE78000A819
:1049400013068002814517F5FB1F1305E57C97C010
:10495000FB1FE780A0A6EFF04FFF97F7FB1F9387A1
:10496000277EE82BFC3B17F4FB1F1304E47A8545F4
:104970003E958D473305F502994797F4FB1F9384C5
:10498000A45E39051375F50F28A03305F50213054C
:1049900005243345050897B0FB1FE780206C88C0CD
:1049A00035C93020994781453306F602130606249F
:1049B00097C0FB1FE78080A09C40382097F4FB1F26
:1049C0009384C459938707249CC0B347F72017F7F3
:1049D000FB1F2329F758093A25211C30944017E67C
:1049E000FB1F130606E733C7D72010C31387170032
:1049F0001377F70F17E6FB1F130646DF3347D72061
:104A000010C313873700890718B093F7F70FB3C7A0
:104A1000D72090C3B240224492444101828097F64D
:104A2000FB1F9386666F2A87BC228832637DF50060
:104A30001306150097F7FB1F83A7475290B2B347A1
:104A4000F52098C382801305F00F82801C41E5CBCE
:104A5000370700F07D8FB706002089476312D70E15
:104A60005A21411122C406C62A8469C719469305F2
:104A7000F00F690597C0FB1FE78060A705478D47CA
:104A8000630AE50A1C4491C75858994745C7185C02
:104A900055C31306C003814517F5FB1F1305456A6F
:104AA00097C0FB1FE78080911306C003A28517F50E
:104AB000FB1F1305E56897C0FB1FE780A08997F7E8
:104AC000FB1F9387E767DA2701E713070010DAA7D0
:104AD000F82719E30547F8A79A2B19E36D479AAB16
:104AE000F83719E31547F8B7B82B19E30547B8AB02
:104AF000B83B19E3F837B8BBD83B11C793763700FA
:104B00000983F4ABF8BBD82B19E35547D8AB182C65
:104B100001E71307C00398AF9C5791C7829797F797
:104B2000FB1F239FA75EFD5717F7FB1F2304F75EAC
:104B3000F1338147B24022443E854101828089475A
:104B40003E85828079714ECE97F9FB1F9389496427
:104B500083A7090006D622D426D24AD052CC829707
:104B600013090064B335250303D6C900814617FA3B
:104B7000FB1F130A6A5A32C633052503EF80122C35
:104B800083248A012A8401456386840232463305E0
:104B9000944063EF840003A589008146B335A902E0
:104BA0003305A902EF809229B3079540338587002A
:104BB000232C8A00B250225492540259F249624A7C
:104BC00045618280011122CC0A852E844146979549
:104BD00002009385A5E006CEEFF08FD318083324AA
:104BE000E420035704FFF240624497F7FB1F83D78A
:104BF000075B37450F00BA97130505243355F502B7
:104C00000561828097F7FB1F83D7675951471D4580
:104C1000637CF702794719456378F702130720038D
:104C200015456373F7021307B0041145637EF7005F
:104C3000130740060D456379F7001307600909451E
:104C40006374F70013B5B70F8280411122C426C2E6
:104C50002E84AA8406C6058CEFF0AFE9B327A40220
:104C6000B2402244338597001375F50F92444101F9
:104C70008280411122C426C22E84AA8406C6058CD5
:104C8000EFF02FE7B327A402B24022443385970008
:104C900033450508924441018280411122C426C255
:104CA0002E84AA8406C6058CEFF0AFE43335A40247
:104CB000B2402244269592444101828041114AC06B
:104CC00017F9FB1F1309C9478327890206C622C4A7
:104CD00026C28DCF829797F4FB1F9384E4439E24D2
:104CE0002A848DC733F7A70A33470708B3D7A70A23
:104CF000B3C70708B307F74051476359F700832745
:104D0000C90291C38297EF10623282A4B24022445A
:104D10009244024941018280011122CC97F7FB1F86
:104D200023A6072417F4FB1F130484415C5406CE0A
:104D3000AA8581C72AC68297B245D1C59C4105453F
:104D4000BDCF9C45ADCFDE25BDCBFE25ADCB9C298F
:104D500081CB7C287838BA976343F506DC41A5C33C
:104D60001306400217F5FB1F1305854297B0FB1F82
:104D7000E780405E97F7FB1F93878741984397F63C
:104D8000FB1F23ABE61C183C19EFCA27930780577B
:104D900037460F003305F502130606248146814588
:104DA000EF80D20908BC183C9D4763E4E700A147A7
:104DB0001CBC17050000130525D915360145F24026
:104DC00062440561828097F7FB1F23A5073697F79A
:104DD000FB1F9387E73B17C7FB1F130747C298C307
:104DE00037873200FD56130727A194C7D8C797F716
:104DF000FB1F2387073AB7C7004023A4D7269DBFD0
:104E0000011122CC17F4FB1F13048433084406CE8F
:104E100026CA4AC801E90545F2406244D2444249E3
:104E2000056182805C58E5DB185C75D770008545AC
:104E300082971844B247E300F7FE4A249305E00442
:104E400017F9FB1F1309492D97B0FB1FE7800021BD
:104E50002320A90269D152249305F00F814497B011
:104E6000FB1FE780A0557C240326090263C1F402DE
:104E7000328597B0FB1FE780802B014597F7FB1F1A
:104E800023AC072A97F7FB1F23AA072A71B74E24E2
:104E90001844B3879502898185043385E7001C5C3B
:104EA00008C28297C9B7011122CC17F4FB1F130463
:104EB00024291C4426CA4EC656C206CE4AC852C42D
:104EC0005AC0AA84AE89B28A6388071A585839CB67
:104ED0001307F01F6366A71017FAFB1F130ACA23F4
:104EE00003290A02631209044A249565938515E093
:104EF00097B0FB1FE78080162320AA022A861DC1D7
:104F00004E245C580844898182971C4403290A0274
:104F10002322FA028947639EF402C1479305090CD4
:104F20006381F9042945BDA003274A02E384E7FE13
:104F30004A249565938525E097B0FB1FE780001212
:104F40002A896DD14E242A865C580844898182972B
:104F5000D1B78D47639AF404C1479305490DE39394
:104F6000F9FCB8219307A0056312F7069E21639F01
:104F700097044E869105568597B0FB1FE780803DCC
:104F800083270A02638727014A8597B0FB1FE780C2
:104F9000001A0145F2406244D2444249B249224AD1
:104FA000924A024B0561828091476397F400930512
:104FB000890EE39999F675B793070010E394F4F618
:104FC000A147E3E137F79305090F61BF83270A0281
:104FD000E38A27F54A8597B0FB1FE780401599B70C
:104FE0001D67637FE506130705E099463347D7023F
:104FF000562417FBFB1F130B2B123307D702330A60
:10500000F70083274B026396470103290B026311C4
:1050100009024A249305E00497B0FB1FE7800004CF
:105020002A8909D14E245C582A8689815285829723
:1050300091451307A00593F5C50FB307B900B42335
:105040006399E60296236394960291054E86CA956B
:10505000568597B0FB1FE780E02F83270B021DB713
:10506000A166F916E3E0A6EC3307E54051B7AC338F
:10507000D9B783270B02A9BF97F5FB1F83A5C50BE3
:10508000E38205EA91479306A00593F7C70F33879C
:10509000F5003023E318D6E81223631B960091072E
:1050A0004E86BE95568597B0FB1FE780A02AD5B5E2
:1050B0003C33E1BF97F7FB1F93878708984721C7C9
:1050C000985F31C385466310D504411122C417F49B
:1050D000FB1F13046404105006C615C2CE274850A7
:1050E00089810297085097B0FB1FE780400497F72B
:1050F000FB1F23A3070497F7FB1F23A10704B2405C
:10510000224441018280828001114AC817F9FB1FA5
:10511000130909034EC68329890022CC26CA52C42A
:1051200006CE56C2AA842E84328A638D091A83273A
:10513000890399EB2945F2406244D2444249B2497D
:10514000224A924A0561828083274903E5D7930763
:10515000F01F63E0A70C97F9FB1F9389E9FB83A776
:10516000090295CF0325890083A749026395A70407
:105170008947639FF404C147E31EF4FA03A50902BB
:105180001305050C9307A0053CA106A12286D28534
:10519000110597B0FB1FE780E01B014569BF035570
:1051A000C9009305E00497B0FB1FE78020EB23A024
:1051B000A9024DF941B78355C9008327490303A6C6
:1051C0000902898182978327890023A2F9024DB7BA
:1051D0008D47639AF400C147E31EF4F403A5090266
:1051E0001305450D45B791476399F400E31494F412
:1051F00003A509021305850E71B793070010E39B01
:10520000F4F2A147E3E887F203A509021305050FAD
:1052100095BF9D676373F506930705E01947B3C70C
:10522000E7020357C90097FAFB1F938AEAEEB38798
:10523000E702BE9983A70A02A1CB83A74A02639122
:10524000370703A50A0291479305A0051308F00F3D
:1052500013F7C70FB306E500B0226313B60683D871
:105260000600B032639C9804B307F64063C6870417
:1052700011072286D2853A9529BF21677917E36BFA
:10528000A7EAB307F54071BF0355C9009305E004D1
:1052900097B0FB1FE78080DC23A0AA0259FD59BD0F
:1052A0008355C9008327490303A60A0289814E85D5
:1052B000829723A23A0371B723900601B28749BFB0
:1052C0003386870011061308F00B6374C8002D4560
:1052D0009DB5ACA213063400719A1106B29786A24E
:1052E000BCB279B797F9FB1F938909E383A7090239
:1052F0009DCB03A5090291471308A0059305F00F64
:1053000013F7C70FB306E500B0226310060583D874
:105310000600B03263979800B307F640E3DA87F4EB
:105320008EA2B287F1BF8347E9000355C9009305F8
:10533000E0043305F5023345050897B0FB1FE7800D
:10534000E0D123A0A90255F5F5B30356C900834562
:10535000E900B385C502338687001106E3E9C5F687
:105360002381060185BF014582809C211CA1BE21AD
:105370001CB1BE21A1833CA1DC213CB1114582803E
:1053800097F7FB1F23A807BE97F7FB1F23A207BEB3
:1053900082800DCD411122C426C206C6AA842E8465
:1053A000014585C1228541469785020093850566A2
:1053B00097B0FB1FE78000FA9C2005455CA49C3059
:1053C0005CB4B24022449244410182800145828013
:1053D000011122CC26CA06CE8947AA843284639E54
:1053E000F5006383B602414781476395E6048A85E9
:1053F0004D3741468A8522850DA841476392E504D1
:10540000638FF600639EB6022E86A2856244F24048
:105410002685D244056117B3FB1F670023058A85E3
:105420003285853F41468A85268597B0FB1FE780F8
:10543000E003AA87F2406244D2443E85056182803F
:105440008147CDBF97F7FB1F23A4A7B2828097F7B0
:10545000FB1F23A1A7B28280011122CC622106CEBC
:1054600026CA4AC84EC63DC8832985002A88AE840C
:1054700003C9090081471317496063550702B14703
:10548000054563F687040355280051143344040886
:105490004E8633878900A2868545EFB0D003B337A7
:1054A000A0008507135569487D141379F903334427
:1054B00004089CA088B023812401C2A0014719C020
:1054C0001387190098C409476383E7000145F24038
:1054D0006244D2444249B249056182800545C5BF54
:1054E000C167F917630AF502D94763F7B7020111DB
:1054F00022CC2EC606CE2A84EF90C007B245636840
:10550000B50022856244F24005616FA0A07CF240A4
:10551000624405450561828005458280C167F917AF
:105520006314F5006F900005411106C6EFA02069D5
:1055300011E15D45B240410182809147639DF500D4
:105540001C211CA23C211831A207D98F3EA23C315C
:1055500001455CA28280114582804111814522C4AF
:1055600026C206C6AA849D232A8409E997F7FB1F51
:1055700083A707A081C7F94526858297B240228577
:10558000224492444101828039714ED652D45AD07D
:105590005ECE06DE22DC26DA4AD856D22A8A2E8B46
:1055A000B289B68B0DE79D3F9145EF90C00A2A84E2
:1055B0004D49854A19EDF2506254D254B259225ADB
:1055C000925A025BF24B4A854259216182803A84A9
:1055D000814A230034018544630A0B00DE851305EC
:1055E0001400029B93041500B3C404089399496006
:1055F00063D30902C1455285EFA0A06A654915E54C
:1056000033069400A6852285EFB000322A8911ED79
:10561000B104B3C4040891472C0052857C8422C68F
:105620006485EF90D07F2A8959D5E3860AF82285D0
:1056300097B0FB1FE780A0AFBDBF011122CC26CAE7
:105640004AC84EC606CE2A893284B689353FAA8416
:105650000DE197F7FB1F83A7E79181CF05476317FC
:10566000E40003C4090005041374F40FA2854A85FD
:105670008297F24062444249B2492685D24405618C
:105680008280AE860147054697050000938525CEAA
:105690006DB79E211CA19E21A1831CB1094582806A
:1056A0009E211CA19E21A1831CB1BE213CA1BE2133
:1056B000A1833CB1114582809E211CA19E21A18322
:1056C0001CB1BE213CA1BE21A1833CB1DC315CA157
:1056D000FC215CB18A2519053345050882809E218D
:1056E0001CA19E21A1831CB1094582809E211CA181
:1056F0009E21A1831CB1BE213CA1BE21A1833CB14E
:1057000011458280CA2106053345050882809E2105
:105710001CA19E21A1831CB1AA21090533450508BE
:1057200082809E211CA19E21A1831CB1BE213CA18F
:10573000BE21A1833CB1CA211105334505088280F1
:105740009C211CA1054582809E21411122C406C6D0
:105750001CA19E212E841105A183A30EF5FEBE215E
:105760009505230FF5FE83D7D5FFA183A30FF5FE83
:1057700003C6F5FF97B0FB1FE780C0BD4820B240CD
:10578000224411054101828089476399F5001C314B
:1057900018210145A207D98F1EA28280114582805F
:1057A0009A21011106CE22CC2EC6D94763F4E70216
:1057B0002A84EF80305CB2469E22636DF50022851C
:1057C0006244F24001470946970500009385A5EC25
:1057D00005615DBBF2406244094505618280AA878C
:1057E000A9C11421FD150547B3C505086398E60056
:1057F00013D725008D89114589CD82800947114530
:105800006392E602494533D7A502B3F5A5021145D7
:1058100091E9114501CB850734A21AA25CC201456A
:10582000828011458280AE860147114697050000AF
:10583000938545E791BB13F73500AA8701EB898172
:10584000114591C50EA25CC201458280114582803E
:10585000D8218947631BF702011122CC2A84C8454D
:1058600006CEAE8601C92EC69D4597B0FB1FE780C8
:105870008099B2462A8722856244F24019469705EC
:1058800000009385A5E3056101B30945828099E194
:10589000114582801C2105473EA2E37BF7FEFD15E2
:1058A00093F5F50F33D7F502B387E702E392F5FEE0
:1058B000050548C21AA201458280DC210947AE864F
:1058C0006385E70041476399E70001472146970553
:1058D00000009385A5E74DB9094582800EA291E1AC
:1058E000014548C201458280AE8601472946970599
:1058F0000000938505DF49B90EA291E1014548C238
:1059000001458280AE8601473146970500009385A8
:1059100025DE9DB90EA291E1014548C20145828074
:10592000DA21854763FFE702011122CC2A848841EE
:1059300006CE2EC615C1854597B0FB1FE780A08C0B
:105940002A8722856244B246F24039469705000014
:10595000938585DB05610DB9F24062440945056117
:10596000828009458280AA878DC518218D46114500
:1059700063F2E602FD15B3C50508B3C6E5023308B8
:10598000D70263990501850716A23AA25CC20145B8
:10599000828011458280DC210947AE866385E7005D
:1059A00041476399E7000147414697050000938509
:1059B000E5D9D9BE094582803335B0000A05828019
:1059C000011122CC26CA06CE98258547AA842E84AA
:1059D0004946631FF70099363E20491513062009F2
:1059E00063C8A700F2406244D24409450561828041
:1059F000183485476314F70013660604484001C94C
:105A00008D4532C697A0FB1FE780E07F3246A28615
:105A10006244F2402A872685D24497050000938588
:105A200045CF056195B68D4763F7B7021C31182144
:105A3000F115A207D98F1EA23C313821B3C5050844
:105A4000A207D98F014799C1130745003EA24EA274
:105A500018C60145828011458280011122CC2A841A
:105A6000884506CEAE8601C92EC6954597A0FB1F78
:105A7000E7806079B2462A8722856244F24059461F
:105A800097050000938525CA0561FDBC3335B0003C
:105A90000A058280AE86014761469705000093851E
:105AA00065CADDB48547114563F1D7021C320C226B
:105AB0000945A207CD8F81456384A6009305260082
:105AC000F9161EA336A34CC30145828001478146C7
:105AD0007946814555BC9E211CA19E21A1831CB104
:105AE00009458280BC2105471CA18A216397E700F4
:105AF0000A050505334505088280C9473305F502C7
:105B0000CDBF8A210A05334505088280BE211CA12C
:105B10008A21BE213305F50205053345050882803B
:105B20008A2182808A2182808A218280BE211CA1D2
:105B30008A21BE213305F50205053345050882801B
:105B40009E211CA19E21A1831CB1BE213CA1BE218E
:105B5000A1833CB1CA2111053345050882809E21ED
:105B60001CA19E21A1831CB1AA210905334505086A
:105B70008280894711456398F6001C321422014542
:105B8000A207D58F1EA382809A21D947AE8663F9DA
:105B9000E70001470D4697050000938505F471BCA9
:105BA000094582801145639DA6001C3214220145DF
:105BB000A207D58F1EA33C323422A207D58F3EA365
:105BC0008280BC210547FD1793F7F70F6361F70447
:105BD0009E2195CF011122CC2A84C84106CE2EC623
:105BE00015C1894597A0FB1FE780E0612A872285C0
:105BF0006244B246F2401546970500009385C5EE13
:105C0000056125BCF2406244094505618280094571
:105C10008280954763F0D706411122C426C24AC04C
:105C200006C61C323A841822A207B284D98F1EA05D
:105C30003C32382293854400A207D98F3EA0894781
:105C40005CA0094613055400368997A0FB1FE78026
:105C50006070194781476304E900938764006919FC
:105C600023142401B2405CC42244924402490145F9
:105C700041018280114582809E2195CF011122CC65
:105C80002A84C84106CE2EC615C1854597A0FB1FA4
:105C9000E78060572A8722856244B246F2401D465B
:105CA00097050000938525E6056141BAF2406244FC
:105CB000094505618280094582809947B2856388DC
:105CC000F600D147114541466384F60082800946BB
:105CD000411106C650A39C31942113055700A20719
:105CE000D58F1EA3BC31B4219105A207D58F3EA349
:105CF00097A0FB1FE7800066B2400145410182800A
:105D00009E219DCF011122CC2A84C84106CE2EC6E9
:105D10001DC1894597A0FB1FE780E04E2A87228599
:105D20006244B246F240254697050000938545DE61
:105D300005616FF09F90F2406244094505618280E1
:105D400009458280894711456398F6001C32142268
:105D50000145A207D58F1EA38280011122CC2A847F
:105D6000C84106CEAE8601C92EC6854597A0FB1F49
:105D7000E7806049B2462A8722856244F2402D4678
:105D800097050000938505DA05616FF01F8B19BD3B
:105D9000011122CC2A84C84106CEAE8601C92EC686
:105DA000854597A0FB1FE7800046B2462A872285DB
:105DB0006244F2403546970500009385E5D60561BB
:105DC0006FF0BF8793F71600114581EB8947638613
:105DD000F600858256A310C301458280011122CCB2
:105DE0002A84C84106CE2EC61DC1854597A0FB1F3B
:105DF000E78060412A8722856244B246F2403D46F0
:105E000097050000938585D205616FF01F83F240EE
:105E100062440945056182809E219DCF011122CCFB
:105E20002A84C84106CE2EC61DC1894597A0FB1FF6
:105E3000E780603D2A8722856244B246F2404546AB
:105E4000970500009385C5CE05616FF00FFFF24006
:105E5000624409450561828009458280854763F473
:105E6000D70208A70CB71C320C220945A207CD8F18
:105E700081456384A60093052600F9161EA336A368
:105E80004CC30145828011458280014781464D46C1
:105E900081456FF08FFA8D47114563F5D7021C32AB
:105EA0000C22A207CD8F1EA33C322C22A207CD8F3D
:105EB00081456384A60093054600F1163EA356A3D0
:105EC0000CC701458280011122CC2A84884506CE68
:105ED000AE8601C92EC6954597A0FB1FE780A0326C
:105EE000B2462A8722856244F2405D46970500004B
:105EF000938545C505616FF04FF48547114563955E
:105F0000F6001C2201451CA382800147814665469C
:105F100081456FF08FF2011122CC2A84C84106CE50
:105F2000AE8601C92EC68D4597A0FB1FE780A02D28
:105F3000B2462A8722856244F2406D4697050000EA
:105F4000938525C205616FF02FE4011122CC2A84CC
:105F5000C84106CEAE8601C92EC68D4597A0FB1F4F
:105F6000E780602AB2462A8722856244F24075465D
:105F7000970500009385E5BE05616FF0EFE0011124
:105F800006CE2EC6EF90D03F19C5B245F2402A2169
:105F900005616FE0E005F24049450561828097E7C1
:105FA000FB1FA38F07FE97E7FB1F238B07FE97E7D7
:105FB000FB1F23A507FE97E7FB1F23AF07FC97E70F
:105FC000FB1F23A907FC97E7FB1F23A307FC97E709
:105FD000FB1F23A507FA97E7FB1F23AF07F897E7F7
:105FE000FB1F9387271D3706840390D33707B40020
:105FF00037C6070098C3130606B83747A000D8C3B2
:10600000D0D33707100041669306070AB705500042
:106010009308060194C723A41703938605019308E8
:1060200016F8D4C723A61703B706D007B7087F0012
:106030001308070513850601410723A81703B0C3FA
:10604000930816009386060513861500D8CBF8C36F
:1060500023A8070188CF23AE070023AA170323AC88
:10606000070223AE070223A40704F0C7B4CB23AA78
:106070000704ACCF23AE0705B8D33707A000F8D785
:106080001307000AB8DB1307C01CF8DB370714003E
:10609000B8DF0547F8DFE8D323A40706930710F815
:1060A00017E7FB1F2328F7188280011152C42A8AA0
:1060B000214522CC26CA4AC84EC606CE2E84B289B5
:1060C0003689BA8497A0FB1FE780001905C993079A
:1060D00000FD1CA19947A30045013CA12303250114
:1060E00064B123123501AA8522856244F240D2446C
:1060F0004249B249224A05616FE02F95F24062445D
:10610000D2444249B249224A0561828097E7FB1F87
:1061100023A6A7E8828097E7FB1F23AFA7E682802C
:1061200097E7FB1F23A8A7E6828097E7FB1F23A121
:10613000A7E68280011122CC26CA4AC806CE4EC6E6
:106140002A89AE840144B309890063699400F2404E
:106150006244D2444249B24905618280EFE06F99BE
:10616000B3470508A1832380F9009307140093F730
:10617000F70F850963F89700CA97090488A3137479
:10618000F40FD1B73E84D1B7411122C417E4FB1FED
:106190001304840A6A20C16706C6FD17630EF50062
:1061A00017E6FB1F0346462B97E5FB1F938545DD4E
:1061B000EF90007EFD577EA0B240224441018280D4
:1061C00009C925151375F50F1335850E13451500EF
:1061D00082800145828023900500C9C2797122D452
:1061E00026D252CC56CA5AC806D64AD04ECE5EC621
:1061F0002A8B2E8AB28A3684814463FF5405B30702
:10620000940083C907001389140033490908638582
:106210000904B387290163C1FA04B307240183CBBE
:1062200007005E85713F0DC99387F9FF2310FA00BF
:1062300063906B03050933052401B2502254925434
:106240000259F249624AD24A424BB24B45618280BE
:10625000CE94B3C4040855B70145C5B70145828043
:10626000011122CC26CA4AC84EC606CE97E4FB1FAF
:10627000938484FC2E89D0C88CC8C8C42A84414623
:106280009305F00F4A8597A0FB1FE78040268549BC
:10629000631935038848C145713D41469305F00FA8
:1062A000228597A0FB1FE7808024054963152503FD
:1062B0006244C844F240D2444249B249C1450561F2
:1062C00095BD414681454A8597A0FB1FE780202266
:1062D000E31535FDC1B741468145228597A0FB1FD7
:1062E000E780E020E30625FDF2406244D2444249C3
:1062F000B24905618280411122C426C22E84AA843B
:1063000013060002814517E5FB1F1305E5F206C6DB
:106310004AC097A0FB1FE780600A17E9FB1F13091B
:10632000A9F197E7FB1F238B8712A3019900EFD0F8
:10633000704E854719C1814749452300F900B24095
:10634000224492440249410182809DC91DC985476A
:106350006318F500DC3193E707FCDCB1054582806A
:1063600089476316F500DC3193F7F703FDB78D47D6
:10637000E316F5FEDC3193F7F70393E70704F1BF6B
:10638000014582808DC10DC1DC311307000C05452C
:1063900093F7070C638AE700130700040945639528
:1063A000E7000D45828001458280411122C4005DD5
:1063B00006C626C21DC8AA84085009C597A0FB1F9F
:1063C000E780E0D6485009C597A0FB1FE78020D69C
:1063D000085409C597A0FB1FE78060D5228597A0C8
:1063E000FB1FE780C0D423AC0402B2402244924495
:1063F0004101828019ED97E7FB1F83C707E417E58A
:10640000FB1F1305E5E491CB17E5FB1F1305C5B78B
:10641000828017E5FB1F1305A5E3828017E5FB1FAC
:106420000345A5E1828017E5FB1F0325A5E18280D6
:1064300017E5FB1F032545E1828097E7FB1F83A734
:10644000E7E08843828017E7FB1F1307E7DE544B22
:106450009C4285079CC228339307F00F6307F50021
:10646000916517C3FB1F670083598280011122CCFD
:1064700006CE2E8432C6EF9030019147B245631E9E
:10648000F50097E7FB1F83A7A7B099CF9C4389CF5F
:1064900022856244F2400561828797E7FB1F83A74C
:1064A000A7AF99C3DC43E5B7F240624405450561F7
:1064B0008280797122D42A844A214ECE06D626D2F1
:1064C0004AD097C0FB1FE780406A97E9FB1F93897A
:1064D00029AD29E983C409009307F00F639DF400F7
:1064E00097E5FB1F83C5D5AB2685513C09E597E7AA
:1064F000FB1F238707AA4A20EF9000799147631C6E
:10650000F50097E7FB1F938727D35620FA23639460
:10651000E6007D57FAA3B250225492540259F24930
:1065200045618280582504212A893AC6BD3D4A85A5
:10653000EF9050344A20EF90607083C709003247D3
:1065400099C3E38F97F89307F00F5220E385F4FA8D
:1065500074202820A685913E79BF79715AC82A8B6C
:106560002E854ECE52CC56CA06D622D426D24AD03A
:106570005EC62E8AB28AB68997C0FB1FE780E05EAE
:1065800075C5045D2A89FDC09C501305400391E345
:1065900061459C5489C79307450133C50708638645
:1065A00009009307C50133C50708DC5089C7930765
:1065B000750133C5070897A0FB1FE780E0C92A844F
:1065C00055C56146814597A0FB1FE78020DF97EB0B
:1065D000FB1F83CB2BC163940B00834B09009307F4
:1065E00000FD1CA0A947A30064013CA023035401A3
:1065F0008C50231244011305840191C908C47146CB
:10660000130A440397A0FB1FE780C0D452858C5423
:1066100091C948C45146130A450197A0FB1FE78062
:1066200060D35285638C090008C87146CE85130A71
:10663000C50197A0FB1FE780E0D15285CC5099C5DA
:1066400048C85D4697A0FB1FE780C0D0A2855E8545
:10665000EFD0BFBF2254B2509254F249624AD24A9C
:10666000424BB24B4A850259456181B3B250225424
:1066700092540259F249624AD24A424BB24B4561A6
:10668000828001114EC6AA892E8526CA06CE22CC4A
:106690004AC8AE8497C0FB1FE780204D21C917E987
:1066A000FB1F034929B46314090003490500194578
:1066B00097A0FB1FE78040BA2A840DC9814519467F
:1066C00097A0FB1FE78080CF930700FD1CA0B94770
:1066D000A30034013CA046A0A2856244F240D2440B
:1066E000B2494A85424905616FD03FB6F2406244E3
:1066F000D2444249B24905618280797162C42A8CD0
:106700002E8526D24ECE52CC56CA5AC85EC606D662
:1067100022D44AD0AE84B28B368BBA8A3E8AC289E2
:1067200097C0FB1FE780604435C52A89414597A083
:10673000FB1FE78060B22A8431CD4146814597A096
:10674000FB1FE780A0C717E5FB1F0345A5A919E1BB
:1067500003450900930700FD1CA0BD47A300840169
:106760003CA023047401A304640123055401A30580
:10677000440146A023263401A2852254B2509254EB
:106780000259F249624AD24A424BB24B224C45610D
:106790006FD0BFABB250225492540259F249624AB0
:1067A000D24A424BB24B224C45618280011126CA2B
:1067B000AA8439454AC84EC652C406CE22CC2E8A77
:1067C000B289368997A0FB1FE78000A915CD9307F2
:1067D000000D1EA1B1472A84231245013CA1CE859C
:1067E0001905194697A0FB1FE780C0B623062401B0
:1067F000A2856244F2404249B249224A13F5F40F9D
:10680000D24405616FD07FA4F2406244D244424931
:10681000B249224A05618280411126C206C622C4BD
:106820004AC097E4FB1F938424A1B8309307F00F6C
:106830006308F7042A89394597A0FB1FE780C0A1A8
:106840002A841DCD930700FD1CA1A300250123016F
:10685000050097E5FB1F9385A59F0D05194697A099
:10686000FB1FE78020AF9E24A285A8303EA49C3069
:106870005CA42244B2409244024941016FD0FF9C83
:10688000B24022449244024941018280011156C221
:10689000AA8A314526CA4AC84EC652C406CE22CC60
:1068A0005AC0AE84328AB6893A8997A0FB1FE78026
:1068B000A09A2DCD2A84268597C0FB1FE780E02A69
:1068C00009C55825A1476311F70417EBFB1F034BBC
:1068D000DB96930700FD1CA09D47A30054013CA03C
:1068E00046A0231344012314340123152401A28557
:1068F0006244F240D2444249B249224A924A5A85FD
:10690000024B05616FD07F9417EBFB1F034B1BB548
:10691000E3910AFC97D7FB1F83A7C77C9C47D5DB75
:10692000CA864E86D2852685829765B7F240624434
:10693000D2444249B249224A924A024B05618280BE
:10694000411126C2AA84214522C406C62E8497A0DE
:10695000FB1FE780609015C5930700FD1CA1C5478C
:106960003CA13C30AA853CB15E205EA17C207CA18C
:106970007C307CB12244B2402685924441016FD0E4
:10698000DF8CB240224492444101828041114AC0CE
:106990002A89714526C206C622C4AE8497A0FB1F71
:1069A000E780808B3DC5930700FD1CA1F5473CA106
:1069B000BC302A849385C4003CB1DE2031051946E1
:1069C000231CF5FEFE20231DF5FE9E24231EF5FE4E
:1069D000BC24230FF5FEBC34A30FF5FE97A0FB1FCC
:1069E000E7804097BC28A2854A853CA8DE285EA89F
:1069F000FC287CA8FC387CB89C2C1CAC9C3C1CBCA7
:106A0000BC2C3CAC2244B2409244024941016FD0BC
:106A1000DF83B24022449244024941018280011145
:106A20004AC82A89614526CA4EC606CE22CCAE89FE
:106A3000B28497A0FB1FE780208225C1930700FD49
:106A40001CA1BC302A84938584001CB195473CA1CD
:106A5000FC3011051946A30FF5FE97A0FB1FE78038
:106A6000608FDE2023063401A2853EA4BE2C4A8519
:106A70007EA4DE2C1EA8FE2C3EA883C704025CA8C0
:106A800083C714025CB8BE30F240D2447EA8624490
:106A90004249B24905616FD04FFBF2406244D24493
:106AA0004249B24905618280411122C406C617D409
:106AB000FB1F130464783C209DCBAA85194617D58B
:106AC000FB1F1305654C97A0FB1FE780A0882820BB
:106AD00097D5FB1F9385454BEFF03F872244B2408B
:106AE00017D5FB1F1305454A41016FD06053B240D3
:106AF0002244014541018280411126C206C622C4BA
:106B00004AC097D4FB1F93842473B8309307F00FC7
:106B10006302F7042A8929459790FB1FE780C07319
:106B20002A840DC9930700FD1CA1A147A3002501DC
:106B30003CA1BC2097D5FB1F938505451105A30FEC
:106B4000F5FE194697A0FB1FE780C080A830A285FC
:106B5000EFD0AFEFB8208D47631FF70097D7FB1F2B
:106B600083A7474389CB9C4799C72244B2409244AC
:106B7000024941018287B2402244924402494101C4
:106B80008280797122D406D626D24AD04ECE52CCFB
:106B900056CA09444DCD2A890A212E8A514497C0EC
:106BA000FB1FE78080FCAA845DC197EAFB1F938AE4
:106BB000AA8A83C74A0005474944FD1793F7F70F90
:106BC0006377F7085825A1476314F70063110A0893
:106BD0009C5C4544ADEF9165938545711305C002FA
:106BE0009790FB1FE780804788DCAA894D4425C128
:106BF0001306C00281459790FB1FE780207C8357D6
:106C000009009386490036852391F9007146930562
:106C1000490036C69790FB1FE780C07389472380E1
:106C2000F900DC24B2460356090083C50A00E117C7
:106C300013B51700EF90B07D2A8463060A00D28551
:106C40002685EF90807201C42685EFF00FF6B250D2
:106C50002285225492540259F249624AD24A45612D
:106C6000828097D7FB1F83C7677FFD1793F7F70FC6
:106C700005476377F70801114AC806CE22CC26CA19
:106C80004EC652C4328989472DC22A8AAE893684BB
:106C900097C0FB1FE78060EDAA84D14739C54855EE
:106CA00009C59790FB1FE7808048F1454A8597907A
:106CB000FB1FE780C076C8D4AA85CD471DC5D82460
:106CC000A147631DF70209C8382D12299306250133
:106CD0005285EF90E06F2A84D82093674700638441
:106CE000090093676700DCA0A287F2406244D244A7
:106CF0004249B249224A3E85056182800144E9BF8A
:106D0000C9473E8582809307000463EAA70097D7AE
:106D1000FB1F9387274A3325F5200A21828041658E
:106D20007D158280011122CC2A842E8526CA06CEAA
:106D3000AE8497C0FB1FE78040E30DCDB7470F003F
:106D40009387F723094563E2870281450A85414617
:106D50009790FB1FE7808066A68560800A8541804A
:106D60004081A3010100EF90504AF2406244D244B6
:106D7000056182804945D5BF97D7FB1F238FA76C3C
:106D800082806F903063797152CC2A8A328526D204
:106D90004AD04ECE56CA5AC85EC662C406D622D45F
:106DA0002E8CB28A368BBA8B3E89C289C68497C034
:106DB000FB1FE78080DB05C92A84631A0A189377D2
:106DC0004B000343450085CF1363230163940B16E7
:106DD00063100914639F090885E81C5C1373B3FFF3
:106DE00023026400C5EBB250225492540259F24976
:106DF000624AD24A424BB24B224C456182801373A5
:106E0000D3FF13630301D9B7136343002302640064
:106E10009C484146A6851CD4130584019790FB1F0E
:106E2000E780405363130C12638C0B0A485409C566
:106E30009790FB1FE780A02FF1455E859790FB1F81
:106E4000E780E05D48D4005C59DC1C5091EB916513
:106E50009385357171459790FB1FE780202008D0FE
:106E600008500DC17146DE859790FB1FE780804E6C
:106E700011A81363430023026400D9F8005C630C7B
:106E80000C0235D0639A0902A5E029A0005C21DC40
:106E9000639409022254B2509254F249B24B224CEC
:106EA000CA865A860259424BD6855285D24A624AD0
:106EB00045616FF08FEA05D85C5091EB9165938541
:106EC00025715D459790FB1FE780401948D04850D9
:106ED00045DD5D46CE859790FB1FE780A0476DB7E7
:106EE000005C11D0E39A09FC1C5491EB91659385E9
:106EF000157151459790FB1FE780401608D4085440
:106F000051D95146A6859790FB1FE780A04459B7F9
:106F10001363430023026400E39C04EEE3080CF6D1
:106F2000485405EDF1454A859790FB1FE780204FB7
:106F300048D431A81363430023026400E39A04ECAD
:106F4000E3060CEEE31E09FCFDBDE31B09FC005C3F
:106F5000E30B04E8E39B0BEE35B79790FB1FE7804C
:106F6000001DC9B7011126CA52C406CE22CC4AC898
:106F70004EC62A8AAE8497C0FB1FE78000BF35C18A
:106F80002A8939459790FB1FE780002D2A8431C953
:106F900097D9FB1F83C90925639409008349090018
:106FA0009307000D1EA0AD473CA093056900130593
:106FB000340019469790FB1FE780C03993F71400FF
:106FC0005CA493D4144844B423154401A2856244BC
:106FD000F240D2444249224A4E85B24905616FD0FF
:106FE000CFA6F2406244D2444249B249224A0561E6
:106FF000828001114EC652C456C206CE22CC26CA89
:107000004AC8AA8A2E8AB28997C0FB1FE780E0B5DA
:1070100035CDAA841305C0029790FB1FE780C023DB
:107020002A842DC517D9FB1F0349C91B6314090006
:1070300003C904009307000D1EA0E9473CA09385F7
:1070400064001305340019469790FB1FE7808030D9
:10705000D285231554011305C40041469790FB1FA8
:10706000E780402FCE851305C40141469790FB1F52
:10707000E780402EA2856244F240D244B249224ABF
:10708000924A4A85424905616FD02F9CF240624482
:10709000D2444249B249224A924A0561828017D5B8
:1070A000FB1F032565ED11CD411106C69790FB1F0F
:1070B000E780E007B24097D7FB1F23AF07EA410103
:1070C00082808280411122C406C626C24AC02E8414
:1070D00097C0FB1FE78060A929CD00D517D9FB1FFA
:1070E00003494910AA846314090003490500414576
:1070F0009790FB1FE78040162A8405CD9307000D6B
:107100001EA1A5473CA1DC30938564001105A30FA7
:10711000F5FE19469790FB1FE780C0239C54A2857B
:10712000B2405CC4224492444A85024941016FD076
:10713000CF91B240224492440249410182805D7164
:10714000A2C4A6C286C6AA842E8497C0FB1FE7806D
:10715000C0A10DC954251147AA874945639FE60080
:107160009C5F91C3E02B97B600009386269A0A860F
:10717000894526854080EF904016B64026449644C7
:10718000616182805145D5BF97D7FB1F83C7072D0B
:10719000FD1793F7F70F0547637AF704411126C2ED
:1071A00006C622C44AC0B284894715CA2E8997C030
:1071B000FB1FE780809B2A84D14715C16306090025
:1071C0005C2193E727005CA14146A6851305840155
:1071D0009790FB1FE78000189C481CD48147B24061
:1071E0002244924402493E8541018280C9473E853E
:1071F0008280011122CC26CA06CE2A84AE8497C092
:10720000FB1FE780809619C96C0022854486EF90A9
:107210006012F2406244D244056182805145D5BF7C
:107220006F80901BC1671387E7FF6393E50297D7D1
:10723000FB1F83A767D691EB494582804945B24041
:10724000224492440249410182809C43F5D78287BF
:10725000411122C426C24AC006C6FD172A892E84BF
:10726000B284639AF50297D7FB1F83A7E7D289C739
:107270009C4399C3829711C5A6854A85EFE03FD00C
:107280005DFD97D7FB1F238D27D197D7FB1FA389C0
:1072900097D001456DB72E8597C0FB1FE780E08C26
:1072A00051DD1C210D45E39C27F922852244B24083
:1072B0000249A685924441016FC090539307000490
:1072C00063E1A7064111C16722C426C206C6FD17A5
:1072D0002A84AE8409456380F502C5476312F4022F
:1072E0002E85EFC0905897D7FB1F9387A7EC3324C8
:1072F000F420014506A0B24022449244410182801C
:107300009307A0036316F4002E85EFC0304FE1BF52
:107310009307B003E319F4FC13F5F50FEFC0504EDB
:10732000D9B709458280011106CE2AC6EFE03FC7D2
:10733000EF20404EEF10C07CEF50F229324597D736
:10734000FB1F938767EF130700F0BAA323820700A0
:107350007D5797D7FB1F93872710B8A388A3F240C8
:10736000954505616F70402A757126C306C722C511
:107370004AC1CEDED2DCD6DADAD8DED6E2D4E6D224
:10738000EAD0EECEAE849397556063D1075817DAF2
:10739000FB1F130A6A0C03450A00130B200A930B08
:1073A000F00F9790FB1FE78020F1C167FD172A843B
:1073B000130C1009954C394D97DDFB1F938DCDE7CC
:1073C0003ECC15E01395F468BA402A449A440A4921
:1073D000F659665AD65A465BB65B265C965C065DE5
:1073E000F64D496182801C20639A670103C93D0004
:1073F000E2452A202286EFF06F87E1A003492A00A8
:10740000639A87091C30639097032285EFF06F8A97
:107410002285EFC07FDE03450A009790FB1FE780BF
:10742000A0E92A8479BF639BA7194A208567A5072D
:10743000631AF5040C4497D9FB1F9389E9DF88216F
:1074400015E51946850517D5FB1F130565E09790CF
:10745000FB1FE78020F003C709008547631CF70284
:1074600089472380F900EFC0703B5DB703C709006F
:1074700085476311F70297D7FB1F238F07DAEFF0D9
:10748000AFB979B709679307C70063EFA70405078A
:10749000636BA702E30E79F7A2854A85EFC0FFDA96
:1074A0009DBF370700181307F770B357F748E5CBB0
:1074B00097D7FB1F83A707AEA1DF9C43B1DB2285D3
:1074C000829739F5C1BFF977F917AA972947B3C74A
:1074D00007086366F70C1767020013072754B3C742
:1074E000E7209C43BA978287F9779387A7FCAA97EE
:1074F000F146B3C70708E3F6F6FA3907E31CE5F8E7
:1075000097D7FB1F83A747A9E38407F0DC43E381F8
:1075100007F00965A2853905A5A883298400E38BB6
:1075200009F603C7090097D7FB1F9387E7D019EB2C
:1075300003C7290083C619002207558F9AA703C7DE
:10754000390098B394230947E396E6F403C709008A
:1075500001CB97D7FB1F238107CE03C5090005B7D1
:107560008C338A270D4798A3EF70A00CFDB71C44FD
:107570008823EFF06FD869BD97D7FB1F83A707A2B9
:10758000E38807E89C43E38507E80965A2852D05A4
:10759000829705BF1C449C23E39E07EE95BD896737
:1075A00093871704E318F5EE97D7FB1F83A7079F70
:1075B000E38007E69C43A285E1FF99BD3D476394C4
:1075C000E7064A2089671387D7006306E50013871B
:1075D0009701631AE50097D7FB1F83A7E79BE38911
:1075E00007E2DC43C9BFCD07E316F5EAC16717D749
:1075F000FB1F0357C7C4FD17631FF70097D7FB1F77
:1076000083A78799E38607E0DC43E38307E0096506
:10761000A2854D05B5BF97D7FB1F83A76797E38961
:1076200007DE9C43DDB71307E003E395E7E63C2064
:1076300005476398E7127C2097DAFB1F938ACA9369
:107640006390071083A70A006387070E83C90700AA
:107650002149683093078400BE853ECEEFE09FD27B
:1076600068B013064002814568109790FB1FE780C1
:10767000E0D43C30194693058400A307F1027C3026
:107680004818A309F1029790FB1FE780A0CC5E2069
:107690007010CA852318F1027E244E852313F1044D
:1076A0001E282314F1043E282315F1045C28230628
:1076B000F104FD57A306F1042317F104EFF02FB6F0
:1076C0003C309DE3DD47835804010358E4007430E7
:1076D0004E203EC23E28130784003EC0CA8705469E
:1076E0004E85EF80A07128B083A70A0081C711459D
:1076F000EFF0FF9A97D9FB1F9389898A03C5090088
:10770000E30805D097D5FB1F83C59589EFE03F8738
:10771000E30005D03430930710036389F60052204C
:1077200083C509004A873685EFE03F9897D7FB1F4E
:1077300023880786F1B997D9FB1F83C919B009BF00
:1077400097D7FB1F83A7078597D9FB1F83C9F9AE7E
:1077500099C3DC4399E31149EDBD81450145829709
:10776000DDBFF91793F7F70F13077002E364F7D241
:10777000176702001307472DB3C7E7209C43BA974A
:1077800082877C2097CAFB1F938A0A7FA9EB83A775
:107790000A00A9C383C907002149683093772500EF
:1077A000A5C305891307440168B02286CA854E85A2
:1077B0003ACEEFF0CFA63C3072479DF7DD478358B5
:1077C000C4010358A40174304E203EC27E2C3EC03A
:1077D000CA8731B797D9FB1F83C939A675BF97C729
:1077E000FB1F83A7277B97D9FB1F83C919A599C3C3
:1077F000DC4399E3114955B7814501458297DDBFC7
:1078000013078400BA853ACEEFE0DFB7724769BF4D
:1078100097C7FB1F83A78778E38C07BEDC43E38908
:1078200007BE22858297EDB697C7FB1F83A7077710
:10783000E38007BE9C47E5B722868D454A2065BE9A
:107840009305A10213051031EF50C2606C101305AF
:107850002031EF50226072208357C1024A2063E733
:10786000C70016240357A10263F7E6009305000240
:10787000EFC0A07E71BE6373E6007AA063F3D70009
:107880001EA45A24362412246E2001488147EFC0DA
:10789000807CBDBE2286B14555B797C7FB1F83A725
:1078A000E76FE38707B6DC479DBF2285EF00607B6B
:1078B00085B697C7FB1F83A7676EE38B07B49C4B06
:1078C000B9BF2285EF00F003A1B60145EF003013E8
:1078D00081B697C7FB1F83A7E76BE38D07BADC432D
:1078E000E38A07BA8145054582976DB697C7FB1FA6
:1078F00083A7476AE38007BADC43E38D07B8A28514
:107900000945DDB72286930560020DBF93F7150088
:1079100089CF97C7FB1F83A7676889C7DC4399C3D3
:107920000145829713C5140045B493F7250091CF04
:1079300097C7FB1F83A7076691C7DC4381C78145B3
:107940000545829713C5240041B413F54500E30DA6
:1079500005A697C7FB1F83A7676217D4FB1F1304F5
:10796000A48D89CF85475CA097C7FB1F83A787623B
:1079700091C7DC4381C781450545829748446C1017
:10798000EF8030756810EFF02F9297D7FB1F83D7E9
:10799000878481CF130600643386C702914517D5CB
:1079A000FB1F034565ABEFC07FB013C5440029BC86
:1079B000011122CC2A84554506CE26CAEFF0AFB479
:1079C000AA8413054002EFF00FB42AC61305500233
:1079D000EFF06FB3AA86228562443246F240B33597
:1079E0009000D24405616FC0206F397122DC06DE41
:1079F0000D472E84631AE500BA259625F22128301A
:107A0000CE21EFE0BFE899A809679306D700AA87BF
:107A1000631BD504BC21B9C317C4FB1F1304C45591
:107A20000C408DCDDC87BC31194691054808A3096F
:107A3000F1009790FB1FE780E091930700F03ED69E
:107A40001C40231801002313010202D48823700074
:107A50008145EFE0DFFC0545EFF06FE40545F250AE
:107A60006254216182809306E700E309D5FE930604
:107A700037016319D500A82175D101478146014618
:107A8000814541B76507E30BE5FC31476319E50024
:107A900017C5FB1F0345757AEFE09FEAC1B71307CF
:107AA00060026319E50017C5FB1F03451579EFE078
:107AB000FFED6DB741677D170145E392E7FAD831D5
:107AC000C947E31DF7F8F625D2250A24AE25EFC0F5
:107AD0004068854711C55D45EFF0EFA2B337A000C0
:107AE0004C202A2030007C84EF70F06B3C84BDF782
:107AF0009305A10013051031EF50C2356C0013053A
:107B00002031EF5022353C851A246373F7001EA400
:107B10003C863A2463F3E7003EA41E243A246373B0
:107B2000F7003EA42A20EF4061237A245624322411
:107B30000E242A2001488147EFC0C04F05B74111EC
:107B40004AC006C622C426C217D9FB1F1309C99012
:107B5000034779009307F00F6302F706AA8439CD33
:107B6000682551059780FB1FE780006F2A8439C57F
:107B70009307000D1EA1D9473CA1DE205EA1FC2089
:107B80007CA1FC307CB19C241CA5DC345CB5F024C9
:107B900070A515C28C48510508C89780FB1FE78067
:107BA000607BA285224403457900B2409244024999
:107BB00041016FC08FE923280500E5B7B240224498
:107BC0009244024941018280C1679386E7FF2A8778
:107BD000639DD50097C7FB1F83A7073A8DC39C23DE
:107BE0000D45639FE7006FC02044FD174945639929
:107BF000F50097C7FB1F83A72738F5F78280494513
:107C00008280397122DC06DE26DA4AD84ED652D47A
:107C100056D25AD0182185472A84630BF7001025C5
:107C2000930695009305E1010545EFE0CFDA0DEDF0
:107C30008147014514201147638FE60217C7FB1FD8
:107C40000327C73618338D466307D7028DC705C78C
:107C500011ED0145F2506254D2544259B259225AA0
:107C6000925A025B216182801C21E9B7854663112B
:107C7000D7048D8BF9DF0830930524002EC6EFE082
:107C80006FF008B017C9FB1F130989328327090059
:107C9000AA8981449DC3B24517CAFB1F130A8A31C2
:107CA000130BF00F83470A0063EBF400814481A0BB
:107CB0008946E310D7FA858B75BF054561BF8327D9
:107CC0000900939A4400D6979823630C670598336C
:107CD000631937051946138527002EC69780FB1FA9
:107CE000E780C078B24515CD83240900D6941820CA
:107CF0009147C1E8E30FF7F483240900B9D883461C
:107D00000A0081471306F00FE385F6F403C8040068
:107D100013850401630BC800850793F7F70FAA8446
:107D2000E5B7850493F4F40FB5BF98A01C30138514
:107D3000240019469CB09780FB1FE780A0610824AF
:107D400091659385F57105059780FB1FE7800031EC
:107D500005C1182091476314F702C8C41024930585
:107D600094000505A30FC5FE9780FB1FE780805E8A
:107D70001C24A1F708207D1513351500E1BD88C42A
:107D8000F1BF6311F706C8441C2405C11021630D1F
:107D9000F604182091476317F706C84419C5978061
:107DA000FB1FE780C03823A6040008249165938553
:107DB000E57105059780FB1FE780402A05C1182063
:107DC0009147631AF704C8C410249305940005056D
:107DD000A30FC5FE9780FB1FE780C05708243335EB
:107DE000A0008DBD88444DB793059400050597808C
:107DF000FB1FE780A0678547E31DF5F85545EFE0D9
:107E00009FF09DBF884455D19780FB1FE7802032AB
:107E100023A4040059BF88C445BF397122DC4AD865
:107E20004ED652D406DE26DA56D25AD05ECE2A84F8
:107E3000130925000831CA8517CAFB1F130A0A1740
:107E4000EFE04FD408B083270A000D47AA899C337E
:107E50006391E70217CAFB1F130A8A1583270A00DA
:107E6000814497CAFB1F938AEA1463930710054560
:107E70002DA0EDD3144C70389305E1000545EFE0DB
:107E80008FB5AA841DC903270A0085461C21183313
:107E90006310D7028D8BDDFF0145F2506254D2543E
:107EA0004259B259225A925A025BF24B21618280A6
:107EB0008946858BE310D7FAF9BF1C2011476385EB
:107EC000E7002D47E39AE7FC97CAFB1F938A4A0E07
:107ED00083A70A00014A97CBFB1F938BAB0DCDDF25
:107EE00003C70B00B3470A0863E4E700A5F46DB7C6
:107EF00003A50A00131B4A001C205A951821631081
:107F0000F7021C31639D37011946CA850905978020
:107F1000FB1FE780A05501C583A40A00DA94050A77
:107F2000C1B783A9840059A80C4C13851900978008
:107F3000FB1FE780A05385476317F5085545EFE021
:107F40009FDC4DC191BF1C2011476385E7002D4781
:107F5000639DE700C8C470380505A30FC5FE0C4C2F
:107F60009780FB1FE780003FB5A888C4EDB7850464
:107F700003C70A00B3C7040863F8E70603250A002D
:107F8000139B44001C205A951821E312F7FE1C3164
:107F9000E39F37FD1946CA8509059780FB1FE780D7
:107FA000E04C71D583240A001C201147DA946385C4
:107FB000E7002D47E397E7F683A9C4007C3803C6A2
:107FC0000900E303F6F64E859780FB1FE780201635
:107FD000683891659385E57105059780FB1FE780FB
:107FE000E00735F1E39504E803C70A0083240A009B
:107FF00081479306F00FE3FCE7E68C20138604012B
:108000006387D5008507B284B3C70708EDB7E3805F
:1080100004E61C20CA85138524009CA01C30194648
:108020009CB09780FB1FE780E032683891659385AC
:10803000F57105059780FB1FE7804002E30905E223
:1080400018209147631DF700C8C470380505A30FB9
:10805000C5FE0C4C9780FB1FE780C02F09BD88C46C
:10806000EDB701114AC806CE22CC26CA17C9FB1F9C
:108070001309893E034779009307F00F630DF70654
:10808000AA8435C961459780FB1FE780E01C2A84DC
:108090003DC19307000D1EA1D5473CA1BC3093857F
:1080A00084002EC63CB1DE205EA1FC207CA1E8301D
:1080B000EFE04FADB24568B01946130584009780D4
:1080C000FB1FE7802029FC24A285034579007CA4BE
:1080D0009E281EA8BC283CA8BC383CB8DC285CA85C
:1080E000DC385CB8FC287CA86244F240D2444249A7
:1080F00005616FC08F95F2406244D24442490561E8
:108100008280411126C206C622C497C4FB1F9384F5
:10811000A434F8309307F00F6309F7022A8415C5D9
:1081200019459780FB1FE7802013AA8519CD930777
:10813000000D1EA1DD473CA15E202244B2405EA19D
:10814000E830924441016FC04F90B24022449244C3
:1081500041018280011126CA97C4FB1F938444E524
:108160009C4006CE22CC4AC84EC652C49DC32A8922
:10817000AE89131A45000144884063144403638C9C
:1081800009049780FB1FE78080FA97C7FB1F23A194
:1081900007E2F2406244D2444249B249224A0561B0
:1081A0008280B3078500884709C99780FB1FE78055
:1081B00000F89C40A29723A407009C40A297C847C0
:1081C00009C99780FB1FE78080F69C40A29723A6F1
:1081D0000700410455B755DD228681459780FB1F76
:1081E000E780C01D944081477D5613F7F70FE37277
:1081F00027FB13974700369710A38507FDB77971C2
:1082000052CC17CAFB1F130A6ADA83270A0006D664
:1082100022D426D24AD04ECE56CA5AC85EC6E9C724
:108220002A8997CAFB1F938AEAD8814419ED97C619
:10823000FB1F83A6E6D791CA03C60A0081479305B0
:10824000F00F13F7F70F6369C70213953400210588
:108250009780FB1FE78040002A8415E9214597801D
:10826000FB1FE78060FF2A8435C1C5679387073D00
:108270001CC123220400A9A0139747003697182396
:108280006305B700850493F4F40F85075DBF93077A
:1082900000FD1CA18547A30025013CA124B1F1D814
:1082A0001309850023222501814917CBFB1F130BDE
:1082B0002BD0930BF00F83C70A0063F3F900A1E002
:1082C00083270A00A2858823EFB03FF803C50A0080
:1082D0008145493503250A009780FB1FE78020E58B
:1082E00097C7FB1F23A407CCB250225492540259C3
:1082F000F249624AD24A424BB24B456182808325A1
:108300000B0093974900BE959C216383770323005C
:10831000F9009C3113052900FD14A300F90019464A
:10832000890593F4F40F9780FB1FE780A0022109D1
:10833000850993F9F90F41B797C7FB1F83A707C7B3
:10834000A9C7411122C406C62A8415E10945EFE0F8
:108350009F9B2A8601C9854517C5FB1F0345C50F8D
:10836000EFC0CF940545EFF0AFE42A8411C98545ED
:1083700017C5FB1F0345450EEFC0AFBC2285413535
:10838000B2402244054541018280014582808967CF
:108390009386B7006315D5009C45882371BF9386EB
:1083A000C7006317D5009C458546882319C9FDB7CA
:1083B00093861704E302D5FE938727048146E304DE
:1083C000F5FE36858280011106CE22CC26CA4AC827
:1083D0004EC652C456C261C13C312A898DC3444144
:1083E00099CC5945EFE03F92814997CAFB1F938A88
:1083F000EABB131A45608347390063EBF900F2408A
:108400006244D2444249B249224A924A056182807A
:108410008387840263C8470783A70A00A5C7268508
:10842000EFF02FFE25C1882451059780FB1FE780C0
:10843000A0E22A8421C99307000D1EA1B5473CA1E3
:108440009C201946938524003CB18387840215053E
:108450007CA19C30A30FF5FE9780FB1FE78080EF87
:10846000902450A415C61305440108C893859400B0
:108470009780FB1FE78000EE83A70A00A285882370
:10848000EFB0BFDC85099384940293F9F90FA5B787
:1084900023280400D5B797C7FB1F83A727B1A5D30F
:1084A000B93B6244F240D2444249B249224A924A1C
:1084B000014505616FF0CFCF797106D622D426D25F
:1084C0004AD04ECE52CC56CA5AC85EC655CD3C3163
:1084D0002A898DC744419DC05945EFE0DF82890458
:1084E000814997CAFB1F938A6AAC130B00FDC14BED
:1084F000131A45608347390063EDF900B2502254E6
:1085000092540259F249624AD24A424BB24B4561F7
:1085100082808387D40063C4470783A70A00A5C36A
:1085200051459780FB1FE78020D32A8429C9230067
:108530006501A30005002301750183C7E4FF194607
:10854000A6853CB18387D40015055CB583C7F4FFCD
:10855000A30FF5FE9780FB1FE780C0DFFC2093850B
:1085600074001305C4003CB419469780FB1FE780D4
:1085700060DE83A70A00A2858823EFB01FCD85099E
:1085800093F9F90FC104BDB797C7FB1F83A707A2D3
:10859000B5D7B5312254B25092540259F249624AC9
:1085A000D24A424BB24B014545616FF06FC07971C1
:1085B00006D622D426D24AD04ECE52CC56CA5AC85B
:1085C0005EC662C466C2630C05223C312A8985CB33
:1085D000404115C45945EFE00FF30904814917CA1A
:1085E000FB1F130AAA9C914B354C175B0200130B1F
:1085F000AB4F931A45608347390063EFF900B250DF
:10860000225492540259F249624AD24A424BB24B26
:10861000224C924C456182808307A40063CA57159F
:1086200083270A0063860714834CE4FF93F70C0149
:10863000CDC793870CFF93F7F70F6369FC00B3C7AF
:1086400067219C43DA978287230F04FE1305E4FF1A
:10865000EFF0AFFC630E05108347E4FF63EFFB1000
:1086600005476398E70A51459780FB1FE780C0BE26
:10867000AA84630F050E930700FD1CA1C147A30048
:1086800005003CA18347E4FF1946A2853CB183075E
:10869000A40015055CB58347F4FFA30FF5FE978092
:1086A000FB1FE78020CB7C2419469305F400BCB463
:1086B0001385C4009780FB1FE780C0C965A085476C
:1086C000230FF4FEA30A040051B78947230FF4FED9
:1086D000B5BF8D47E5BF9147D5BF93F78C0099C3D0
:1086E000AD47EDB713F71C0093F74C0011C799C3C2
:1086F0009547F9B7A147D9BF13F72C0011C799C304
:10870000A5477DBF9947D9B799C3A947C1B79D4729
:1087100075BF483851059780FB1FE780E0B3AA84F6
:1087200021C99307000D1EA1B5473CA18347E4FF73
:108730001946A2853CB18307A40015057CA1834797
:10874000F4FFA30FF5FE9780FB1FE780A0C0503811
:10875000D0A419C61385440188C88325640199BF34
:1087600023A8040083270A00A6858823EFB0FFAD65
:10877000850993F9F90F7104BDBD48381305050249
:108780009780FB1FE78040ADAA847DD19307000D41
:108790001EA1C9473CA18347E4FF93FC0C06194680
:1087A000B3E797013CB18347F4FFA2851505A30FFA
:1087B000F5FE9780FB1FE780E0B97C201946930502
:1087C000F400BCB47C3013853401DCA41C24DCB47C
:1087D0001C34FCA48307A400FCB45E249EA87C2463
:1087E000BCA89780FB1FE780E0B6503890BC09C654
:1087F00013850402C8CC95B723AE0400A5B797B77C
:10880000FB1F83A7A77AE38C07DEEFF05F9F22545C
:10881000B25092540259F249624AD24A424BB24B88
:10882000224C924C014545616FF08F9817B7FB1FA2
:108830000327C77705CB1823AA870D456315F702D1
:108840004111854517C5FB1F034505C106C6EFB09D
:108850005FEF13050003EFF09F9AB240014541011D
:108860006FF00F954945828079714AD017B9FB1F87
:108870001309C9738327090006D622D426D2CDEB6B
:1088800017C4FB1F130444BD5820C947298B51CB83
:108890009165AA849385D57111459770FB1FE78078
:1088A000E07B2320A900CD472DCD78309307F00F32
:1088B0006314F7009C207CB01146A6859780FB1FAF
:1088C000E78040A9930531011305F041EF20122400
:1088D00097C7FB1F93874796A02303473101333483
:1088E000800011C3090413051002EFE0CFC1137615
:1088F000F50F0589E14715C5154532C6EFE0AFC054
:10890000BC20E8841945230AF100EFE0CFBF3246CE
:10891000AC30E8867C08380854082285EFB0807BAC
:10892000AA87B2502254925402593E8545618280F2
:10893000C547C5BF1971A2DCA6DA86DECAD897C4BE
:10894000FB1F938464B1DC204944A18BB9CF97B756
:10895000FB1F83A7A7654144A9EB2A89EFE05F8C41
:108960009C2455446373F50497B4FB1F9384C4603F
:108970009C4045449DEB91659385C5712945977051
:10898000FB1FE780A06D88C04D4405C12946CA85FC
:108990009780FB1FE780009C13056002EFE0AFB6F5
:1089A0001374F50F058909E96144F6502285665470
:1089B000D654465909618280130600038145880018
:1089C0009780FB1FE780809F4145EFE0CFB32316E0
:1089D000A1043D45EFE02FB32319A1043545EFE095
:1089E0008FB2231CA1043945EFE0EFB1231FA1048E
:1089F0002145EFE04FB12312A1061D45EFE0AFB0D6
:108A00009C402315A106136424009C33F1C72D4517
:108A1000EFE06FAF2310A1043145EFE0CFAE231399
:108A2000A1041305C002EFE00FAE2317A104130544
:108A3000B002EFE04FAD231AA10413059002EFE05E
:108A40008FAC231DA1041305A002EFE0CFAB2310D0
:108A5000A10613058002EFE00FAB2313A106130557
:108A60007002EFE04FAA9C402316A106A83393851D
:108A70004700EFD09F8D2AD69305F1031305F041EF
:108A8000EF20D20897B7FB1F9387077BAC230347E0
:108A9000F1033256B335B00011C389059440FC0090
:108AA0002287A8223EC8930721053EC6BC083EC4C3
:108AB0009307E1053EC2DC103EC09308A1061308EF
:108AC00061049C009106EFB060612A84E30F05EC1D
:108AD0000D45EFE0CFDCD1BD2545EFE0CFA223105F
:108AE000A10429451DBF97C7FB1F83C72797A18BEB
:108AF00017B5FB1F1305054B91E301456FD0AFE19F
:108B000097B7FB1F2388074AFD5717C7FB1FA3080A
:108B1000F79497B7FB1F23AD074897B7FB1F23A711
:108B2000074897B7FB1F93872773170700001307A2
:108B3000478698C31707000013072789D8C317076C
:108B400000001307A79798C717070000130767A629
:108B5000D8C717F7FFFF1307C7FE98CB97B7FB1FC0
:108B60009387474417F7FFFF1307470698C317F784
:108B7000FFFF1307C7E7D8C38280411122C426C272
:108B800006C617B4FB1F1304E442AA8408208545D7
:108B9000EFF04FDC97C7FB1F83C7478CA98BBDC77E
:108BA00017B5FB1F1305456B04A0EFD02FD697B464
:108BB000FB1F9384E43F9C4099C74D45B24022443B
:108BC000924441018280082019E10145C5BF9165A9
:108BD0009385B57112059770FB1FE780204888C008
:108BE00069DD1020814512069770FB1FE780007D2C
:108BF000142090408147FD5513F7F70FE377D7FC1A
:108C00001397470032970CA38507FDB7014597B727
:108C1000FB1F2381073AEFD06FCF45BF17B5FB1F6E
:108C20000325C53511CD411106C69770FB1FE7809E
:108C30000050B24097B7FB1F23A207344101828046
:108C4000828001111305700306CEEFE0CF8B2AC698
:108C500013058003EFE02F8B2AC413059003EFE088
:108C60008F8A2246B245F240AA86054505616FB05B
:108C7000A0455D711305D00386C6A2C4A6C2CAC0B2
:108C8000EFE06F882A841305C003EFE0CF87AA8442
:108C90001305E003EFE02F872A891305F003EFE0C7
:108CA0008F868A871377F50F9376F90F13F6F40FF3
:108CB0009375F40F0545EFB06043B64026449644E3
:108CC000064961618280011122CC06CE26CA0D4779
:108CD0002E846317E504B831E947CA2197B4FB1F16
:108CE000938484556315F700FE206387A70497A03B
:108CF000FB1FE78080E7722011C172A53A24162479
:108D00004E202830EFD09FB85A20FE206314F70081
:108D1000FD57FEA00545F2406244D24405618280C1
:108D200009674D07AA87631CE500BC2131476385AD
:108D3000E7004547E390E7FEEFD00FC5E1BF3147BD
:108D40006319E50017B5FB1F03455571EFD05FBFF1
:108D5000D1B7130760026319E50017B5FB1F034580
:108D6000F56FEFD0BFC27DB741677D170145E39432
:108D7000E7FAD831C947E310F7FACC212A203000AE
:108D800023140100EF60303D71B71971A2DC17B4F4
:108D9000FB1F1304A41E1C4086DEA6DACAD8CED65A
:108DA000D2D4D6D2DAD00545638A070C9305F105F3
:108DB0001305F041EF2082559305F1051305F041AD
:108DC000EF20C25497B7FB1F93870747BC23034785
:108DD000F105B337F00011C389071840BEC6283328
:108DE00093054700EFD06FD61840AAC40D452C2339
:108DF000AEC2EFD05FF1AAC01145EFD0DFF0832AF9
:108E000004002ADE654503C7AA0003CBBA003ADC9A
:108E1000EFD07FEF2A846945EFD0FFEEAA84714539
:108E2000EFD07FEE2A896D45EFD0FFEDAA89754519
:108E3000EFD07FED2A8A7945EFD0FFEC2648B64780
:108E40006257F256064696451375F50F137AFA0FD8
:108E500093F9F90F1379F90F93F4F40F2ACC131443
:108E6000446002D002CE52CA4EC84AC626C422C2AC
:108E70005AC093884A000545EFB0E01FF65066548B
:108E8000D6544659B659265A965A065B09618280CD
:108E9000411122C44AC006C626C217B9FB1F1309D6
:108EA000F912834709001307E00F2E846382E70459
:108EB0001307F00F6385E70211459770FB1FE780EA
:108EC000A039AA8509CD930700FD1CA189473CA1C3
:108ED000854700B13CB103450900EFB00FB7F95722
:108EE0002300F900B24022449244024941018280A9
:108EF000AA8411459770FB1FE7800036AA857DD1B3
:108F0000930700FD1CA1894700B13CA124B1224474
:108F1000B2409244024917B5FB1F0345250B41019E
:108F20006FB0AFB279714AD017B9FB1F13090905A9
:108F30008327090022D406D626D24ECE52CC4544F1
:108F4000C5EB97B4FB1F93842451DC204944958BD7
:108F5000C5C32E8A916597B7FB1F2389A706AA89E7
:108F60009385757131459770FB1FE780200F232093
:108F7000A9004D4435CD23003501A3000500294645
:108F8000D28509059770FB1FE780C03C03270900C5
:108F900091463C2363E7F606CD4691CF0546F5465C
:108FA000638BC7000946C9466387C7000D46C146A3
:108FB0006383C700D54634A3930571001305F041C0
:108FC000EF20C2349C83C5E317B7FB1F0347E72696
:108FD0008D47631AF708EFD00FC52C00EF70700FA4
:108FE0002800EFD07FAC4545EFD0FFD125E5014407
:108FF000B2502285225492540259F249624A456184
:109000008280ED1793F7F70F95460544E3E2F6FEED
:10901000975602009386C6B0B3C7D7209C43B69735
:10902000828789473CA319A0230107006545EFD03B
:109030009FCD9307F007E301F5F8032709003C23D0
:1090400093E707043CA38DBF8547E9BF9947D9BF84
:109050009147C9BF130600643306C50288209145B5
:10906000EFB0CFC469B715332A8451D1EFF01FBBDD
:1090700041B7011126CA97B4FB1F938424F09C408A
:1090800022CC06CE4AC84944A1C79C230D44639113
:10909000A70417B9FB1F1309293C0345090089459B
:1090A000EFB02FEA03450900914597B7FB1F239DB9
:1090B00007F0EFB00FE99C400147814680B31306EB
:1090C000F100854785450145DC87EFA0B07F2A8404
:1090D000F24022856244D2444249056182800111F6
:1090E00006CE22CC26CA4AC84EC68547631EF50660
:1090F00017B4FB1F130444ED1E20B1CB17B7FB1FA1
:109100000347C71329E71307B003636EF70297B449
:10911000FB1F9384643488208945EFB08FE21220CE
:109120009307006488203306F6028945EFB00FB834
:1091300097B7FB1F239A07E8F2406244D2444249A2
:10914000B24905618280938747FC1EA0F5B797B7A7
:10915000FB1F83A7A7E2EDD36244F240D244424909
:10916000B2498823056131B797B9FB1F938909E19B
:1091700083A70900F1D317B9FB1F1309E92D834712
:109180004900918BD5DB89476311F5062D45AE84E7
:109190009770FB1FE780400C2A8459DD930700FD80
:1091A0001CA1E547A30005003CA1BC3015051946EC
:1091B000230FF5FEDC2093855400A30FF5FE977076
:1091C000FB1FE7802019034559009307F00F631533
:1091D000F50083A709008823A2856244F240D244A7
:1091E0004249B24905616FB04F8603450900894580
:1091F000EFB02FD56244F240D2444249B24997B70A
:10920000FB1F239307DC05616FF05FA197B7FB1F7E
:1092100083C7C724958B89CF97B7FB1F83A707DA2E
:1092200091CB854717B7FB1FA301F7DA6FF07FA13A
:10923000494582804145828097B7FB1FA38707D8A5
:10924000854501456FA0D06897B7FB1F83C70721ED
:10925000958B81CB854717B7FB1F2308F7D66FF097
:109260005FA14945828097B7FB1F238007D68145C0
:1092700005456FA0F06797B7FB1F83C7271E958B27
:10928000638B0712011122CC06CE26CA4AC84EC6ED
:109290009307C01C328463FAC7000945F240624458
:1092A000D2444249B2490561828097B7FB1F83A728
:1092B000E7CC6384071097B7FB1F938737D1B68934
:1092C00094231307E00F639AE60E88A31305860024
:1092D00033450508ADC99165938565719770FB1F8E
:1092E000E780C0D7AA8455D917B9FB1F130989CDC8
:1092F0000325090009C59770FB1FE78040E313852C
:10930000840088C022868145232099009770FB1F26
:10931000E780C00A832709002286CE85884397709C
:10932000FB1FE780200383270900A286F240C2A327
:109330006244D2444249B249984305468D450545A9
:1093400005616FA0B0579165938555719770FB1FAC
:10935000E780C0D0AA8431D117B9FB1F130949C6D1
:109360000325090009C59770FB1FE78040DC1385C2
:10937000840088C022868145232099009770FB1FB6
:10938000E780C003832709002286CE858843977033
:10939000FB1FE78020FC83270900A286F240C2A3BE
:1093A0006244D2444249B249984305468D45054539
:1093B00005616FA0F050494582804945C5B59307C6
:1093C000C01C63FCA700094582800945F240624445
:1093D000D2444249B24905618280011122CC06CEB5
:1093E00026CA4AC84EC62A8425C1AE899165210580
:1093F00093856571334505089770FB1FE78000C6AC
:10940000AA8461D517B9FB1F1309C9BB032509003D
:1094100009C59770FB1FE78080D11385840088C041
:1094200022868145232099009770FB1FE78000F971
:10943000832709002286CE8588439770FB1FE7802B
:1094400060F183270900C2A397B7FB1F83A707B367
:1094500085CF97B7FB1F83C76700958B85CB97B7E1
:10946000FB1F83A727B691CF9843D6236244F240CF
:10947000D2444249B24905468D45054505616FA074
:10948000F04301478146DDB7014589B749453DBFF6
:109490009307C01C63FCA700094582800945F24080
:1094A0006244D2444249B24905618280011122CC12
:1094B00006CE26CA4AC84EC62A8425C1AE89916501
:1094C000210593855571334505089770FB1FE7808B
:1094D000E0B8AA8461D517B9FB1F130969AE03254B
:1094E000090009C59770FB1FE78060C413858400DD
:1094F00088C022868145232099009770FB1FE78052
:10950000E0EB832709002286CE8588439770FB1FF6
:10951000E78040E483270900C2A397B7FB1F83A716
:10952000E7A585CF97B7FB1F83C747F3958B85CBFF
:1095300097B7FB1F83A7C7A891CF9843D623624450
:10954000F240D2444249B24905468D450545056180
:109550006FA0103701478146DDB7014589B74945FE
:109560003DBF9307C01C63F4A70009458280797151
:1095700022D406D626D24AD04ECE2A842DC1AE8918
:109580009165210593857571334505089770FB1F1B
:10959000E780C0ACAA840945A9C817B9FB1F130905
:1095A000E9A10325090009C59770FB1FE78020B8D2
:1095B0001385840088C022868145232099009770F6
:1095C000FB1FE780A0DF832709002286CE85884322
:1095D0009770FB1FE78000D883270900C2A397B7C5
:1095E000FB1F83A7A79989EB0145B25022549254DF
:1095F0000259F2494561828097B7FB1F83C707E68E
:10960000958B4945FDD36C001305D030EF309204A3
:10961000B24793F7070FE9DB97B7FB1F83A7079ABA
:109620009443D2238D450545EFA0502A7DBF97B7BF
:10963000FB1F83A7279989CFD2238C43411106C6EC
:109640009770FB1FE78000D1B24001454101828045
:109650000945828097B7FB1F83A7C79685C717B7B1
:10966000FB1F0327E795894719CF52230C4341116C
:1096700006C69770FB1FE780E0CDB24081473E856C
:109680004101828089473E85828097B7FB1F83A76F
:10969000679385C717B7FB1F03274792894719CFE1
:1096A00052230C43411106C69770FB1FE78080CA06
:1096B000B24081473E854101828089473E85828054
:1096C000797126D206D622D44AD04ECE97B4FB1F4B
:1096D000938484B68D4783C9240063FAA7000945A3
:1096E000B250225492540259F24945618280982026
:1096F0002A844145E316F7FE9307F4FF93F7F70F2B
:10970000854663E8F60A2E89B1ED99452800EFC039
:109710007FA2A0A0914517B5FB1F0345E5D3EFB08D
:109720004F822800EFD04FB855E99305710013051B
:10973000F041EF10B23D9C83D1EB8D476318F408E4
:109740004545EFD04FDC59C137761800130606A007
:109750003306C502914517B5FB1F0345E5CFEFA0C2
:109760005FF6ADA01946814528009770FB1FE78082
:10977000E0C419462C004A859770FB1FE78000CF94
:1097800039FD19469305F00F28009770FB1FE780FD
:10979000E0C219462C004A859770FB1FE78000CD78
:1097A0001DFD1946CA8528009770FB1FE78080BA07
:1097B0008DB7630FE400914517B5FB1F0345C5C97D
:1097C00097B7FB1F238B07A6EFA0BFF7014509BF83
:1097D000C8442C00EF70E00FA0A00DDD2381340100
:1097E00001B797B7FB1F83C767C7918B8DC3411123
:1097F00017A5FB1F1305457C06C6EFC01F93B2409B
:10980000FD5717B7FB1F231CF7A2410182800145BA
:109810006FC0BF91FD5717A7FB1F2309F77AF957B0
:1098200017A7FB1FA304F77A97A7FB1FA38F07783F
:1098300097A7FB1F238B077897A7FB1F2396077813
:1098400097A7FB1F23A0077897A7FB1F23AA0776DC
:1098500097A7FB1F23A4077697B7FB1F938707A142
:10986000170700001307E72098C317070000130726
:109870004787D8C317F7FFFF1307675198C717F734
:10988000FFFF1307473CD8C717F7FFFF1307A73E93
:1098900098CB97F7FFFF9387474317A7FB1F232D0D
:1098A000F7708280411126C297A4FB1F9384046D38
:1098B0009C4006C622C495CB2A840D459770FB1F99
:1098C000E7808099AA8519C9930700FD1CA18D47DF
:1098D00000B13CA19C408823EFA03F9719C42244CB
:1098E000B240924441016FF06FB3B24022449244BF
:1098F0004101828079714AD017A9FB1F13090968B9
:109900008327090006D622D426D24ECE6383070EC3
:1099100098338547AA8497B9FB1F9389E99163011E
:10992000F70483C749008DE70D459770FB1FE7805B
:10993000A092AA8501CD930700FD1CA1914704B117
:109940003CA1832709008823EFA03F90EFF00FADE3
:109950000545B250225492540259F2494561828021
:1099600097A7FB1F83A7076689CB9443D223930550
:10997000E1000545EFC03F8611ED0145EFD0AFB8DE
:109980002A8621C6894517B5FB1F0345E5ACEFA024
:10999000FFB125A81C21858BEDD30545EFD0AFB6CF
:1099A0009307B0032A8463F1A7045D66130606706B
:1099B000894517B5FB1F034525AA130444FCEFA0F6
:1099C0005FD097A7FB1F2391876083270900094772
:1099D00098B383C7490091C797B7FB1F23800786B9
:1099E00085BF2685C135ADB7930700643306F50200
:1099F00049BF0145B9BF411122C42A840D4506C69D
:109A00009770FB1FE78040850DC1930700FD1CA1E7
:109A1000CD4700B13CA12244B240AA8517A5FB1F47
:109A20000345C55A41016FA05F82B2402244410103
:109A30008280411122C42A840D4506C69770FB1FFF
:109A4000E78080810DC1930700FD1CA1ED4700B1A7
:109A50003CA12244B240AA8517A5FB1F0345055728
:109A600041016FA08FFEB2402244410182805A2101
:109A70000111896606CE22CC26CA13866600AA8703
:109A80006316C7009C4701458C2371A81386060402
:109A90006365E60413865603636FE600138696003B
:109AA000630BC7081386A600630DC712A1066309DE
:109AB000D7060145A5A8F9769386A6FC3697A94650
:109AC00033470708E3E7E6FE974602009386C6069B
:109AD0003347D72018433697028713861605630746
:109AE000C71893862605E316D7FC1C45802397A745
:109AF000FB1F83C7874D2285639D07160D45976021
:109B0000FB1FE7806075AA850DC1930700FD1CA1AE
:109B1000F14700B13CA117A5FB1F0345254B91A2BE
:109B20009C4705458C23EFF0AFB60545F2406244F3
:109B3000D2440561828017A7FB1F032727440145F4
:109B400075D79C47882359E985471CB30545EFA085
:109B5000604DE1BF1C4597A4FB1F93843447130756
:109B6000E00F80239C20638BE7021307F00F6384D0
:109B7000E70211459760FB1FE780006EAA8501CDC3
:109B8000930700FD1CA1894700B13CA1A30105007A
:109B90008820EFA08FEBF9579CA041BF97A4FB1F33
:109BA0009384C43D9C400145D1D305E805447D45DF
:109BB0004085EFD04F95688613050002EFD0AF9433
:109BC0009C40C8851307B10080B374001306A10040
:109BD00085450545EFA0004F89BF2285EFF09FCC5A
:109BE000A9B79C476244F240D244882305616FF0D4
:109BF0007FD01C4509458C233DB71C4588232DE5A6
:109C00006C001305D030EF30E224B247414793F7A0
:109C1000070FE38CE7F09305B10013056031EF30D7
:109C2000622388858545EFA0A04A01B71C458023A3
:109C300097A7FB1F83C7773922859DE70D4597605E
:109C4000FB1FE7806061AA85E30105EE930700FD35
:109C50001CA1D14700B13CA197A7FB1F83A70732E6
:109C60008823EFA08FDED1B57933C1B51C45882399
:109C700019C1C1335DBD85450545EFA0604775B588
:109C8000411122C417A4FB1F0344447D06C6158856
:109C900009CC17A5FB1F1305655DEFC06FC84D44C8
:109CA000B24022852244410182800145EFC04FC766
:109CB000C5BF9821937625009377D70F99C29367F4
:109CC000270093F6F707131745606354070093E6E0
:109CD00007081378850093F7760F6304080093E76D
:109CE00086009376050299CE93E707029CA16357FD
:109CF00007001C2293E7C7001CA282801375A502EF
:109D00006DF9828093F7F7FD9CA1E34407FE9377FA
:109D1000A502E5F37DF11C22CD9BF9BF2D45631C07
:109D20000710011126CA4AC84EC606CE22CC982179
:109D3000BE8989472E89B684631EF704DC413284CC
:109D4000983394232207558F8D66938746A0131668
:109D5000576063C9C7029386F69F63DDC602F57735
:109D60009387F75F3E978D47C8453347070863E7FA
:109D7000E702974602009386E6DE3347D7201C436E
:109D8000B6978287938766AA630EF608938686B88D
:109D9000630FD60823900400054525A09760FB1F9C
:109DA000E780E064334605083356360B92A08325DE
:109DB000C9001DA01E2109479AA01CA0A1831CB0A8
:109DC0000145F2406244D2444249B2490561828071
:109DD00099479EA01946AA8522859760FB1FE780B8
:109DE0006057F9BF85479EA01C211CA0D1BF05C9A3
:109DF000A1479EA01E211CA01E21A1831CB03E21B4
:109E00003CA03E21A1833CB05E215CA05E21A183E9
:109E10005CB07E217CA07E21A1837CB055B72390CD
:109E2000040079BF85479EA0DC459C237DBFE147A8
:109E30009EA06146ADBF8280797122D44AD006D6F9
:109E400026D24ECE52CC56CA3A89982189472E84C2
:109E5000631DF7025C40B684B28503C817009423E3
:109E60008D6722083368D800938627A0131858609E
:109E7000630BD8102A8A63CC0601938607A0630B74
:109E8000D802938717A06300F80A854711A81387A3
:109E900037A0630FE80A138767AA8D47E317E8FE28
:109EA000B250225492540259F249624AD24A3E8533
:109EB00045618280484432C69760FB1FE78020538B
:109EC0009D4733450508E36D25FD97AAFB1F938A3F
:109ED0002A1183C70A00B3099900B24563D4370138
:109EE000B5477DBF48442686B3C909084A9597609F
:109EF000FB1FE780204603C60A004844814505064B
:109F0000330636414E959760FB1FE780204B97A79D
:109F1000FB1F83A7270D99E3814759B79C438145D0
:109F2000E5DF528525A0AD47E31C09F6E39AE4FA84
:109F30001C321822A207D98F58441EA397A7FB1FD3
:109F400083A7470AF1DB9C438545F9D78297E9B798
:109F500017A7FB1F034777088D4739D3AD47E31198
:109F600009F49947E39EF4F6484419469760FB1FAD
:109F7000E780403E97A7FB1F83A7C706D1DF9C431E
:109F8000C1DF8D4579BF17A7FB1F034787F4218BDE
:109F90008D4719D7AD47E31509F08547E392F4F4EF
:109FA000182293070008E3EDE4EE5C4498A3ADB7F4
:109FB000411122C4094497A7FB1FA38D87F097A7DF
:109FC000FB1FA38887F097A7FB1F238487F097A721
:109FD000FB1F23A9070097A7FB1F238A07FE97A74C
:109FE000FB1F238F07FE97A7FB1F239A07FE97A748
:109FF000FB1FA38407FEA1471946814517A5FB1F38
:10A00000130545FD06C617A7FB1FA303F7EC9760D2
:10A01000FB1FE780A03A97A7FB1F238B87EAB707B0
:10A02000A00017A7FB1F130727EA938707051CC388
:10A03000B707E8035CC397A7FB1F238587E885471D
:10A040006146814517A5FB1F1305853617A7FB1F22
:10A05000A309F7E697A7FB1F238587E697A7FB1FB2
:10A06000A38087E697A7FB1F238407F69760FB1F53
:10A07000E780C03413060013814517A5FB1F1305A5
:10A08000252097A7FB1F238D87E297A7FB1FA3809F
:10A0900007F49760FB1FE780603297A7FB1F938749
:10A0A00067DCB240224417070000130767C798C354
:10A0B00017070000130787D8D8C323A4070041015E
:10A0C0008280797122D426D206D64AD04ECE52CC86
:10A0D000A1472E84B28463EBA70017470200130741
:10A0E00067A93345E5201C41BA978287930710087A
:10A0F0006304F51C63ECA70093072004630EF516B8
:10A10000930700086303F518094591A093072008F9
:10A11000E31CF5FE8547639BF50208229377250033
:10A1200095E797A7FB1F83C747EB1387F7FF97A513
:10A13000FB1F9385E514120792072E97A10750473E
:10A14000BE9585AA9307800F63FBB7006145B250A7
:10A15000225492540259F249624A4561828017AAF8
:10A16000FB1F130A2AD783470A0017A9FB1F1309ED
:10A1700029119207CA97C84709C99760FB1FE78052
:10A1800000FB97A7FB1F238D07E41306140013762B
:10A19000F60F916593850571328583490A0032C6B1
:10A1A0009760FB1FE78080EB83470A009209CA99FA
:10A1B000920723A6A900CA97C84749D932468145C4
:10A1C0009760FB1FE780801F83470A002286A685D1
:10A1D00092073E990325C9009760FB1FE78080170F
:10A1E00097A7FB1F238E87DE014595B78947E39F1D
:10A1F000F5F41E2217A7FB1F2313F7DEF5B78547DB
:10A20000E396F5F41C2217A7FB1FA308F7DCE9BFB0
:10A210009947E39DF5F21946A68517A5FB1F13057F
:10A2200065DB9760FB1FE780E0127DBFA147E39FDE
:10A23000F5F02146A68517A5FB1F1305E5C8D5B780
:10A240008547E395F5F01C2217A7FB1FA30BF7C664
:10A2500061BFE147E39CF5EE6146A68517A5FB1FAC
:10A26000130505157DBF8547E392F5EE1C2217A760
:10A27000FB1FA30EF7D48DBF8547E399F5EC1C2295
:10A2800017A7FB1F2307F7C485B78547E390F5ECB5
:10A2900097A7FB1F83C707C41387F7FF97A5FB1F6B
:10A2A000938505FE12072E97920750478820A10735
:10A2B000BE95EFF01FA00DBF8547E399F5E897A77E
:10A2C000FB1F83C7A7D1C9BFAA8721472E85636D0E
:10A2D000F700174702001307278CB3C7E7209C43FA
:10A2E000411106C6BA97828713072004638BE708DB
:10A2F00089473E85828017A7FB1F0347A7BD12072A
:10A3000097A7FB1F9387C7F7BA97CC47894785C1A3
:10A3100017A6FB1F0346C6CC9760FB1FE780800390
:10A3200031A097A7FB1F83D787CB9EA18147B2405F
:10A330003E854101828097A7FB1F83C717CA1CA1D6
:10A34000F5B7194697A5FB1F9385C5C8F1B72146F8
:10A3500097A5FB1F938545B7EF909FDBC1BF97A7DC
:10A36000FB1F83C717B6E1BF614697A5FB1F938507
:10A3700025045DB797A7FB1F83C777C5C9B7894772
:10A380007DB797A7FB1F83C7C7B49CA1814795B72B
:10A390006300053A97A7FB1F938767C39823631948
:10A3A0000738054798A397A7FB1F938767ED894652
:10A3B00098A717A7FB1F231A07EC17A7FB1F130764
:10A3C00067B394A397A6FB1F938686B6D8C7D4C35A
:10A3D0007D57630CE53413771500854529C717A60B
:10A3E000FB1F231C06EA094797A6FB1F938686B32B
:10A3F00017A6FB1F130616AE98ABD4CBD0CF85465D
:10A4000017A6FB1F2308E6AC2380E70217A7FB1F54
:10A410001307C7B0D8D394AF2384D70217A7FB1F65
:10A42000231507E88D451377250025C313974500AD
:10A430003E9797A6FB1F9386E6AE094654C317A81E
:10A44000FB1F130818A9854610A314A7232607018C
:10A4500023150700138715003347070817A8FB1FAC
:10A46000230EE8B612073E9710A314A717A6FB1FEA
:10A47000130686AA97A6FB1F938666B6890550C366
:10A480002315070054C7B3C505081377450025C336
:10A49000139745003E9797A6FB1F9386A6A80946EB
:10A4A00054C317A8FB1F1308C8A2854610A314A7FE
:10A4B00023260701231507001387150033470708D4
:10A4C00017A8FB1F230BE8B012073E9710A314A791
:10A4D00017A6FB1F130606A497A6FB1F9386F6AFCD
:10A4E000890550C32315070054C7B3C50508137762
:10A4F000850021CF139745003E9717A6FB1F130633
:10A5000066A250C30546894610A717A6FB1F13066F
:10A51000369C14A32315070050C713871500334733
:10A52000070812073E9714A397A6FB1F9386469E23
:10A5300054C3A14614A797A6FB1F9386A6A9890515
:10A540002315070054C7B3C505081377050121CFAC
:10A55000139745003E9797A6FB1F9386A69C094636
:10A5600054C317A8FB1F1308A896854610A314A769
:10A570002315070023260701138715003347070813
:10A5800012073E9710A314A717A6FB1F13060698E1
:10A5900097A6FB1F93864693890550C32315070092
:10A5A00054C7B3C505081377050221CF139745009B
:10A5B0003E9797A6FB1F9386E696094654C317A8B5
:10A5C000FB1F13082890854610A314A72315070026
:10A5D00023260701138715003347070812073E9704
:10A5E00010A314A717A6FB1F1306C69197A6FB1F5F
:10A5F0009386368D890550C32315070054C7B3C50C
:10A6000005081377050421CF139745003E9797A6B9
:10A61000FB1F93862691094654C317A8FB1F1308F6
:10A62000488A854610A314A723150700232607018F
:10A63000138715003347070812073E9710A314A786
:10A6400017A6FB1F1306468C97A6FB1F93864698FA
:10A65000890550C32315070054C7B3C505081377F0
:10A66000050821CF139745003E9717A6FB1F130639
:10A67000668B50C35146894610A717A6FB1F1306C9
:10A68000368414A32315070050C7138715003347DA
:10A69000070812073E9714A397A6FB1F93864686CA
:10A6A00054C3854614A797A6FB1F938666D08905D9
:10A6B0002315070054C7B3C505081375051039C91C
:10A6C000139745003E9797A6FB1F9386A68554C314
:10A6D000094685461795FB1F1305857E10A314A711
:10A6E0002315070048C713871500334707081207CB
:10A6F000BA9717A7FB1F1307A780D8C317A7FB1F7D
:10A700001307F78C890590A394A723950700D8C752
:10A71000B3C505089796FB1F9386C674414617A5D7
:10A72000FB1F1305E5B56F3000421305300345B933
:10A73000014582800111FD1522CC06CE328426CA45
:10A740003E864AC813F8F50FAD4763E8070B3A8910
:10A7500017370200130787463348E820832708008D
:10A76000B684BA9782878545EFB0FFB801E5EFF070
:10A770002FD10145F2406244D244424905618280B2
:10A780008945EFB05FB77DF52285EFE00FBFD5B704
:10A79000914532C6EFB03FB6324669FDCA8526857F
:10A7A000EFB01FACEFF0CFCDEFF0AF83EF60A07A4A
:10A7B000C9B7A14532C6EFB01FB4324645FDCA85C0
:10A7C0002685EFB0FFA92285EFE02FBBEFE0AFB108
:10A7D000EF60407679BFB14532C6EFB0DFB13246A7
:10A7E00051F9CA852685EFB0BFA72285EFE0EFB803
:10A7F000EFE06FAFEF60007475B70945A5BF7971E1
:10A800004ECEAE896C0022D426D24AD006D62A89F2
:10A81000B284EF00306E2A840DE1CE854A85EFB018
:10A82000AF8C2A8419E93245268797B6FFFF9386B5
:10A83000260B2D468145EF100006B250228522548A
:10A8400092540259F24945618280397126DAAE8408
:10A850004C0022DC4AD84ED652D406DEAA89328970
:10A86000368AEF0030692A8421E9A685630D090044
:10A870009E202C007C84BE207C85930720307C8623
:10A88000930780025C874E85EFB02F832A840DE505
:10A890005946A6851305A100230421019760FB1FDB
:10A8A000E78040AB1245528797B6FFFF938666FE5E
:10A8B00025462C00EF00307EF25022856254D2549F
:10A8C0004259B259225A21618280797126D2AE84CE
:10A8D0006C0022D44AD04ECE06D6AA893289EF0027
:10A8E00070612A840DE1A6854E85EFB0AF812A8480
:10A8F00019E932454A8797B6FFFF93862600354609
:10A90000A685EF005079B250228522549254025904
:10A91000F249456182807547AA876365B70211478E
:10A9200001456378B702ED1593F5F50F6147636153
:10A93000B702973602009386662BB3C5D52098419F
:10A940003697028793F5F50713072005638AE5001C
:10A9500001458280C8478280884382808847828000
:10A96000C84382809307F00F630FF506011126CAD2
:10A97000AA841305000222CC4AC84EC652C456C24D
:10A9800006CE2E8AB28AB6893A899760FB1FE78085
:10A99000A08C2A844D450DC8930700FB1CA0A30082
:10A9A000540123114401230234011305840061463C
:10A9B00063050902CA859760FB1FE780A099A285FD
:10A9C0002685EF909F880145F2406244D244424977
:10A9D000B249224A924A0561828081459760FB1FF5
:10A9E000E780C09DE9BF09458280011122CC06CED7
:10A9F0002A844C86D0869780FB1FE780001705C10C
:10AA00005425214797A7FB1F938707A5639DE60061
:10AA1000E82378009306E0070146A285A137F240BB
:10AA2000624405618280C83378009306E0070146DE
:10AA3000A285EDB7930700643306F6026F905FBC02
:10AA400015C1411122C406C62A8408219307D00FDC
:10AA500063E6A700EF909FD8FD571CA0B2402244A8
:10AA6000410182808280797122D406D626D24AD0D2
:10AA70004ECE9E2509448DEBAE846C00AA893289A6
:10AA8000EF0050472A840DE1A6854E85EFA05FF3C5
:10AA90002A8419E932454A8797B6FFFF938606F262
:10AAA0004D468145EF00305FB250228522549254CA
:10AAB0000259F249456182801A219307000B631005
:10AAC000F7025C214947639AE70018398547639884
:10AAD000E7002A2185456F30902A6D47CDBF8280DF
:10AAE00001116C846C0022CC26CA4AC806CE2A8981
:10AAF000B6847085EF0010402A840DE12C004A8551
:10AB0000EFA07FD22A8419E93245268797B6FFFF46
:10AB1000938626CD15462C00EF00F057F240228593
:10AB20006244D244424905618280797193072030A2
:10AB30006C8470857C862C0093078002014606D6C3
:10AB40005C87EFF09FD0B25045618280C177797108
:10AB500085073EC4894726D27C86AE84930780024F
:10AB60004C0022D44AD006D62A895C87EF00903860
:10AB70002A840DE12C004A85EFA0FFE12A8419E91F
:10AB80001245268797B6FFFF938626DE45462C00A2
:10AB9000EF007050B2502285225492540259456100
:10ABA0008280B28605466FF05FCA797126D2AE8484
:10ABB0006C0022D44AD04ECE06D6AA893289EF0044
:10ABC00070332A840DE1A6854E85EFA07FBD2A84CF
:10ABD00019E932454A8797B6FFFF938626BB0D4693
:10ABE000A685EF00504BB250228522549254025950
:10ABF000F249456182807971930720206C847085C9
:10AC00007C862C0093078002014606D65C87EFF015
:10AC1000DFC3B25045618280011122CC26CA4AC8E6
:10AC200006CE2A84AE84328936C69780FB1FE78021
:10AC3000C0F315C95025A146324797A7FB1F93873C
:10AC4000A781631DD600E823CA862686A2856244B2
:10AC5000F240D244424905616FF0DFD0C833CA8662
:10AC60002686A285EDB7F2406244D24442490545AA
:10AC7000056182806FF0BFB86FF07FB86FF0FFC4DE
:10AC80006FF0BFC479714ECEAE896C0022D426D24B
:10AC90004AD006D62A89B284EF00D0252A840DE155
:10ACA000CE854A85EFA0DFC72A8419E93245268779
:10ACB00097B6FFFF938646C63D468145EF00B03DFF
:10ACC000B2502285225492540259F2494561828041
:10ACD000B28601466FF07FB7011122CC2E846C0042
:10ACE00026CA06CEAA84EF00F020DD476309F500EE
:10ACF000930710101EA4A2852685EFA07FCCF240FA
:10AD00006244D24405618280239405006FF0BFD570
:10AD1000E5BF1797FB1F03476731854763F8E702D5
:10AD2000011122CC2E846C0026CA06CEAA84EF0024
:10AD3000701C01E9930700101EA4A2852685EFA0D0
:10AD40003FC8F2406244D244056182805945828006
:10AD50009797FB1F23ACA72882809797FB1F23A5FB
:10AD6000A7288280011122CC26CA06CE2A84AE846E
:10AD70009780FB1FE78060DFA6852285EFA04FF656
:10AD800005E9228564869780FB1FE78000DE0DC100
:10AD9000542521479797FB1F9387076C639FE60015
:10ADA000E82378009306F0070146A285EFF09FBBE9
:10ADB000F2406244D24405618280C833DDB77971C4
:10ADC00022D44AD0AE8706D6BA8526D24ECE754753
:10ADD000328436896364F7042147636CF7001547B2
:10ADE0006388E7021947638DE708C167FD1785444B
:10ADF0001DA037061400DD1713060620B317F02830
:10AE00007D8E49EE19677D8F25EB93F71710F1DFE3
:10AE1000C167FD1789446316F40221A813F7F707E9
:10AE200093062005E313D7FC41677D17631EE604F4
:10AE30008D442EC6EFA08FEEB245330495403344C7
:10AE400004083385840033450508EF30D000AA8715
:10AE5000B3C9040821C963040900231089002254DE
:10AE6000B25092540259B3053041F2493E854561D2
:10AE70001753FB1F67002339C167FD17954461BF56
:10AE8000C167FD179D4441BF1307200D8D44E39A10
:10AE9000E7FA1304C6003344040865B7C167FD1719
:10AEA0008D4495BFB250225492540259F2494561E3
:10AEB0008280011122CC26CA06CED0212E8413070F
:10AEC000000281469945AA84DD3D2AC621C51E207F
:10AED0005020930554007C803E207C8189477C82F1
:10AEE000930780025C839750FB1FE780A0465C209D
:10AEF0008A8526857C84EFA0BF952A8411C53245BA
:10AF00009750FB1FE780A022F24022856244D24482
:10AF1000056182804D44CDBF397122DC26DA4AD8E2
:10AF200006DE89472A84AE8436896306F600C14767
:10AF300009456315F60432C6A9C04C082285EF0006
:10AF4000607B324605EDC1778507A6851305D101E3
:10AF50003ECC230EC1009750FB1FE780A03F2C087A
:10AF60002285813F01ED52454A8797B6FFFF9386C0
:10AF7000C68C1D462C08EF0010120145F250625499
:10AF8000D254425921618280397126DA4AD84ED68C
:10AF90003289AE893686BA84814613071002D945B4
:10AFA00022DC06DE2A8432C6EFF07FE12ACE1DCDF8
:10AFB0003246A685231A3101F084231B21019750C4
:10AFC000FB1FE780203922854C08EFA01FA92A84A7
:10AFD00011C572459750FB1FE7806015F25022851E
:10AFE0006254D2544259B259216182804D44FDB716
:10AFF000011122CC06CE26CADD472A84639FF508BC
:10B000005439B1441C49B38696023287B6979043AF
:10B0100014436306D6020A20230601006C00EFA049
:10B020007FA70824B165938505B8EF904FBAE5472F
:10B030003CA097B7FFFF9387A7A55CC091A85623B4
:10B04000D223E31AD6FC88470C479750FB1FE780B2
:10B05000E041AA870A2089E7230601006C00C1B7F6
:10B060005C385828850793F7F70F5CB863F4E7025C
:10B07000B38797021848BA979847D623B2238E23EE
:10B08000213751F90824B165938505B8EF902FB4A5
:10B09000D94431A87C285C86D1B70A21AE846C00E3
:10B0A00023060100EFA01F9F8547E39CF4F6F240C2
:10B0B00062442685D24405618280011122CC06CEED
:10B0C00026CADD472A840A216398F508EFA00FC538
:10B0D000522C3E284E286D162A9633460608330712
:10B0E000F64052ACAA86334707080A206372B706B7
:10B0F0001388C6FFB388E54063D40803AE97918FE9
:10B10000B3C607081C4C0E283E97EFF0FFE709ED89
:10B110000824B165938505B8EF906FABD944B1A011
:10B12000ED16B3C60608F9BF0A20230601006C001D
:10B13000EFA05F960824B165938505B8EF902FA91D
:10B14000E5473CA097B7FFFF938787945CC0F9B7AA
:10B1500085475C866C00E9BFAE846C002306010065
:10B16000EFA05F938547E397F4FCF24062442685A5
:10B17000D24405618280397126DAAE842C0022DC4B
:10B180004AD84ED606DE2A89B289AD232A8431E513
:10B190004A85EFA0AFB8D6206D1563C4A600B346AC
:10B1A00005089844B2208E204A85EFF0FFDD2A84FE
:10B1B0000DE53146A6850808230601009750FB1FC0
:10B1C000E7804019BE2022454E8797B6FFFF938641
:10B1D000C6855D466C00FC867D2DF250228562544A
:10B1E000D2544259B2592161828071B769B77971DD
:10B1F00022D406D626D24AD04ECE52CC56CA5AC8EF
:10B200000944C1CD3289094449CAAE84BA8A2A8A1E
:10B21000368BEFA0AFB0138744008147711516231A
:10B2200063DEA608850793F7F70F3107E319F9FEE8
:10B230008A855285C1212A842DE131453305A90231
:10B240009165938515704D449750FB1FE78000E191
:10B25000AA8921C531463306C902A6859750FB1F2E
:10B26000E780400F9844D620B2208E205285EFF020
:10B27000BFD12A8415ED02458547568797A6FFFF63
:10B280009386A67A5D464C005C824EC4230621015B
:10B29000A306010023076101FD2BB2502285225431
:10B2A00092540259F249624AD24A424B4561828025
:10B2B0004E859750FB1FE78080E7C5B76D44F1BF0F
:10B2C00079714ECEAE89C16526D20147AA848946DE
:10B2D0001796FB1F130686C2FD15054522D406D618
:10B2E0004AD0EF101001054429C92A8913073002FA
:10B2F00081461146F5452685EFF07FAC2AC65544B8
:10B300000DCD0357A900CE86014678841147788574
:10B31000054718A1B2472C002685A38007003247B5
:10B32000FD573CA332473CB3EF10E0712A8411C5AE
:10B3300032459750FB1FE78080DFB25022852254B0
:10B3400092540259F24945618280411106C6EFF0DC
:10B350008FDC19C5B24041011753FB1F670023DD85
:10B36000B24041018280011106CE2AC6EFA04F8172
:10B37000324591459797FB1F23AA07C69797FB1F56
:10B3800023A407C69797FB1FA388A70CEF30C027FD
:10B39000F24005616F20700F79714AD006D622D431
:10B3A00026D201499397556063D807041795FB1F70
:10B3B0000345950A2E899750FB1FE780E0EF2A840A
:10B3C0005DC518219307000A6310F70A85474C08EA
:10B3D000DC85EFA06F88AA841DC59C8599C70844A9
:10B3E00009C59750FB1FE78080D42A208545EF30A0
:10B3F0000019CD47639AF406B250225492544A85FC
:10B400000259456182808347610191CF714763632F
:10B41000F7064D476378F7069386C7FE1307301487
:10B420003357D74825C31797FB1F0327E7BB01C72F
:10B43000034751012DCB9C8599C7084409C59750F6
:10B44000FB1FE780C0CE5247B7070001938707F084
:10B450007D8FB7071200938707106307F700034734
:10B460006101ED476302F70A2285EF80FFD81319C7
:10B47000F96859B7138717FE1377F70F9306000281
:10B48000E3F3E6FA858B9DCB9797FB1F83A707B65F
:10B49000A5C72A201306B1004C0882979C85AA8470
:10B4A000ADEBD5D099B75C8699472308F1002A20E7
:10B4B0006C0023170100EFA0CF9CB5BF9797FB1F2F
:10B4C00083A787B285CB2A201306B1004C08829748
:10B4D000AA8435D183475101E39107F023089100F5
:10B4E000834761012A206C005C8623170100EFA0CE
:10B4F0004F99E5B59944F9BF9C8599C7084409C59A
:10B500009750FB1FE780A0C22A208545EF30200717
:10B51000A1BF084459D59750FB1FE78040C151B7E0
:10B520005D71A2C4A6C286C6CAC04EDE52DC56DA1F
:10B530005AD85ED6A5472A84B2846392F50E834713
:10B5400045021A22322285072302F5029307F7FFEC
:10B55000B307F602D440B3C70708B697542503CB08
:10B56000070003C917008547638BF604931789000A
:10B57000B3E7670141677D17638AE70A1A2863F713
:10B58000E70A50248507B3C7070885467EA40A202A
:10B590009305E400631BD6007C84930720307C86EF
:10B5A0009307800278855C872C00EFA00FB10824F8
:10B5B000B165938505B8EF809FE159458DA83307A4
:10B5C000C702239004008149014A930B3501B34A15
:10B5D0000708E3FD59F9B620DC402C2813865900F2
:10B5E000ED163E965E85B3C60608EF907FDE1DC160
:10B5F000630B3A01C840B220B3053501529597500C
:10B60000FB1FE78020D5BE203E9A9E20334A0A08C1
:10B6100085079EA0BE20BE99B3C909085DBF582208
:10B62000A9476311F7028347450289CF0145B64018
:10B63000264496440649F259625AD25A425BB25B9A
:10B64000616182803428130934014A86894517953F
:10B65000FB1F1305E58DEF90BFD739ED34284A86DF
:10B6600089451795FB1F1305658CEF907FD629E55B
:10B6700034284A8689451795FB1F1305E58AEF9004
:10B680003FD51DE934284A8689451795FB1F1305C8
:10B690006589EF90FFD30DE1DC2009476380E70265
:10B6A000ED1793F7F70F29476368F70013079048E2
:10B6B000B357F700858B99E3054595BF834744024F
:10B6C00085072302F402BE2075B5411122C406C6C7
:10B6D0002E849770FB1FE780003F09C93C25138724
:10B6E00017006315E40093F707F83CA5B240224425
:10B6F00041018280411122C406C62E849770FB1F2F
:10B70000E780603C1DC111C008C01C251307E00F75
:10B710005D456388E7001307F00F59456393E70021
:10B720000145B2402244410182800945DDBF4111FB
:10B7300022C42A84210526C206C64AC0EFF04FB0B3
:10B740002420A51493F4D40F81E858248547631D61
:10B75000F7041C483149A1E3FD57230104001CB440
:10B76000230204021305C4002244B2409244024959
:10B770006146814541011753FB1F670023C4B3870E
:10B7800024033E95084509C59750FB1FE780209A82
:10B79000850493F4F40F5C280848E3E2F4FE975024
:10B7A000FB1FE780C0984DBF084C75F975B7411174
:10B7B00022C4416406C626C29307E4FF6301F50272
:10B7C000AA849DE19770FB1FE780E02F09E913052C
:10B7D000F4FF9770FB1FE780002F11C106A1B24054
:10B7E000224492444101828085476392F504977018
:10B7F000FB1FE780402D2A847DD1FD571EA11C240C
:10B800001307F00F6382E7021307E00F6389E70075
:10B810003420083401475146A685EFF0AF942285C5
:10B82000EFF0FFF0FD571CA4230504004DBF89472E
:10B83000E397F5FA8545EF40C04655F126859770A8
:10B84000FB1FE78040282A845DF951BF21C5011103
:10B8500022CC06CE18259307F00F2A846308F7023E
:10B8600034210E21083501475D46EFF0AF8F3820B7
:10B87000E1476318F7000A206C0023060100EFA0DF
:10B880006FA1F9571CA42285EFF07FEAF2406244D1
:10B890000561828082809307F00F6306F70601112D
:10B8A00022CC26CA2A844AC84EC652C4B689328AD5
:10B8B0003A8993068500AE847946AA85170500006B
:10B8C000130505F906CEEFF0EF96A304240123013A
:10B8D00044012322340185C01305C4006244F240B0
:10B8E0004249B249224AA685D244614605611753AE
:10B8F000FB1F670023A6F2406244D2444249B2498A
:10B90000224A0561828082809787FB1F2384A76E6D
:10B910008280411122C406C695472A846391F506A8
:10B9200083474502854685072302F5021E225842B9
:10B930003022FD17B3C70708631ED602B3C7E7203E
:10B9400098239C330145A207D98F7A2463F0E7023C
:10B950000A2085075EA49305C400EF90DFEC08245D
:10B96000B165938505B8EF809FA65945B240224442
:10B9700041018280C946B387D702BA97D1B758220E
:10B98000A9470545E314F7FE0345440213351500A6
:10B99000F1BF411122C406C69D472A846396F5046F
:10B9A0008347450285072302F5021E225842FD17F0
:10B9B000B3C7E72098239C33A207D98F7A25014586
:10B9C00063F0E7020A2085075EA49305C400EFF048
:10B9D0004FCE0824B165938505B8EF805F9F594528
:10B9E000B2402244410182805822A9470545E3190B
:10B9F000F7FE0345440213351500DDB7411122C49B
:10BA000026C206C6B5472A84B2846394F5048347E8
:10BA1000450285072302F5020A21EF903FB09E20E0
:10BA20001307F5FF014563C1E7027A240A20930555
:10BA3000C400BA977EA4EF90FFEC0824B16593850B
:10BA400005B8EF80DF985945B24022449244410145
:10BA5000828058229D470545E318F7FE03454402BE
:10BA600013351500D5B7411122C406C6C5472A842F
:10BA70006390F5061E223A22FD17B387E7020347BB
:10BA8000450205072302E5025842B3C707083E975F
:10BA90003C333823A207D98F41677D176397E700AE
:10BAA0000145B240224441018280138717005AA504
:10BAB0007A25E3F7E7FE9305C5000A21EF90BFED75
:10BAC0000824B165938505B8EF807F905945D1BFB3
:10BAD0005822A9470545E316F7FC034544021335F0
:10BAE0001500C1B7011126CA4AC84EC656C206CEB5
:10BAF00022CC52C4BC211547AA8A2E89B289B684A9
:10BB0000639EE7023686CE854A85EFF09FE02A8461
:10BB1000631E05108547034599006393F910D820EB
:10BB2000A9476319F70C054A834629000345990084
:10BB300001476946D685EFE0FFE2F9A83547638CF7
:10BB4000E7086361F7041D47638BE7062547638EAB
:10BB5000E706A547638FF90A054403459900268740
:10BB6000CE860146D685EFE0FFDF054A19E5CE8592
:10BB70002685EFE05FDA133A15005DD4D9476306F6
:10BB8000F40259A84547638EE7045D47E393E7FC59
:10BB9000D82585473686CE854A85631AF704EFF0A7
:10BBA0002FC58547054AE306F5FAF2406244D244C0
:10BBB0004249B249924A5285224A056182803686BC
:10BBC000CE854A85EFF0FFDC99B73686CE854A856B
:10BBD000EFF01F952DBF3686CE854A85EFF01FE228
:10BBE0003DB73686CE854A85EFF0FFE70DB7EFF01B
:10BBF000CFCC45BF268785460146D685EFE09FD648
:10BC0000E31305F285452685EFE0FFD0133A1500D2
:10BC100021BF9E20B1F3054A4A85EFF05FB171B7AD
:10BC2000A547E39CF9F29E208DFBF5BDA547E39661
:10BC3000F9F29E20E39307F2054A89B79E21639F9C
:10BC4000071C397126DA4ED652D406DE22DC4AD8D9
:10BC5000A021ED47AA89AE84328A6315F4021787C2
:10BC6000FB1F034727399307F00F0144631FF704B5
:10BC70009947F2506254D2544259B259225A3E85E1
:10BC800021618280F5476311F4089786FB1F83C604
:10BC900066361307F00F9947E38DE6FC9770FB1F9C
:10BCA000E78060E22A8415C1302505C293174660FB
:10BCB00063D40700814775BFF5454E85EFE0FFD29D
:10BCC0003C2493E707F83CA4F5B7D62090448C3089
:10BCD00088203800EF901FDDAA8741FDB42038008E
:10BCE0000146CE851785FB1F0345C530EFE09FC792
:10BCF000AA8741F1B24799C323000A00BC207547C7
:10BD0000E39AE7FA69F07DB79770FB1FE780A0DB45
:10BD10002A894DD185476317F404CE20884430002A
:10BD2000EF90BF81AA8731F58347290015476382C9
:10BD3000E702E51793F7F70FC14663E1F6043317FF
:10BD4000F0281377574411E7639AD7028327090134
:10BD500095C7B0203400CA854E85EFF0BFD82300C8
:10BD6000AA0089BF38219147E31587F05841E302C3
:10BD700007F0CE208844300002976DB70345990044
:10BD80009787FB1F83C7576D6381A702B4203800D4
:10BD90000146CE85EFE01FBD2A8409E9AC202800CA
:10BDA000EFE07FB719C123000A00014403472900CF
:10BDB0008D476318F7043C840357C90063F4E70018
:10BDC0002316F9008355C9004E85EFE0BFF91787A8
:10BDD000FB1F0357E737ED4763F5E7028357C900B9
:10BDE000DD4663F0F6029386370063D1E602116602
:10BDF0009385470013060629B3C505084E85EF80D5
:10BE0000A01F4A85EFF0BF92A287A5B511669305E2
:10BE1000B00F13060629B355B70ACDB799473E852B
:10BE20008280011106CE26CA4AC822CC4EC652C410
:10BE30009784FB1F93844462882493078002916552
:10BE40003305F502938565701789FB1F1309491A9D
:10BE5000334505089740FB1FE78040209024930757
:10BE6000800281453306F6022320A9009740FB1F7C
:10BE7000E780C054832709004D459DCB0144130A38
:10BE80008002FD599C24636DF40217050000130520
:10BE900025DBEFE0FFEB1705000013054583EF906E
:10BEA0006FDA170500001305C590EF30B056014555
:10BEB000F2406244D2444249B249224A056182803A
:10BEC000B307440303250900614681450504137443
:10BED000F40F3E952310350123010500231435018D
:10BEE000230505002302050231059740FB1FE7806B
:10BEF000E04C49BF014582801787FB1F0347575617
:10BF0000814763E4E70001458280922193864500E2
:10BF10006314A6002E8582808507B685DDB71DC512
:10BF2000411122C406C638219307D00F2A8463EB3F
:10BF3000E7000E2128310147F9465D46EFE09FA258
:10BF4000F9573EA0B2402244410182808280178787
:10BF5000FB1F0347F7508147FD5663E3E7008280EC
:10BF600016A12301050085071105C5BF0145828083
:10BF70009785FB1F938515F79307000285469CA1C3
:10BF8000FD571787FB1F230FF7F41787FB1FA30A23
:10BF9000F7F41787FB1F2306F7F49787FB1F2391FE
:10BFA000D7F49787FB1F239507069787FB1F23AFBF
:10BFB00007049787FB1F23A907049787FB1F23A369
:10BFC00007041786FB1F130626F19787FB1F93872D
:10BFD00067F65CC29787FB1FA38E07009787FB1F3E
:10BFE0009387C7E9094718A298A398AB2380E70273
:10BFF0002388E7021787FB1F130787F294A7D0C790
:10C0000094AFD8DB1785FB1F130585F20D47178604
:10C01000FB1F130626F19786FB1F938626EE238CC3
:10C02000E702C8C323950700D0CB239D0700CCCFE0
:10C03000D4D3238407022395070223A60702239D56
:10C0400007021787FB1F032727FBD8DF9787FB1FF4
:10C05000938707E2170700001307870B23A0070049
:10C06000D8C323A407008280411106C6EFF0DFE8A1
:10C0700009C52821B240410182800145E5BF411137
:10C0800022C426C24AC006C6AA842E893284EFF092
:10C09000BFE6AA8711E94165CA857D15EFF0DFE5A6
:10C0A000AA87454581C786A3A0A30145B240224483
:10C0B000924402494101828021E309483547639E49
:10C0C0000603011106CE22CC182210322206598E08
:10C0D00032C6B377F64085E7CC452A842EC4EFF00C
:10C0E000BFF832460147630EC50022856244A2456F
:10C0F000F24005616FF0BFF82D473A858280130743
:10C100000008F24062443A850561828083C80500D8
:10C11000094863910803DC4103C807009C33A20768
:10C12000B3E707010D681308289063950701894755
:10C130006FF09FF80545828001114EC606CE22CCD5
:10C1400026CA4AC89789FB1F9389B9D903C7090032
:10C150009307F00F630FF7022A892945AE843284D2
:10C160009740FB1FE780400FAA8505C59307100B7A
:10C170001EA12302050002A562442311250166A128
:10C18000F24003C50900D2444249B24905616F80BB
:10C19000CF8BF2406244D2444249B2490561828069
:10C1A000411126C2AE849785FB1F83A5E5E422C416
:10C1B00006C62A84EFF05FEB098909C9228522446B
:10C1C000B240A685924441016FF08F8FB240224465
:10C1D0009244054541018280411122C426C24AC0D1
:10C1E00006C6AA84130445001309850B1E209DC3AF
:10C1F000084409C59740FB1FE78060F3228531465C
:10C2000081459740FB1FE780601B3104231A04FE21
:10C21000E31E24FDB2402244FD579EA002499244F1
:10C22000410182809786FB1F83C696239787FB1F59
:10C2300083A707DD01476394E600014582808E23D2
:10C240001386870B6394A5003E85828005071377CC
:10C25000F70FB287CDB7AA871785FB1F0325C5DA6D
:10C2600001C95A216314F700084582800841CDBFF7
:10C270008280411106C6EFF01FFE09C50845B24095
:10C28000410182800145E5BF797122D413844500C4
:10C2900026D24AD052CC5AC82E8A06D64ECE56CA7C
:10C2A0005EC622892287014B814481468147BD4574
:10C2B000122345CAB5EE46233E23B286A697B3C7DE
:10C2C0000708050B3107E315BBFEADC491659385E7
:10C2D000457026859740FB1FE78040D8AA8B39C957
:10C2E0000C44D1C9814A8149522033853B01974092
:10C2F000FB1FE78020065E200844BE99B3C90908E9
:10C300009740FB1FE780A0E263980A003109854A45
:10C31000832589004A84E9F9314681452285850AC9
:10C320009740FB1FE780800963826A053109CDB71A
:10C33000630ED6000145B250225492540259F2497C
:10C34000624AD24A424BB24B456182803223E313A8
:10C35000F6FE5223B294B297B3C40408B3C70708D9
:10C360008DB78547E3E367F70545F1B723267A01E3
:10C3700023149A00D5BF1309C400854A814949BFD7
:10C38000AA871785FB1F0325E5C711E182801845A1
:10C390003A276314F700110582800841FDB7411167
:10C3A00006C6EFF0FFFD09C50A21B24041018280B7
:10C3B0000145E5BF411106C6EFF09FFC09C52821E4
:10C3C000B240410182804145E5BF41111786FB1F04
:10C3D000130646C322C40042AA8606C62E8501471C
:10C3E0001DCC1C44AE271C406396D5021DC71CC340
:10C3F00001C92146930544009740FB1FE78080F563
:10C4000022859740FB1FE78080D20145B24022443D
:10C410004101828022873E84E1B71CC2D1BF05451D
:10C42000F5B701119786FB1F938606BE26CAAA841C
:10C43000884222CC06CE2E8401470DCD52211C41CC
:10C440006315960215C71CC39740FB1FE78020CEDB
:10C450002C002685EFF07FF701E519C0B2471CC01C
:10C46000F2406244D244056182802A873E85F1B75A
:10C470009CC2D9BF0545EDB7411122C42A840905E4
:10C4800006C6EFE0EFDBFD573CB0B240224441016D
:10C490008280411122C4416406C626C29307E4FF8C
:10C4A0006301F502AA849DE19760FB1FE780C064E9
:10C4B00009E91305F4FF9760FB1FE780E06311C1F2
:10C4C00006A1B24022449244410182808547639292
:10C4D000F5049760FB1FE78020622A847DD1FD5719
:10C4E0001EA13C201307F00F6382E7021307E00F41
:10C4F0006389E70028300147F9465146A685EFE0F9
:10C500006FC62285EFF05FF7FD573CA023020400C1
:10C510004DBF8947E397F5FA8545EF30807855F1AF
:10C5200026859760FB1FE780205D2A845DF951BF57
:10C530005D71A2C4CAC086C6A6C24EDE52DC56DAFF
:10C540005AD82E84AC21F9472A896392F504976062
:10C55000FB1FE780605A2A8405C138219307D00F5A
:10C5600063ECE70028310147F9460146CA85EFE050
:10C570006FBF2285EFF05FF00145B6402644964438
:10C580000649F259625AD25A425B61618280832A1B
:10C590000400B7070001938707F037071200B3F7CD
:10C5A000FA0013070710B28981446388E7022EC698
:10C5B0009760FB1FE7804054B245AA8419CD5021F3
:10C5C00009CE93174660E3C907FA4A85EFE0EFC149
:10C5D000DC2093E707F8DCA045B7178AFB1F130A96
:10C5E0006A9003470A009307F00F1945E307F7F82D
:10C5F000E147E3E4B7F893D71500FD1717170200DA
:10C600001307C76AB3E7E72003A80700E30708F6A4
:10C6100003AB4700E3030BF6B3CA0A0863850A00BD
:10C62000C947E39CF5F4562010440C300820380824
:10C63000029821F52C084A85029B1DCD183015FF64
:10C640003820230AA100B9472308E1006314F70248
:10C65000E24798239C33A207D98F0C084A85FC81B6
:10C66000EF902F8211D914080546D9454A85EFE08D
:10C67000AFDA21B7BC84D5B734209147E38EF6EE0C
:10C6800003450A0038080146CA85EFE0AFADE3165E
:10C6900005EE2C202808EFE00FA819C1238009001F
:10C6A0001840B7070001938707F07D8FB707120086
:10C6B00093870710E302F7ECE38004EC3C2021BFF2
:10C6C000411122C406C62E849760FB1FE780C0423A
:10C6D00009C95C21138717006315E40093F707F875
:10C6E0005CA1B240224441018280397152D42E8A29
:10C6F0004ED69305E100AA89528522DC4AD856D24B
:10C700005AD05ECE06DE26DA3289368BBA8BBE8AE6
:10C710009760FB1FE780C040054425C1AA84288795
:10C720003944EFF05FB331C90328450063070804BB
:10C73000D6875E87DA864A86A6854E8502982A8441
:10C740000DED9307E00F638AFA029820894763167C
:10C75000F702DC4098239C33A207D98F0D6713079B
:10C760002790639CE7008347190003460900D285A0
:10C77000A2075D8E4E85EFF03F9CF25022856254F9
:10C78000D2544259B259225A925A025BF24B216159
:10C790008280797122D422214ECEAA89228556CA5E
:10C7A00006D626D24AD052CC5AC85EC662C4AE8AD9
:10C7B000EFF05FA705E52285EF902FF5594411E1D1
:10C7C0000144B2502285225492540259F249624ADD
:10C7D000D24A424BB24B224C4561828003C789004A
:10C7E00085476307F700EFF03F9F03D52900E9B7BE
:10C7F000AA85AA8413858900EFF01FA92A8415CD84
:10C80000FA209624D044CE2003D52900E147EFF04A
:10C81000DFEDD9472A846318F50023A60400268596
:10C82000EFF09F9B71BF19E1268575BFDE2026853D
:10C830002390FA00EFF05F9A69B713894400014A28
:10C84000B94B594C3D4B8355090085CDE1476307F2
:10C850007A010357C900D94711E3E147035729007B
:10C86000835649000326890003D52900EFF0FFE72E
:10C870002A846310850323240900050A3109E3147F
:10C880006AFD2685EFF05F952DD0D947E31BF4F2C2
:10C8900005BF65D5835709002390FA00F9BF011140
:10C8A00070879307E00F1306E1000147894606CE23
:10C8B000EFF0BFE3F2400561828079714AD00359FD
:10C8C000850022D426D22A84AE844A85930521018C
:10C8D00006D69760FB1FE780A02479C51C252AC6D1
:10C8E00093F707029DC7A881EFF0BF98B245AA87CA
:10C8F00011E9239024013945B2502254925402592F
:10C90000456182802A204946829701C51E249EA047
:10C91000E5B7035924004A85EFF0DF9001ED41654A
:10C920007D15EFF03F9009E51E2425459EA0E9B74F
:10C9300023102501130745008147BD46122339EE18
:10C940003147B387E7029305840031462EC691072D
:10C950003E959740FB1FE780E09FB245314648086F
:10C960009740FB1FE780009F52242A2041478146C1
:10C97000DD45EFE0CFC42ACE09E51E2445459EA043
:10C98000A5BF0C4852249740FB1FE780A09C2A209B
:10C990004C08EF904FD32DD15945B9BF85073107CA
:10C9A000E39ED7F825459DB705458DB7797122D40B
:10C9B0002A840A254AD02E899305E1004ECE06D658
:10C9C00026D2B2899760FB1FE78080152DC91C25F0
:10C9D000AA8493F707028DEF18389307200511E317
:10C9E0005C20362450440E242A200147EFF0FFCF6C
:10C9F00021E11C38B9E32A20EF902FC9AA875945B5
:10CA00008DCFB250225492540259F249456182802E
:10CA10002887EFF01F86AA870DC52A204946A685DC
:10CA200082975DD91E242310F9001C3899E7D1BFE5
:10CA3000D947E319F5FE238009000145D9B705451B
:10CA4000D5B73945C5B7797122D44AD04ECE52CC2C
:10CA500056CA06D626D2AA892E8AB28A3689976005
:10CA6000FB1FE780600909440DC53C211307E00F57
:10CA7000AA845D44638FE7001307F00F5944639A5B
:10CA8000E70063920A02D2854E85EF900FCC2A848C
:10CA900021C1B2502285225492540259F249624A6D
:10CAA000D24A4561828003550A009305E1002317AD
:10CAB00001009760FB1FE780A0062887EFF09F8F9B
:10CAC000AA8505464E85EF20107D2A844DDDD1B71D
:10CAD0009307F00FE30FF9FA938624007946A685B1
:10CAE00017F5FFFF1305E543EFD0DFF4A381240121
:10CAF0004DB7797126D24ECE52CC56CA5AC85EC6B0
:10CB000006D622D44AD062C466C2AA8A2E8BB28BC1
:10CB1000368ABA899774FB1F83A4C44EB9C0804477
:10CB200083DC44000149035CA40063149901844040
:10CB3000F5B73E2463F75701050941043349090855
:10CB4000EDB7E36BFBFE63090A000C204840D28678
:10CB50005E86EF80FF876DD1638409002390890191
:10CB6000A284B25022540259F249624AD24A424B3C
:10CB7000B24B224C924C26859254456182809A2178
:10CB8000B621854763E3E60429C3D4210111138646
:10CB9000550022CC1775FB1F130585392E84894556
:10CBA00006CE32C6EF80DF82C14719C95420324613
:10CBB0002E200A200147EFF0DFF3A94711C181477A
:10CBC000F24062443E85056182803E8582802E86E9
:10CBD0000A22AE21854763E1A50219CD54224111F5
:10CBE0000147150606C6EFF0DFF0A94711C18147DE
:10CBF000B2403E85410182803E8582802E860A2297
:10CC0000AE21854763E1A50219CD542241110147A8
:10CC1000150606C6EFF0FFEDA94711C18147B240E6
:10CC20003E85410182803E85828039714ED6BE218B
:10CC300083D9050006DE22DC26DA4AD852D456D241
:10CC40005AD05ECE62CC66CA63E437152A8A05459F
:10CC500063830912416BAE8A2314010002C60144AA
:10CC600001497D1B894B054CC94C83D52A000147DE
:10CC7000814601464E8523130100EFF09FE7AA8409
:10CC800071C509EC13072002930661005A86954589
:10CC90005285EFE0CF922A84630E050E38849C20E3
:10CCA00025C718856301870541476394E70ABE24B9
:10CCB0004146130524001CA0BE24A1831CB0CC4017
:10CCC0009730FB1FE780006949043C848507B3C7A0
:10CCD00007087C8463FC2707BE24638967078509EE
:10CCE000B3C9090859B763967707BE2409461305E7
:10CCF00024001CA0BE24A1831CB0CC409730FB1F95
:10CD0000E78040651104D1B722C603596100B824F9
:10CD100013052400638F77013359990323057101AB
:10CD200018A0BE244146A1831CB0CC401379F90F52
:10CD300041BF2305810118A0BE241359290013798E
:10CD4000F90FA1831CB0CC4009464DBF3C84294556
:10CD50009DC32C005285EF80DFE609CD34001546D7
:10CD6000D9455285EFD05FEB11C532459730FB1F97
:10CD7000E780E03B0145F2506254D2544259B25927
:10CD8000225A925A025BF24B624CD24C2161828051
:10CD90000545D5B74545C5B71777FB1F0347072995
:10CDA000854763F7E706011122CC26CA4AC806CE9A
:10CDB0002A84AE8432899760FB1FE780E0D311C5D7
:10CDC00038219307E00F6307F704631B09002285EE
:10CDD0006244F2404249A685D24405616F90AF9308
:10CDE0008A209305E100231701009760FB1FE7806D
:10CDF00020D32887EFF00FDCAA8505462285EF2097
:10CE0000904971D5F2406244D24442490561828022
:10CE1000594582805D45FDB7411122C406C626C230
:10CE200093F705022A84328585C3EFF0AFD8AA852F
:10CE300005462285EF20304695476305F500BD473E
:10CE40006315F502214515A093F78500B6849DC3AF
:10CE5000EFF04FD6AA8505462285EF20D04309C5BD
:10CE60009C3481C79C2491C30145B2402244924422
:10CE7000410182809397456063D70700EFF08FD31D
:10CE8000AA850146D1BF89890D45F9FDF9BF7971A0
:10CE9000AE8622D42A848A229305E10106D636C6BC
:10CEA0009760FB1FE780C0C711C90C25228522545B
:10CEB000B246B087B25045616FF01FF6B2502254AF
:10CEC000054545618280411122C406C693F70502DB
:10CED0002A8432858DC3EFF0EFCDAA8505462285E1
:10CEE000EF20703B1547AA876305E5003D47631DAA
:10CEF000E502A14715A893F7850099CBEFF08FCBFA
:10CF0000AA85054622852244B24041016F20B038EF
:10CF10001397456063570700EFF0CFC9AA85014614
:10CF2000D5B7898991E18D47B24022443E854101C0
:10CF300082807971AE8622D42A848A229305E10107
:10CF400036C606D69760FB1FE78080BDB24609C98A
:10CF50000C2522852254B087B25045616FF0BFF690
:10CF6000B25022540545456182803E257971416762
:10CF700022D426D24AD04ECE06D6231701007D17E2
:10CF8000AA84328436898149638DE7009420D04099
:10CF9000138517001307E10033450508EFF07FB54F
:10CFA000AA899420D04089451775FB1F130545F8C1
:10CFB000EF800FC215C5A2242285EFF04FBE09C530
:10CFC0007D142A9433440408630409002310890063
:10CFD000B2502254925402594E85F24945618280E2
:10CFE0009420D04089451775FB1F130525F4EF8069
:10CFF0002FBE71F19420D04089451775FB1F130592
:10D0000065F2EF80EFBC11C9E38809FA3C87E3952C
:10D0100087FA03D4A9007D1475B7A22475B73971B6
:10D0200022DC26DA4AD84ED652D456D25AD05ECE18
:10D0300006DEBE8B9C252A8AAE84C18BB28A3684DA
:10D040003A89C289468B9DEF942089476383F6060F
:10D050005685EFF04FA005CD8328050063890802AF
:10D0600022866254F250925A5A88CE87025BB25995
:10D070005E87CA86F24B4259A6855285D254225AFF
:10D08000216182883285EFF0CF9EAA8709ED39456C
:10D09000F2506254D2544259B259225A925A025B07
:10D0A000F24B216182802946A6855285829749DD0F
:10D0B000C5B7DC4003C3170098238D672203336391
:10D0C000E3001386479013175360E343E6F8138693
:10D0D000F78F634BE60293862780630FD70863C8F8
:10D0E000E604F977938707803E9385473343030827
:10D0F000E3E067F62D45E39D0BF8DC449023CC4339
:10D100002310C90022851DA2F5779387F76F3E9300
:10D110008D473343030863E06712171702001307B4
:10D1200027B33343E32083270300BA97828793878B
:10D130003780E31FF7F02D45E39C0BF48547231060
:10D14000F900DC4481459C231CA0AA240505334535
:10D1500005089760FB1FE780A09C835709004DE9F5
:10D1600091072310F90011468145130514009730EB
:10D17000FB1FE780A02441A82D45E39B0BF0DC4476
:10D180006C0083C917009823A209B3E9E90011478D
:10D190002310E9009C234E851CA0DC449C331CB06A
:10D1A0009760FB1FE780C097AA8425C13086C165C0
:10D1B0009306E100FD158329C500EFF01FDB09EDA3
:10D1C0009420D04089451775FB1F130525D6EF80A5
:10D1D0002FA019E1FD577C8703C709008947631019
:10D1E000F70283A549000946130544009730FB1F49
:10D1F000E78040168357090089072310F9003C8710
:10D200003CA0A1833CB0014561B523173101C5BFE6
:10D2100018218907BA972310F9003E251CB03E2536
:10D22000A1833CA010214C41130534009730FB1F13
:10D23000E7804012C9BF2D45E39C0BE42310D900C1
:10D24000DC449C231CA0DC449C331CB06DBFC84450
:10D250009730FB1FE780A019334705081D45E36998
:10D2600077E36380EB02B386790163C6E600330798
:10D270007741B3490708CC44231039014E86DE9527
:10D2800051B58149CDBF2D45E3940BE0CC44528587
:10D29000EFE09FDD89472310F90008A0218108B045
:10D2A0009DB72D45E3960BDE89472310F90049BF52
:10D2B0002D45E39F0BDCDC441D472310E900982338
:10D2C00018A0983318B0BA2338A0BA23218338B0F5
:10D2D000D82358A0FA2358B0FE23A1837CA025B7F9
:10D2E0005D71A6C2AA842A214EDE52DC56DA5AD8D3
:10D2F0005ED662D466D26AD06ECE86C6A2C4CAC0DA
:10D30000AE8AC16BEF808FA1130CF5FF2A8A814989
:10D31000977DFB1F938D4D0B977CFB1F938C0CCF40
:10D32000177BFB1F130BCBCEFD1B334D0C08DE24EC
:10D3300063F6F90083D70D0063CD8701AA209775A6
:10D34000FB1F93856508EF807FA92A841DCD594472
:10D350002DA89C449305E100B3A7F92003C9170049
:10D360009C2322093369F9004A859750FB1FE78007
:10D37000207BAA851DE923902A0103A54D0009C53C
:10D380009730FB1FE780A0DA0544B640228526448B
:10D3900096440649F259625AD25A425BB25B225C09
:10D3A000925C025DF24D6161828083C8440083A675
:10D3B0000C003087AA206A8881475A87EFF03FC661
:10D3C0002A8419C923902A0103A54D005DDD9730F9
:10D3D000FB1FE780C0D555BF83A74D0099EFAA205A
:10D3E000514781465E86BD45EFD07F9D23A2AD00AB
:10D3F00009E523902A01454449BF83D70D0003570F
:10D400000B003E97634747013307FA407D1723100F
:10D41000EB0003A54D0003560B0083A50C003E95C1
:10D4200085099730FB1FE780E0F283D70D00035793
:10D430000B00B3C90908BA972390FD00CDBD39711F
:10D4400026DAAA842A214ED65AD006DE22DC4AD811
:10D4500052D456D25ECE62CC66CA6AC82E8BEF809A
:10D46000EF8BAA89D424AE248A2478001386D400B2
:10D47000EFF02FE805C5938BB9FF2A84E519014920
:10D48000177CFB1F130C8CB8977CFB1F938C4CB83C
:10D4900033CA090863497901631B09109E24294591
:10D4A0002310FB009DA8035DC10083C844008326B0
:10D4B0000C00AA205288814766876A86A285EFF011
:10D4C0001FB619C9AE2422859306E1006A86EFF0E3
:10D4D000DFA92A8461F0C9B783D70C009228E3132F
:10D4E000F6FE83250C00C8489730FB1FE78000F844
:10D4F00071D99779FB1F938929ED83A7490095EF8F
:10D50000AA204166454781467D169D45EFD03F8B59
:10D510001DE19E2445452310FB00F2506254D25475
:10D520004259B259225A925A025BF24B624CD24C87
:10D53000424D2161828023A2A900AE24835AA40017
:10D5400022859306E1006A86EFF03FA22A84E383F6
:10D550000AF883A749001307190033470708CA9739
:10D560002380570183A7490093DA8A009306290094
:10D57000BA972380570113073900110983A749007F
:10D58000B3C60608334707083349090811C930876D
:10D59000B69790A383A749002182BA9790A3DDBDD7
:10D5A000B697FD5694A383A74900BA9794A3AA20DF
:10D5B0009775FB1F938545E1135929002390250199
:10D5C000EF808FEB39D9594589BF411122C406C676
:10D5D00093F705012A84328585C3EFE0BFDDAA8574
:10D5E00005462285EF20204B95476305F500BD4792
:10D5F000631DF502214515A893F7450099CBEFE08F
:10D600007FDBAA85054622852244B24041016F2076
:10D61000804893F7050491C7EFE0DFD9AA8501465A
:10D62000DDB713C5F5FF05890605B2402244410167
:10D630008280797122D426D252CC06D64AD04ECEE0
:10D6400056CA5AC82A8AAE840144DE206364F400B4
:10D65000014581A083AA04009319140013891900BD
:10D66000B327542103CB0700B3872A0188239305EE
:10D67000E1002205336565019750FB1FE780404AB2
:10D680001DE123806A019C4005453E99034709003E
:10D6900098B3B250225492540259F249624AD24A83
:10D6A000424B456182800C2530875285EFF0FFF1B7
:10D6B00001CD9C40BE9903C7090098A39C403E99A8
:10D6C0000347090098B3F1B7050433440408B5BF14
:10D6D0000111AE8722CC2A848A239305E10006CE6D
:10D6E0009750FB1FE780C04309C90C25228562447F
:10D6F0003087F24005616FF05FEDF240624405450E
:10D700000561828039715AD02A8B2A2126DA4AD8BB
:10D7100006DE22DC4ED652D456D25ECE62CC66CA2B
:10D72000AE84EF70BFDF2A898346CB008355AB0000
:10D7300003558B0078001306DB00EFF08FBB630509
:10D740000516C16A130AA9FFAA8B01449779FB1F2A
:10D750009389C98B977CFB1F938C0CC7FD1A6D199D
:10D76000334A0A08035CC10083C58B0003552B00B4
:10D770006286EFF09FE56318051483484B0083A68B
:10D78000090003552B00528881471777FB1F1307A9
:10D7900027886286DE85EFF09F886316051205CC28
:10D7A00083D72C001777FB1F0357878611076395D4
:10D7B000E700A29763C427079775FB1F9385C5C031
:10D7C000BE2103552B003354F40282A1EF80CFE435
:10D7D00015C1594505A003552B004947814656867A
:10D7E000C545EFD0CFDD23A2AC0015E183D7AB0058
:10D7F00045459EA0F2506254D2544259B259225A21
:10D80000925A025BF24B624CD24C21618280976744
:10D81000FB1F83D7E77F91072391FC0083A74C0070
:10D8200003D7AB006286A29798A383A74C00130787
:10D83000140033470708BA9703D7AB009306E100FB
:10D840005E85218398A38355AB00176CFB1F130CD7
:10D850002C7CEFF08FF103A74C003C8713062400CB
:10D860003346060832971CA303A74C0093063400E6
:10D87000A183B3C6060836971CA3AA8B03A54C0048
:10D8800011043344040803560C0083A509002295B3
:10D8900063910B029730FB1FE780C0AB83570C00EE
:10D8A000A29733C4070809F883578B0029459EA027
:10D8B00091B79730FB1FE780E0A983570C003E9497
:10D8C0003344040845B583D7AB009EA0E31604EEAD
:10D8D00083578B009EA039BF1D71A6CACAC8AA84EF
:10D8E000035985002A21A2CCCEC6D2C4D6C2DAC042
:10D8F0005EDE62DC6AD886CE66DA6ED6AE8AEF70FD
:10D90000FFC1130BD5FF01447115138CD400976B25
:10D91000FB1F938BAB6F176AFB1F130A6A6F177D90
:10D92000FB1F130D6DAAB3490508635D6411D42470
:10D93000AE241307E10162864A85EFF08F9BAA8C23
:10D94000630205100359A500B0870C25AA2032C632
:10D95000EFF0BFC7631D050E83C8440083A60B000C
:10D960003246AA204E8881475287E685EFF02FEB9A
:10D9700079ED15C483570A0003572D008907630208
:10D98000F7069775FB1F938525A4BE21AA20B357E0
:10D99000F4029EA1EF80CFB60DC1594539A8AA2047
:10D9A00041664D4781467D16A545EFD04FC12322E4
:10D9B000AD001DE123902A014545F6406644D6445A
:10D9C0004649B649264A964A064BF25B625CD25CEF
:10D9D000425DB25D2561828083570A008907231169
:10D9E000FD0083570A00A29763DE670583274D0079
:10D9F00003D7AC00930D2400A29798A383274D0072
:10DA000003D7AC000504334404082183A29798A3EC
:10DA100003254D0003560A0083A50B00B3CD0D0866
:10DA20006E959730FB1FE780E09283570A00BE9DFA
:10DA3000C167FD1733C40D08E309F9EE0509334941
:10DA40000908E5B5294515FC23902A01BDB76DDC11
:10DA50000DBF1E21411126C206C622C44AC0444140
:10DA600089EB8947B2402244924402493E854101F4
:10DA700082809420D0402A8489451765FB1F1305B6
:10DA8000254BEF70FF9411C93C202547E51793F70C
:10DA9000F70F637FF700E147F1B79420D040894545
:10DAA0001765FB1F13058548EF709F9271FD55BFE9
:10DAB0001769FB1F1309C942835609008547DDD248
:10DAC0001A203697C166E3CFE6F8916593852570F5
:10DAD00031459720FB1FE7806058AA84CD4759D174
:10DAE000314681459730FB1FE780408D1A208355D2
:10DAF000090001468147B386F500B3C6060863E90D
:10DB0000E70201C62E972310E90023A00400214656
:10DB1000A285138544009730FB1FE780A083176719
:10DB2000FB1F1307274E1C4381CF3E879C43EDBF4D
:10DB300050401395470085072A9636A6054665BFCF
:10DB400004C3814705B7011106CE22CC26CA4AC8B4
:10DB500009E90944F24022856244D2444249056100
:10DB600082802AC6AA84280036896C845085EFF00A
:10DB70005FEE2A8465F1E30F09FCBE24F9DB9165B1
:10DB80009385557031459720FB1FE780204DAA876C
:10DB900015C1BA249766FB1F93860647232005000C
:10DBA0005AA198422324250101C7BA861843EDBF24
:10DBB0009CC24DB74D4479BF9767FB1F938797432E
:10DBC00098230DE3054798A3058909CD9766FB1FA8
:10DBD0009386062A414691451765FB1F1305052AC2
:10DBE0006FF07FF6014582809767FB1FA38BA72EFE
:10DBF000828041677D176315E5002E856FE02FB5A4
:10DC0000411106C6EFE04FAF09C5FD571EA1230124
:10DC10000500B24041018280011126CA06CE22CC05
:10DC20004AC88547AA846392F5042685EFE08FDF12
:10DC300031E941699305F9FF1307E1008946176649
:10DC4000FB1F1306E62D0545EFE0BFEA2A847D1988
:10DC500005C44C442685EFF0DFF9308722858146E4
:10DC6000CA85EFF08FB02A84E5B789476396F5003F
:10DC70008545EF20000355D9F2406244D244424921
:10DC800005618280EFE04FD56DB7411122C406C611
:10DC900026C21764FB1F1304247C08349767FB1FFC
:10DCA00023A007369767FB1F23AA07349767FB1F3C
:10DCB00023A4073459C59307200C3305F502916559
:10DCC000938515709764FB1F93848433190533453E
:10DCD00005089720FB1FE780603810349307200C5D
:10DCE00081453306F60288C019069720FB1FE7809E
:10DCF000E06C9C4018348145938647007D5563EA6B
:10DD0000E5069306800BB306D70201460507FD55CD
:10DD1000B6979766FB1F23A3F62EBE868EA2ACB2E3
:10DD2000ACA22382060005069906E369E6FEF956D1
:10DD300096A399463307D702BA971767FB1F232D7F
:10DD4000F72A17E5FFFF1305E57EEFD00F8117F5E2
:10DD5000FFFF13052597EF708FEF17E5FFFF130502
:10DD60008573EF10306BB24022449244014541016B
:10DD70008280239EA6FE36861388460B231006005B
:10DD8000232406003106E31B06FF85059386860BD8
:10DD9000BDB7411106C622C42A84EFC06FA1EFE0CF
:10DDA0002F9D1765FB1F032525259767FB1F238ADA
:10DDB0008712EFE0CF999767FB1F238587122244D4
:10DDC000B24017050000130565E541016F1090642E
:10DDD0009397556063DB072E79711765FB1F034529
:10DDE000451022D44AD006D626D24ECE2E89972070
:10DDF000FB1FE780604C2A8441CD18219307000B5C
:10DE00006315F70885479764FB1F93842420DC84FF
:10DE10009C402315010081EFEF00C075916593854B
:10DE200035709720FB1FE780602388C031C96146A9
:10DE300081451765FB1F130525599720FB1FE780B8
:10DE4000E0578349440089476393F908252797647D
:10DE5000FB1F938464578AA02A20A685EF70DFD227
:10DE6000AA869E202A201A248DEE6363F7001EA442
:10DE70000E24EFC03FEF2285EFC01FC49C8491C7E2
:10DE80004C2013058400EFD04FCC2285EF60CFB635
:10DE9000B25022549254F2491315F968025945615F
:10DEA00082806363F7001EA41E24D9459766FB1F7A
:10DEB000938686510D469EA0EFC01FD68D4545DD49
:10DEC0001765FB1F13054550EFD02FC86DB793871B
:10DED000A9FF93F7F70F4947E36FF7F81707020019
:10DEE000130707D8B3C7E7209C43BA9782879305E7
:10DEF000A1002285EFF0AFD4AA8435DDD947639421
:10DF0000F40A85092A2093F9F90F9766FB1F938677
:10DF1000A64B4E86D945EFC03FD031DDCE854DB7FB
:10DF20009305A1002285EFF03F9BF9B78359840048
:10DF30006C004E859750FB1FE78080BEAA842DC1E0
:10DF40002A2041669306E10055477D16AD45EFC096
:10DF50001FE79769FB1F9389294723A2A900AA8677
:10DF600055CD834844000358E10030862A20A68519
:10DF700081474E87EFF0AF8AAA846312050E2A20EC
:10DF8000CE85EF709FDDE30805EE2A20D945CE86C9
:10DF90002D46EFC07FC8AD45E30F05EC4E852DB78C
:10DFA0002315310185441830D147E306F7EC5C2096
:10DFB0009769FB1F938949412A202380F9003C85FA
:10DFC000CE85238299002391F900EF708FEBE30453
:10DFD00005EA2A20CE860546D945EFC0FFC3E30CEB
:10DFE00005E8854565BF835984006C004E859750D0
:10DFF000FB1FE780E0B2AA8445D52A20416693063C
:10E00000E10059477D16B545EFC07FDB9769FB1FDF
:10E010009389893B23A2A900AA8609E51E24C54449
:10E020007C8551B7834844000358E1003E24308684
:10E030002A20A6854E87EFE09FFEAA840DE12A20C4
:10E04000CE85EF70FFD4E30805E22A20D945CE86BD
:10E050003546EFC07FBCB545E30F05E081B7D94732
:10E0600003A549006397F4009720FB1FE780200C6D
:10E0700019B59720FB1FE780800B1E247C8525B7F0
:10E080009305A1002285EFF0AFA5BDB59305A100D2
:10E090002285EFF02FE78DB5130691009305A100BF
:10E0A0002285EFE0BF9089BD9305A1002285EFE0B6
:10E0B000DF80AA84E31405E4A30401006DBB93058B
:10E0C000A1002285EFE0EFEC05BD01458280F1CE95
:10E0D000011156C2AE8A854526CA4EC652C406CE26
:10E0E00022CC4AC82A8AB284B689EF10903BD14725
:10E0F0001DC51767FB1F034777F39767FB1F83C790
:10E10000B7F2014999E03E89BA87131749001764AD
:10E11000FB1F0324A4F03A94636DF900D547F24045
:10E120006244D2444249B249224A924A3E8505613C
:10E13000828036201307040191C605091379F90F6F
:10E140003A84D9BFB1C89565938525C013050002EF
:10E150009720FB1FE78080F048C469D113060002B6
:10E160008145130909049720FB1FE7802025230020
:10E17000040023112401231344019C341767FB1F5F
:10E18000032707EA998C1CA45C4491849180C4AF56
:10E1900023A08900814761B72326040023000400DF
:10E1A0002313440123045401E5B785473E8582804B
:10E1B000AA869765FB1F83C575E71767FB1F0327B3
:10E1C000E7E581476394F5000145828032233A8573
:10E1D00019C2E30CD6FE850793F7F70F4107DDB7A9
:10E1E000AA861766FB1F034676E41767FB1F032703
:10E1F000E7E281476314F600014582802E233A85C9
:10E2000081C54C23E38BD5FE850793F7F70F4107B4
:10E21000D5B7AA869765FB1F83C525E11767FB1F46
:10E22000032707E081476394F500014582801223AC
:10E230003A8519C2E30CD6FE850793F7F70F41071D
:10E24000DDB7AA861768FB1F034818DE9767FB1F18
:10E2500083A7C7DC01476314E80001458280B2232D
:10E260003E8509CAF2236317D600D04701C6322281
:10E27000E306B6FE05071377F70FC107E9BF4111A3
:10E2800026C2444522C406C62A8495C0C84409C58E
:10E290009720FB1FE780A0E9C84809C59720FB1F0E
:10E2A000E780E0E826859720FB1FE78040E822858D
:10E2B000414681459720FB1FE7804010FD571CB465
:10E2C000B2402244924441018280011122CC2A842E
:10E2D0002A2106CE2EC6EF102069324622858145BE
:10E2E000EF00505822856244F24005616FF03FF91B
:10E2F00005C53E21411122C406C62A8491CBDD45C5
:10E30000EF00505922852244B24041016FF03FF79F
:10E31000B2402244410182808280411122C4B1472F
:10E320001304C5FFB307F40226C29764FB1F93844E
:10E33000240B06C6A697BA276315B702C84315C1B2
:10E340009307F00F6305F6001C21639CC70097201C
:10E35000FB1FE780C0DDB1473304F402A29423A27F
:10E360000400B2402244924441018280411122C4FF
:10E370002E8426C24946AA848145228506C6972056
:10E38000FB1FE780A0038DCCD82C9767FB1F83A7CA
:10E3900027C91207BA979A231AA0BA23FE233AA0D4
:10E3A0001767FB1F035707C85AA09A207AA0BA2004
:10E3B0001AA4DA203AA4FA205AA49A241EA87AA40D
:10E3C000B24022449244410182802A869765FB1F15
:10E3D00083C5D5C51768FB1F032888C49766FB1F34
:10E3E00083A6C6C3014701456393E50082809C2252
:10E3F00081CFDC4691CBDC2F9207C2976316F600E3
:10E400009307150013F5F70F05071377F70FC106EC
:10E41000E1BF130600643386C50293069500AA8502
:10E4200017050000130505ED6F608F9D411122C493
:10E4300006C62A840835EF606FBAFD571CB4B24097
:10E44000224441018280011122CC4AC84EC652C4E6
:10E4500056C25AC006CE26CA2A89AE890144176A16
:10E46000FB1F130A7ABC976AFB1F938A2ABB1D4BBA
:10E4700083470A006369F404639D09029769FB1FDF
:10E480009389D9BA176AFB1F130A4AB9930AF00F86
:10E4900083C709006364F4061144A144228513066E
:10E4A000F00FCA850504EFF05FE733440408E31773
:10E4B00094FEF2406244D2444249B249224A924A0E
:10E4C000024B0561828083A40A0093174400BE9426
:10E4D0009C208DC3FE20639F270163956901AA20BC
:10E4E000EF10804826854E868145EF00B03726859F
:10E4F000EFF0FFD805041374F40F9DBF83240A00C6
:10E5000093174400BE949C208DC39C34638F5701A5
:10E51000FE20639C27012685EFF05FF12685D1451B
:10E52000EF0050372685EFF09FD505041374F40FE4
:10E5300085B7C167F917630BF502411122C406C6FE
:10E5400085472A846399F50022852244B24081459B
:10E5500041016FF05FEF89476396F5008545EF1045
:10E5600040747DD1B24022444101828082809D4529
:10E570006FF07FED1765FB1F0355C5AA828001115F
:10E5800006CE68876C861767FB1F0347E7A9854798
:10E590006318F70070009305E1000545EF509026E1
:10E5A000F24005618280A947631DF6029C319821E3
:10E5B000A207D98F1EA1BC31B821A207D98F3EA1D5
:10E5C000DC31D821A207D98F5EA1FC31F821A20746
:10E5D000D98F7EA19C359825A207D98F1EA501450C
:10E5E0008280054582809147631EF6009C31982108
:10E5F000A207D98F1EA1BC31B821A207D98F3EA195
:10E6000001458280054582809387C5FF0D47B3C6CB
:10E610000708636ED70031473387E7029767FB1F10
:10E62000938707DCBA97A8A38EA30145828009458A
:10E630008280930740203355F50A71159767FB1FB9
:10E640002392A79E9767FB1F2382B79E9767FB1FA6
:10E65000A38DB79C8280956541111905938535C0BE
:10E6600006C6334505089720FB1FE780209F01C998
:10E67000B240E95541011723FB1F6700C3B8B24000
:10E68000410182809767FB1FA382079A9767FB1F50
:10E69000238E07989767FB1F238907989767FB1FAF
:10E6A000A38407989767FB1F23800798854741112C
:10E6B0001767FB1FA309F79606C622C426C22A8441
:10E6C0009767FB1F238107969767FB1F239C07947F
:10E6D0009767FB1F23A40794EF10E0311765FB1F1A
:10E6E000130505D01306000381459767FB1F2380A0
:10E6F00087949720FB1FE78060CC1764FB1F1304EF
:10E70000649108209764FB1F938414921DC995653A
:10E71000938545C012059720FB1FE780209417675B
:10E72000FB1F232FA78E11CD1C30102081459CA0EC
:10E730009767FB1F238BC78E12069720FB1FE7806E
:10E74000E0C79C201765FB1F034585D11764FB1F9D
:10E750001304D48D3E951375F50F956508A0938528
:10E7600055C012059720FB1FE780408F9764FB1F61
:10E770009384C48A88C035CD102081451206972025
:10E78000FB1FE780A0C398401420814725077D56D2
:10E79000639BF604EF106047B1473305F5029565BA
:10E7A000938565C0334505089720FB1FE780008BE4
:10E7B0009767FB1F23A2A7862A8401CDEF10E044B0
:10E7C00031463306C502814522859720FB1FE7802D
:10E7D000E0BE2244B2409244170500001305A5D5BF
:10E7E00041016F102043850710A393F7F70F4107EE
:10E7F00045B79767FB1FA38B07829767FB1FA3850E
:10E80000078249BF411126C206C622C44AC0AE844F
:10E810009397556063DB07081769FB1F130929816C
:10E82000034509009720FB1FE78000A92A8421C91E
:10E830001821930700096311F7041831CD476314B9
:10E84000F7069756FB1F9386667E28219C22176841
:10E85000FB1F0348D88F13066400814501476318E6
:10E86000E50291C19CA29C2281CB0345090085450C
:10E870009740FB1FE780A0182285EF50FF97139564
:10E88000F468B240224492440249410182800E223F
:10E8900005071377F70FAE9793F7F70F090685452E
:10E8A000B3D7070B6DBF0123C1BF13F5150071D995
:10E8B000EF00105319CD9757FB1F83C7277791CBD4
:10E8C00085451755FB1F034585769740FB1FE7805D
:10E8D000001313C5140075B70547637EC7029C314A
:10E8E0009421A207D58F1EA16399E700BC31B821FE
:10E8F000A207D98F3EA1014582800947E39DE7FE2B
:10E90000BC31B821A207D98F3EA1DC31D821A207A2
:10E91000D98F5EA1CDB7054582809147631EF60071
:10E920009C319821A207D98F1EA1BC31B821A20722
:10E93000D98F3EA101458280054582809147631EA3
:10E94000F6009C319821A207D98F1EA1BC31B821B5
:10E95000A207D98F3EA10145828005458280A1474B
:10E960006318F6029C319821A207D98F1EA1BC31F1
:10E97000B821A207D98F3EA1DC31D821A207D98FB7
:10E980005EA1FC31F821A207D98F7EA101458280CA
:10E990000545828089476319F6009C319821A207BA
:10E9A000D98F1EA101458280054582803E22797162
:10E9B0004ECE06D622D426D24AD01307F007AE890F
:10E9C0006371F70209473AC47C86300093F5F50F6E
:10E9D000EF007078B250225492540259F2494561C6
:10E9E00082805A22D9462A89328463F7E6007E2241
:10E9F00063F4F6006379F70023140100300093F507
:10EA0000F90F4A85F1B70A2202C4EFF09F80AA8469
:10EA100035C5EFF09F9B9C246369F5001146A24623
:10EA2000CE854A85EF00F06975B7340026869305D8
:10EA3000F00F4A85EFF0AFE975F1A2471A24DC47E1
:10EA40009AA33A20BAA35A20DAA37A20FAA3DA20AA
:10EA50009AA7DC4495C793F4F90F2286A6854A85C8
:10EA60008297C167FD172A86E31BF5FA224599476D
:10EA7000F9451CA144A1EFF0DF99A9BF094645B7AC
:10EA8000014671BFA947631DF6029C319821A20778
:10EA9000D98F1EA1BC31B821A207D98F3EA1DC318C
:10EAA000D821A207D98F5EA1FC31F821A207D98F06
:10EAB0007EA19C359825A207D98F1EA5014582808D
:10EAC000054582809C211CA19C311CB1BC31B82120
:10EAD000A207D98F3EA1828023220500D821894731
:10EAE0006304F70005458280F62101114EC606CE6B
:10EAF00022CC26CA4AC80D47AE896379D7049C4503
:10EB000084339023A033A204D18CB02322049387B2
:10EB10004400518C639CD7029307C4FF2A89B3C772
:10EB200007086361F70203A58900231199002310E8
:10EB30008900F1559710FB1FE780E06C2322A900A4
:10EB4000014531A02285EFF0AFE671FD0545F240A9
:10EB50006244D2444249B24905618280797122D42B
:10EB600026D22E8406D64AD01C201947AA84B28504
:10EB70006390E70630202800EFF03FDA0DE92884A3
:10EB8000EFF00FE30C302A890DC92E86171700000D
:10EB90001307E7D134009D452685EF00D0304A8524
:10EBA00009468145C1214A85EFF06FED0145B2501C
:10EBB0002254925402594561828089477C803C846A
:10EBC0000A867C813C857C822685EF00D058F9BF7F
:10EBD00049476395E70232202800EFF05FD861F9DA
:10EBE0001755FB1F1305C57F5E25E9D3183068252F
:10EBF0003C00C9460146A685DD2C4DBF5147639DAB
:10EC0000E70032202800EFF01F9A55F10C30300059
:10EC10002685EFF0BFD959BF5947639CE7043220DE
:10EC20002800EFF05F9C41F52C842685EFF06FE122
:10EC300015C9584534851E23B697B3C707081EA3C8
:10EC4000B5D75C47A5D79757FB1F83C7273EB9DFCA
:10EC500085451755FB1F0345853D9740FB1FE78002
:10EC600000DAA9B789473EC03C840C300A867C8212
:10EC7000A1BF0C30231001000A8681BF5D71A2C4C0
:10EC800056DA86C6A6C2CAC04EDE52DCAA8A8831CF
:10EC90002E8432C6EFF0CFD4B24501ED0144B64028
:10ECA0002285264496440649F259625AD25A616135
:10ECB0008280230205002311050083490400854753
:10ECC000AA846399F90030202808EFF0FFC02A8455
:10ECD00005491DA09D476391F90418218D47E31F45
:10ECE000F7FA302028080549EFF05FC52A8409E5C6
:10ECF000054681452685BD262685EFF02FF388241D
:10ED00003C080147CE862286D685D522E30909F83C
:10ED10002685EFF0CFD661B7CD47639BF900182168
:10ED20009147E31DF7F630202808EFF0BFC645B73E
:10ED3000D547E395F9F6034A05008947E310FAF64B
:10ED4000302028080549EFF0FFD32A8455F5835772
:10ED50000102A1EBB8841306F003DC44930607FC20
:10ED6000B3C60608636AD600B085D94663F6C60006
:10ED7000B486D94563EDD500BAA30145EF00D03E76
:10ED8000054903560102D2852685AD2CB5B7AC875F
:10ED9000BAA3D2A38EA3F6A385479CA0014A01493A
:10EDA000CDB7014AF9BF7971AA8522D426D2222192
:10EDB000AA84280806D64AD0EFF01FD2F24599E57A
:10EDC0003DE185452285EFF08FFB75A0BC8415479A
:10EDD0006395E706B8858D4763F7E7046800EFF0B1
:10EDE0007FCE0359E100DD4763FB27018C86B7071F
:10EDF00017008507100822853EC8EF00D035BC8576
:10EE00001109638527012285EFF06FF61C86724693
:10EE10006C00858B1106228591CFEFF03FE601C58E
:10EE20002285EFF0CFF4884449DD9710FB1FE7807F
:10EE3000003041BFEFF09FD2DDB711476389E70093
:10EE40001387A7FF85463347070863ECE60231477F
:10EE5000F117B387E7021757FB1F13076758BA97D5
:10EE60009A2371D3A8233008A2850D204DFDB884C4
:10EE70009147E318F7F4B250225492540259456175
:10EE800082802C082285212E59FDF5B701114AC830
:10EE90002A89314526CA4EC606CE22CCAE89B28416
:10EEA0009710FB1FE780403B29C19307000A2311FD
:10EEB00035011EA12A842146110595C0A68597100B
:10EEC000FB1FE7802049A2854A85EF500FB8014516
:10EED000F2406244D2444249B24905618280814590
:10EEE0009710FB1FE780804DF9BF0545D5B701118D
:10EEF0004AC82A891305000226CA4EC652C456C201
:10EF00005AC006CE22CCAE8A328BB6893A8ABE84EB
:10EF10009710FB1FE780403421C9930720FA1CA1FA
:10EF2000A30065012311550123024501A302350108
:10EF30002A84614621059DC0A6859710FB1FE780A6
:10EF40006041A2856244F240D244B249224A924AC8
:10EF5000024B4A85424905616F502FAF814597109A
:10EF6000FB1FE780A045F1BFF2406244D244424912
:10EF7000B249224A924A024B056182805C4579710E
:10EF800022D406D62A84AE86A5C7BA23F8851307ED
:10EF900020066396E504FA231756FB1F03568608DE
:10EFA0003357C70AB22B9E2B1377F70F918F93F726
:10EFB000F70F01E6890793F7F70FBA97FD17B3C765
:10EFC000E702FC863E206E200824FC8401473C08B2
:10EFD0000146EFF0DFF1B250225445618280D82F14
:10EFE0009757FB1F83A7C7031207BA97FE23D1BF0A
:10EFF0002EC61946814528089710FB1FE780003C64
:10F00000B246C9B7797122D406D626D22A8491CDC8
:10F0100008242E866E202254B25092548147014714
:10F020009306000645616FF09FECB28428005946B4
:10F030009710FB1FE7808038648499E43E204844A1
:10F040006C007C85EFF08FB26E2008243C000147F5
:10F05000930600060146EFF09FE9B2502254925405
:10F0600045618280797106D6814799E53E21708697
:10F070007C845C4589EF3C002E866E210825014783
:10F0800093060006EFF0BFE6B25045618280BE23D2
:10F090007C85D5B7411122C406C61C2111472A849C
:10F0A0006392E7022E866E21082581470147CD46EF
:10F0B000EFF0FFE349466E202244B240154541017E
:10F0C0006FF0AFA513F7B70F89466317D700014656
:10F0D000EFF05FF35146C5B70D476398E700224450
:10F0E000B240014641016FF0FFF7B24022444101B6
:10F0F00082809A21B14771173307F7029757FB1F98
:10F100009387072EBA97D84301EBD841AAA70145A8
:10F11000D8C3BA219AA7828059458280797126D2B4
:10F12000444522D44AD006D62A842E89B1C4C84484
:10F1300019C59710FB1FE78080FF23A604009E20BF
:10F140006E2008247C85BE200147930640067C86FD
:10F150009E244A867C879C483EC83E207C843C0096
:10F16000EFF0FFD8A38E240123A80400B25022544C
:10F17000925402594561828028003146814597109A
:10F18000FB1FE780A0233E206E2008247C840147DB
:10F190003C00930640064A86EFF07FD5C1BF7971E7
:10F1A00052CC2A8A8A2126D206D622D44AD04ECEE2
:10F1B00056CAAE84EFE0DFFF6302051240452A899C
:10F1C000630E04107E21639B47111E24638A07107F
:10F1D000542C975AFB1F938AAAE403A70A009206AD
:10F1E000FD1736977A23B3C707081EA46316F700E6
:10F1F00093053006EFF09FD85C48B5EBC8408349D3
:10F2000015001C21A209B3E9F900BE2013872900CB
:10F21000631AF702F9559710FB1FE780C0FEC8C0BC
:10F2200023913401034589002686D285EFF01FC65D
:10F230001DEDB250225492540259F249624AD24A08
:10F24000456182809565938515C04E859710FB1F9B
:10F25000E780C0E048C8C840231C3401F955971026
:10F26000FB1FE78040FABE20C8C0F917BEA048487F
:10F270002DCDB220362C1E2C3308D60063C90707CB
:10F28000582C83A70A0095451207BA97BE2363CA74
:10F290000705CC4036959710FB1FE780A00B3A2C52
:10F2A000BE20BA971A2CB3C707083EAC6398E70292
:10F2B0000357290003458900300078845848D285D7
:10F2C0007C853AC6EFF09FBC11C548489710FB1FDC
:10F2D000E780E0E5232A0400232C0400054591BFC4
:10F2E00099454A85EFE07FFED5BFA545DDBF914535
:10F2F000CDBFBE21F9C3011126CA06CE22CC1757B5
:10F30000FB1F035727D2AA846D456363F70A2E8437
:10F31000484091459710FB1FE780E0EE3E20AA860B
:10F320001CA13E20A1831CB11E203CA11E20A18354
:10F330003CB13220C167F917110633460608639FB6
:10F34000F4022AC4314532C69710FB1FE780C0F093
:10F35000AA854D45B1CD930700F93246A2469CA13E
:10F36000F957BEA18947DCA1F2A194C51755FB1F2F
:10F370000345E5CBEF407FED01451DA8814526857E
:10F38000EF40F05C11E91757FB1F130727CA1C2336
:10F39000E5D7FD171CA3CDB789476302F5029D474A
:10F3A0006301F502C9476300F502FD47E30DF5FC73
:10F3B000F2406244D244056182806D4582805145AD
:10F3C000C5BF1145F5B70945E5B7011122CC4AC8BB
:10F3D00031441309C5FF3304890226CA9754FB1F21
:10F3E0009384040006CE26945C40A9C31757FB1FE4
:10F3F0000347C7C30DC768843EC62A241E242C00B9
:10F400007C85EFF01FEF11C548409710FB1FE78088
:10F4100000D2B1473309F902CA9423A2040005457A
:10F42000F2406244D2444249056182800145CDBF29
:10F43000797126D244454ECE52CCFE20BA28975937
:10F44000FB1F83D929BE06D622D44AD056CAB3D9C7
:10F45000F90A2A8A9E282DCF998F4E8463D43701CA
:10F4600033C4070889452285EFF0EF9E2A89CD4AEB
:10F4700031C5BE202AC660857C84BE2899EB9E28B3
:10F48000130925001CA19E28A1831CB163743405B7
:10F490008228BE28CC4422864A85BE959710FB1F41
:10F4A000E78040EB03556A002C00EFF09FE4AA8A46
:10F4B00015C54A859710FB1FE78060C7B2502254DC
:10F4C00092540259F249624A5685D24A4561828075
:10F4D000890761B779143344040865BFBA289E20B0
:10F4E0003A949A28FD17B3C70708334404089EA02E
:10F4F000A2A86376E400F9F3FD57DCBCC1B78145EF
:10F500005285EFF0BFC15DBF797122D44ECE56CA8D
:10F510005AC85EC662C406D626D24AD052CC975983
:10F52000FB1F938949B003CA0900975AFB1F938AAE
:10F53000EAAE054B5284930BF00F175CFB1F130CC4
:10F54000BCAE83A40A0093174400BE9403C9040010
:10F55000631D6907DC44B5CBD84725CB9A2339CB4B
:10F560009757FB1F83C787AC99CF2685EFF05FECD9
:10F57000AA8505ED05049757FB1F83C7F7AA6351BA
:10F58000F40223808900B25022549254F249624A14
:10F59000D24A424BB24B224C4A8502594561828085
:10F5A0009757FB1F238107A8F9BF2685EFF01FB7E8
:10F5B0000149D1BFDC3F639A770193052006268578
:10F5C000EFF0DF9BDC44A38E070083470C000504AB
:10F5D0001374F40F6363F4000144E31444F7C9BFE8
:10F5E0004111154506C6EFF05FDE09C50545B2407D
:10F5F000410182801945EFF05FDD6DF91145EFF0B3
:10F60000DFDC6DF51D45EFF05FDC6DF11755FB1F7D
:10F61000034595A169DDB24041016FF0FFEE9E21E7
:10F620000D47F117B3C707086363F706DC414111C3
:10F6300022C406C626C22E84A9CF8545AA84952554
:10F6400039CD2685AD2BC167F917638FF40009ED1D
:10F650003E2099CB162019476395E6041757FB1FE8
:10F660000357479C63FFE7029757FB1F83C7079C1D
:10F67000A285268599C72244B240924441016FF089
:10F680005FC72244B240924441016FF09FA60945F2
:10F6900082800945B2402244924441018280514512
:10F6A000D5BF6D45C5BF797126D252CCAA842E8AAA
:10F6B0005D4589454AD04ECE56CA06D622D4B28977
:10F6C000B68A3A89EFE03FF925C52A8401456306E9
:10F6D0000900D685130544000299935785003CB074
:10F6E00093074500230044017C85954728A07C842E
:10F6F000A300340122C69757FB1F83C727932C0012
:10F70000268585C7EFF0FFBEAA8411C52285971014
:10F71000FB1FE780C0A1B25022540259F249624A4D
:10F72000D24A2685925445618280EFF09F9CE9BFC2
:10F73000CD44D5B7797126D24AD052CC56CA2E893B
:10F7400006D6BE8522D44ECE9947B284368ABA8A6E
:10F750006314F9062A220944EFE09FA52AC625C5AD
:10F760005C4583596500BE239EA0B24715472380A0
:10F770005701BAA31757FB1F1307F78A10239305E6
:10F78000160093F5F50F0CA3D0A399E1854614A3B9
:10F7900051476317E9001547BAA0DC479A249AA796
:10F7A0005287A686CA854E85EFF0FFEF2A84324540
:10F7B0000DC4EFE0DFAC01A842867400AA89EFE037
:10F7C0001F912A845DD1B25022852254925402594D
:10F7D000F249624AD24A45618280F945EFE07FC32F
:10F7E000DDB79E211CA19E21A1831CB1BE213CA19D
:10F7F000BE21A1833CB1114582809E211CA19E2186
:10F80000A1831CB1BE213CA1BE21A1833CB1DE215C
:10F810005CA1DE21A1835CB1FE217CA1FE21A1833C
:10F820007CB1214582809E211CA19E21A1831CB117
:10F83000094582809E211CA19E21A1831CB1BE216D
:10F840003CA1BE21A1833CB1DE215CA1DE21A183CC
:10F850005CB1FE217CA1FE21A1837CB19E251CA56B
:10F860009E25A1831CB5294582809A218546AA87B9
:10F8700018A19A21218318B19A216319D700BA21BE
:10F8800038A1BA21218338B1114582800945631D11
:10F89000A700BA211945B8A3BA212183B8B3DA2148
:10F8A000D8A3DA212183D8B382809E211CA19E2176
:10F8B000A1831CB1BE213CA1BE21A1833CB1114555
:10F8C0008280797126D24AD04ECEB2842A89AE89FE
:10F8D00029468145480022D406D636849710FB1F5E
:10F8E000E780C0AD64868DE43E207C829747FB1F95
:10F8F00083D747737C845C4481CFD42F1747FB1F89
:10F90000032707729E27920636973A237C857883D1
:10F910004A8517070000130727F2540013F6F90F62
:10F92000D545EFF05FD82A8911C195E085471CA025
:10F9300023020400014681452285EFF0AFECB2506E
:10F9400022549254F2494A850259456182802285A7
:10F95000EFE0FF92EDB7B28617070000130727F11B
:10F960002E8685456FF03FD4011168874165700090
:10F9700001489307F00F0D47970600009386A6E60F
:10F9800099457D1506CEEFF0FFDAF24005618280E1
:10F99000B28701482E86114797060000938626E617
:10F9A000C9456FF03FD9B286170700001307E7E794
:10F9B0002E86CD456FF03FCF011122CC26CA4AC812
:10F9C0004EC606CEAA842E891754FB1F130444A4E6
:10F9D0009759FB1F9389C9A61C4081C7CA852685F4
:10F9E00082971104E31A34FFF2406244D244424940
:10F9F000B24905618280411122C406C626C217475A
:10FA0000FB1F1307E7737C2B783B1754FB1F130472
:10FA1000A4A41CB4BA9793F7F70F1CA4A5CB1305A5
:10FA2000C0033385A702A56585059744FB1F938412
:10FA300024609700FB1FE780606210249307C003D7
:10FA400081453306F60288C09710FB1FE7800097B8
:10FA500014249C4001477D566341D7022244B240A2
:10FA600092441306000381451755FB1F1305459A61
:10FA700041011713FB1F67006394B2A323820700A1
:10FA800023A6070205079387C703F9B7B2402244AC
:10FA9000924441018280411122C426C24AC006C656
:10FAA0002A892E84B2849730FB1FE780000C09ED71
:10FAB000C167F91751456313F9000145B24022446B
:10FAC000924402494101828054555C2195C213F74A
:10FAD00027014146630BC700C18B3D45E5D3BC2ED2
:10FAE0000145E3FD87FC3145D1BF1545F5D4F9B794
:10FAF000C18B0145E1F71545D1B779714AD041690C
:10FB000022D426D24ECE52CC56CA5AC806D6AA8481
:10FB100001449759FB1F93892994174AFB1F130A25
:10FB20002A51930AC0037D19054B83C7890063647A
:10FB3000F400014525A83307540383270A00BA9728
:10FB4000BA236316270105041374F40FF9BFC833F1
:10FB5000300093856700EFB0511C1946A685280038
:10FB60009710FB1FE7808090E31F65FDB250225481
:10FB700092540259F249624AD24A424B456182800C
:10FB80004166AA869755FB1F83C5858D1747FB1FC6
:10FB90000327074A81477D166394F500014582805B
:10FBA000035827003A856306C80003480700E308A6
:10FBB000D8FE850793F7F70F1307C703F1BF41116D
:10FBC00006C69730FB1FE78040FA09C54A29B240B4
:10FBD000410182800145E5BF1747FB1F03274745C9
:10FBE0009756FB1F83C6C68711078147014563935C
:10FBF000F6008280102301C605051375F50F8507F1
:10FC000093F7F70F1307C703DDB71755FB1F03451E
:10FC1000258582801747FB1F1307877F81473A8618
:10FC2000B1460C4391E5B3C7C72088C30145828024
:10FC300085071107E397D7FE4D458280411106C61F
:10FC400022C49730FB1FE78040F20DCD2A842A2181
:10FC50008545EFF07FD6485409C59700FB1FE78024
:10FC6000004D22851306C00381459700FB1FE780E6
:10FC7000E074FD573EA0230204000145B240224437
:10FC8000410182800945DDBF411106C69730FB1F47
:10FC9000E780A0ED09C54825B240410182800145B9
:10FCA000E5BFC167F9176305F502411122C406C615
:10FCB0002E849730FB1FE78040EBAA87014589C758
:10FCC000DC237D8C33358000B240224441018280A8
:10FCD00005458280411122C406C62E849730FB1F41
:10FCE000E780A0E801CD5A29AA870545630487006B
:10FCF000C2AB0145B2402244410182800545DDBFCF
:10FD000039CD01114AC8416922CC26CA4EC652C417
:10FD100056C206CEAA8401449749FB1F9389C97332
:10FD2000174AFB1F130ACA30930AC0037D1983C701
:10FD30008900634BF400F2406244D2444249B24924
:10FD4000224A924A05618280B307540303250A00C0
:10FD50003E953E216383270182940504C9BF8280BA
:10FD60009747FB1F83A7C72CC1661746FB1F034697
:10FD7000266F890701450147FD1691456313E6008B
:10FD8000828003D807006309D80003C8A700631561
:10FD9000B80005051375F50F05071377F70F93875F
:10FDA000C703E9BF9746FB1F83A686281746FB1F9C
:10FDB0000346066B910601478147631FE600858372
:10FDC00093C7F7FF0545B3C707086361E50233151D
:10FDD000A0283345050882808C2299C1CE36CD8F6C
:10FDE00005071377F70F9386C603C1BF93F6170075
:10FDF000F9FE050585831375F50FC1BF797156CAE4
:10FE0000AA8A2E8526D24AD04ECE52CC5AC85EC679
:10FE100062C406D622D4AE84328B368CBA8B3E8A2C
:10FE2000C28946899730FB1FE78020D43DED4165AC
:10FE30007D159730FB1FE78040D32A84554531C894
:10FE40001946DE8513056400A30284019700FB1F99
:10FE5000E78040508357010326A0230264013EA897
:10FE60008357410323005401232604025EA823067E
:10FE700044012317340123182401EFF0BFF20AB81C
:10FE8000232A04022685232C04028145EFF0DFB2E9
:10FE90000145B250225492540259F249624AD24A60
:10FEA000424BB24B224C456182804545DDB79746B7
:10FEB000FB1F83C6E65A1747FB1F032767178147B7
:10FEC0006395F60041657D1582800E3B1306C703DE
:10FED0006394A5002A238280850793F7F70F328762
:10FEE000C5B741661748FB1F034888579746FB1F55
:10FEF00083A6061401477D16954811436314E80054
:10FF000001458280BE223685638EC702CC5A9DC9C8
:10FF1000BC31AC2189CD938597FD93F5F50FE37244
:10FF2000B3FE9387D7FA93F7D70F89EF8280938533
:10FF3000F7FD93F5F50FE3F6B8FC9387D7FA93F73F
:10FF4000D70FE1D305071377F70F9386C6037DB765
:10FF500041669745FB1F83C5A5501747FB1F032725
:10FF6000270D81477D1625486394F5000145828061
:10FF700036233A85638BC600545B81CAB4329386BC
:10FF8000E6FD93F6F60FE374D8FE850793F7F70FB7
:10FF90001307C703D1BF011122CC2A84494506CEDD
:10FFA000EF607FD61DC12AC622859730FB1FE780F0
:10FFB000C0BB01CD624432460E39F2401745FB1FEB
:10FFC0000345B54905616F406FCEF240624405615B
:10FFD000828079714ECE52CCAE892A8A9305300543
:10FFE000414526D24AD056CA5AC806D622D4328BA8
:10FFF0003689BA8A9700FB1FE7804006CD4429C99D
:020000025000AC
:100000002A848944638109044146814523126101A0
:100010009700FB1FE780803A5686CE8522859700A1
:10002000FB1FE78020332146630F0902CA852800A1
:100030009700FB1FE7800032A28650002C005285FB
:10004000EF400000AA8422859700FB1FE780200E66
:10005000B25022540259F249624AD24A424B268592
:10006000925445618280814528009700FB1FE780FC
:10007000E034D9B7411122C4405926C206C6AA8429
:1000800029CC085409C59700FB1FE780400A28586F
:1000900009C59700FB1FE7808009685809C59700CC
:1000A000FB1FE780C008285C09C59700FB1FE7809D
:1000B0000008685C09C59700FB1FE780400703251F
:1000C000040809C59700FB1FE7806006228597009A
:1000D000FB1FE780C00523AA040222448E38B240E9
:1000E00092441745FB1F0345553741016F406FE5AB
:1000F000411126C206C622C4AE849730FB1FE7809A
:10010000C0A631C9032345032A8463060304832858
:10011000C30703288307832743070327030783466F
:10012000630003560300834523002685EF60BFC5A7
:100130002285EFF03FF4EFF0BFE111CD2244B24051
:1001400092441745FB1F034555318545410117333F
:10015000FB1F6700C38AB24022449244410182805F
:10016000411122C426C206C6AA842E849730FB1FE2
:10017000E780A09F5C5989CF9E23639B97008547AA
:100180006318F4002244B240924441016FF09FEEA4
:10019000B2402244924441018280411106C622C4E9
:1001A00026C2EFF01FD429C144592A8495CCBC2023
:1001B0009DC79747FB1F83A727E889C7DC4399C3DF
:1001C00026858297B8309307F002631FF7002A2034
:1001D0002244B2409244814541016FF07FF197473C
:1001E000FB1F83A727E5D1BFB240224492444101BF
:1001F0008280411126C24AC006C622C4AA842E8922
:100200009730FB1FE780609605CD405955C41E20EE
:100210006394970A3C30130710026395E7083C206B
:10022000ADCF7C5403270408DE2B15E313F717002A
:1002300019CF18545A23058B19CB930720023CB0D1
:10024000B24022449244024905454101828013F79D
:10025000270001CB18545A23098B01C7930740028A
:10026000F9BF918B81CB1C54DE23918B81C79307FF
:100270006002F1B79747FB1F83A707DCF1D3DC438C
:10028000E1D32285829738309307F0028145E31944
:10029000F7FA2685EFF0DFE565B79747FB1F83A7E1
:1002A00067D9E9BF1307A0026398E7006304090058
:1002B00013092003CA85F1BF631C09002685973006
:1002C000FB1FE780808A09C55C2193E707015CA1D9
:1002D000A6854A85EF60EFBAA5B7011126CA9947EE
:1002E0006C85AA842E858D4522CC4AC806CE3289DB
:1002F00036847C84EFE02FB62AC61DC9AA854A85BC
:1003000002942A8419E52C002685EFF04FB12A8447
:1003100011C532459700FB1FE78060E12685EFF0AD
:100320009FC7F24022856244D244424905618280DF
:100330004D44EDB7411122C42E862E84971600003D
:100340009386667B894506C626C24AC02A89EFF095
:10035000DFF80C20AA844A85EFF09FD9B2402244EE
:10036000024926859244410182809747FB1F83A75B
:1003700067CC85CB9C4395C71D71A2CC86CE984196
:1003800010082A843AC8D84185453ACA829711C5CF
:1003900048862A206C00EFF0FFF9F640664425619C
:1003A00082808280AA872E8591CFFC5781CF9823A7
:1003B00098A1983398B1B82BB8A1982FDC4BB8B15D
:1003C000DCC18280414681451703FB1F670003FFA4
:1003D0009747FB1F83A747C681C79C4791C3828766
:1003E000094582801747FB1F032787CB1DC758434A
:1003F000AA8705450DC703A50708411106C6930640
:1004000005021306050C930505061305050402975E
:10041000B2401375F50F41018280054582808280CC
:100420004DC9357122CD2A840A2126CB52C556C327
:100430005AC106CF4AC94EC7DEDE2E8AB28A368B33
:100440009720FB1FE7806072AA8431C50C182285B3
:10045000EFF05FF53C20938B6400A9CBEF501FFCBD
:100460002A89014583C95400EF50DFF8AA840C1093
:100470000818EF10804A08542C10EF10A04ADE88AC
:10048000A68B5AC04E88DE874A8714103010D68556
:100490005285EF200076FA406A44DA444A49BA4964
:1004A0002A4A9A4A0A4BF65B0D618280EF501FF789
:1004B000AA89014503C95400EF50DFF32ACE08543E
:1004C0000C10EF1080452C100818EF10A045F248D2
:1004D0004DBF8280AA8701CD1855414511CBFC57ED
:1004E00081CB28333D476375A700882F8280414523
:1004F00082806DC5411122C406C626C2AA872E84F9
:100500000945E1C998337D761306F67F98A1B82393
:100510004D4598B1B833B8A1D823B8B1D433DA2156
:10052000858AA2061377F7EF558FDAA1D4333347C4
:1005300007081377F7DF93D61648A606558FDAA17A
:10054000D433334707081377F7BF93D62648AA0654
:10055000558FDAA1D43333470708718F93D63648C5
:10056000AE06558FDAA1F42333470708799B858AB5
:10057000558FDAA1F42333470708759B898A558F75
:10058000DAA1F423334707086D9B918A558FDAA1CE
:10059000F823DE21218BDD9BD98FDEA1EF60AFF642
:1005A000AA845145EF602FF6383093F4F40FAA87F0
:1005B00049456360970293F7F70F63ECE700182053
:1005C0009147614563E7E7001830854763E3E7003B
:1005D0000145B24022449244410182800945828013
:1005E00015C52A87AE87094585C5411106C614334E
:1005F00013851700194694A1930527009700FB1F48
:10060000E78040D5B24001454101828009458280A2
:1006100082800DC9AA872E8709459DC5411106C64E
:10062000B423903313052700A206D18E96A121464C
:10063000938537009700FB1FE780C0D1B24001458A
:10064000410182800945828082801DC12A87AE8750
:1006500009458DC141113E8541469305170006C6E7
:100660009700FB1FE78000CFB24001454101828027
:10067000094582808280AA87094591CB89C99C332C
:100680003D4761456365F7009CA1014582808280FA
:1006900005C52A87AE87094595C141113E851306D8
:1006A00000049305170006C69700FB1FE78080CA69
:1006B000B2400145410182800945828082801D71DE
:1006C000A2CC2A84084586CEA6CA230601000421AE
:1006D00035479387F4FF93F7F70F6362F70A17D74D
:1006E00001001307A762B3C7E7209C43BA9782872C
:1006F0000C08EFF01FE0C947631CF50499475C86BE
:100700002A206C00EFF01FC3F6406644D6442561F2
:1007100082800C08EFF03FF61DED2A209720FB1F8A
:10072000E780A044A14705C15825631CF70417477B
:10073000FB1F032767909D4719C7184309C7100877
:10074000A6850297AA875C8629A00C08EFF07FECAB
:1007500069D51C86D5F72A20EFF0FF8375B70C0802
:10076000EFF01FE8F5B71C312308F1007DB70C0846
:10077000EFF01FF2F1BF0C08EFF03FEDD1BF9D4746
:10078000BDBF1747FB1F0327E78A75B7411122C476
:1007900006C626C24AC01821930720092A84631A74
:1007A000F7101C3139476395E70A5621096761073D
:1007B00081476398E6089744FB1F93842488884008
:1007C00049C10C4403C90500631D09001C218505AE
:1007D0002146B9CB29059700FB1FE780A0B79C40B5
:1007E000A5C349459700FB1FE78000A72A841DC1C8
:1007F000930710FC1CA1A30025018C40090541466C
:1008000089059700FB1FE780E0B49C40A2858833F0
:10081000EF30BFA388409700FB1FE78040919747C8
:10082000FB1F23AD078029A809059700FB1FE78060
:1008300060B2EF30B00005495DF19C402380270194
:100840008547B2402244924402493E85410182805C
:100850001307E003639DE706382195476319F70204
:100860004A21EFF06FC29147E31CF5FC9737FB1F5D
:1008700083A7477CF1D79C47E1D772244A20930590
:1008800064002244B2409244024941018287A14758
:10089000631BF7006C204A202244B2409244024974
:1008A00041016FF01F95930600038147E31BD7F8C2
:1008B000D5B79306000A8147E315D7F8EFF03FE07C
:1008C00008443DDD9700FB1FE780608695BF8147A8
:1008D0008DBF011122CC06CE26CA4AC8094415CDC7
:1008E000AE8409449DC92A898D456800EF509F84D4
:1008F0001C8726866C0093F7F70393E707044A8565
:100900005C87EF2000262A8409E90D466C001385D8
:1009100034009700FB1FE780E0A3F2402285624489
:10092000D2444249056182805D714EDE86C6A2C412
:10093000A6C2CAC052DC56DA5AD85ED6894955C911
:10094000328989495DC6138B45002A8AAE8A334BAA
:100950000B08930530055A8597F0FA1FE780007061
:100960002A84CD4959C5EF505FADAA845686D285F9
:1009700093DA840013DA040193FBF40F13054400A7
:1009800093FAFA0F137AFA0FE1809700FB1FE780C2
:10099000A0B2A301740123015401A300440104A0E7
:1009A000EF501FA9AA85414608089700FB1FE78062
:1009B000A0B0214734005A86A2850808EF20E04005
:1009C000AA891DE121462C0023007901A3005901C9
:1009D00023014901A3019900130549009700FB1F5A
:1009E000E78080ADEF503FA6228597F0FA1FE780A1
:1009F0000074B640264496440649625AD25A425B75
:100A0000B25B4E85F25961618280411126C2AA848F
:100A10002E854AC006C622C42E899720FB1FE78078
:100A2000C01469C5405969C45C30094793F6B70FD3
:100A30006387E60011471305E00F6395E7081E2062
:100A4000094563912709130984004146A6854A8513
:100A50009700FB1FE78000904146A685130584019F
:100A60009700FB1FE780008F383085469307F7FE1D
:100A700093F7F70F63EEF6049304C4039737FB1F55
:100A800083A70762C14526858DC79C4F9DC382976A
:100A90009306C4022686CA852285EFF07F983C2003
:100AA00081CF22852244B2409244024941016F1015
:100AB000C00CEF502FE8E9BF3830C947E303F7FE19
:100AC0003CB00145B2402244924402494101828037
:100AD00093071005E317F7FE3C20E5D72285224453
:100AE000B2409244024941016F10600F0945D9BFDD
:100AF0004945C9BF797152CC2A8A328522D44AD05D
:100B00004ECE06D626D2AE8932899720FB1FE780CB
:100B1000C005494405C9445949448DC49E20639386
:100B20002703DC30A18B85EB0944B8309307B0056F
:100B3000631AF7002685EF106007BC20ADCB930742
:100B4000C005BCB0B2502285225492540259F249D9
:100B5000624A456182801739FB1F13096954832754
:100B600009001304E00FF9DF9C47E9DF13848401D7
:100B700022854146D28597F0FA1FE780A07D832722
:100B8000090083A5040822869C47938505042E85C9
:100B90000A87814682972A844146CE850A85970036
:100BA000FB1FE780A08C49D11374F40FBDBF9307DE
:100BB000E00541BF39C9011122CC26CA06CEAA845C
:100BC0002E84094595CD0D468D05280097F0FA1F16
:100BD000E78040781C8570002C0093F7F70393E7BB
:100BE000070426855C85EF10D07719E90D46A285AC
:100BF00068009700FB1FE78060877D153335A000F4
:100C0000F2406244D244056182800945828001112C
:100C100052C42A8A32854EC656C25AC006CE22CC4B
:100C200026CA4AC82E8BB28AB6899720FB1FE78056
:100C3000C0F309ED8944F24062444249B249224A74
:100C4000924A024B2685D244056182805C592A89EA
:100C5000C544F5F34D45EF600F8B1374F50F514507
:100C6000EF606F8AE38809FC03C78901E36487FCAE
:100C70009377F50FE3E0E7FC930530051305400893
:100C800097F0FA1FE780803D232AA9022A84CD44E9
:100C90005DD113064008814597F0FA1FE780007286
:100CA000A301040023014401230264012310540121
:100CB0002326340723240402A302040063070A0046
:100CC0002285EF00D065AA8419E18144ADB74A8539
:100CD000EFF04FBA8DB7397122DC06DE26DA4AD83A
:100CE0004ED652D456D25AD05ECE62CC66CA094491
:100CF000630A0610BA84094463060710AA8B2E897A
:100D0000328B368C9720FB1FE78020E6AA8A51445D
:100D100075C993053005414597F0FA1FE780003407
:100D2000AA894D4465C198309C2003CA340022072B
:100D30005D8FBC20620AC207D98F336AFA0083A78D
:100D40008A0263E647017D5709446398E70A63070F
:100D5000090083C74A000544898BC5C321468145E4
:100D60000A8597F0FA1FE7806065930C4C009305A5
:100D70003005B3CC0C08668597F0FA1FE780002E8B
:100D80002A894D443DC96286DA85110597F0FA1F1C
:100D9000E78080721146A6854A8597F0FA1FE780A2
:100DA000A071414693858A014E8597F0FA1FE7802E
:100DB000A07021478A866686CA854E85EF20E000AE
:100DC0002A841DE521468A85280097F0FA1FE780CE
:100DD000A06E214693854400280097F0FA1FE78013
:100DE000E0688547631EF502D2855E85EF608FADB2
:100DF0004A8597F0FA1FE78080334E8597F0FA1FF7
:100E0000E780E032F25022856254D2544259B259FE
:100E1000225A925A025BF24B624CD24C2161828080
:100E20000544F9B7797122D406D626D24AD04ECEDF
:100E30002E849397556063D607049734FB1F9384E1
:100E4000A461A83097F0FA1FE78000472AC609CDB1
:100E5000EFF0DF93B24511E5A8209307F00F631F71
:100E6000F5002E85EF304FB91319F468B2502254B3
:100E70009254F2494A85025945618280EF30EFBCB5
:100E8000E5B713F9150063070900EFF00FB1134937
:100E90001400E9BFE1DD854421A0850493F4F40F3B
:100EA000EFE0BFD6E3F4A4FCB3179028B3C907085A
:100EB000E18FE5D74E85EFE09FFFC167FD17630522
:100EC000F500DD45EFF0CFA23349340145B7973740
:100ED000FB1F23A507169737FB1F23AF0714973770
:100EE000FB1F23A907149737FB1F93872756170764
:100EF00000001307475E98C3170700001307472F2A
:100F0000D8C317F7FFFF1307070D98C79737FB1FC5
:100F100093870753171700001307C74698C317177F
:100F20000000130747FFD8C3171700001307872ACD
:100F300098C782809737FB1F83C74752A18B014711
:100F400089C71737FB1F130767509737FB1F23A568
:100F5000E70E014582809737FB1F83C72750918B8F
:100F6000014789C71737FB1F1307874D9737FB1FAB
:100F700023A2E70C01458280011106CE2AC6EFF0BC
:100F80001FF5324599459737FB1FA388A74CEFD033
:100F9000AFE7F24017F5FFFF1305C51C05616FE0D1
:100FA0007FC71C5599C321458280411122C426C2A6
:100FB0002A84AE84130500049305300506C64AC092
:100FC00097F0FA1FE780800908D469C91306000466
:100FD000A68597F0FA1FE780E0377454B82A937714
:100FE0008700FDCB1C54BC23A18BFDC783270408BD
:100FF000D5E7930530051305001097F0FA1FE78039
:10100000E005AA872320A4080D45D1CB74549C3059
:101010009832C1CF3337E0000E07936707016C5455
:101020005CB0B829058B19CB1854854638230D8B35
:101030006316D70078201367170078A003270408E9
:1010400009C778201367870078A00547639FE70CDE
:1010500013098400414681454A8597F0FA1FE780CD
:10106000E035814513058401414697F0FA1FE7807A
:10107000E0349304C4039737FB1F83A76702C1457D
:101080002685B5CF9C4FA5CF829783270408BDCB7B
:101090002285EF00D0349307000549C12145B240B5
:1010A00022449244024941018280A1472DFBBC2089
:1010B000918B91E7BC2A918B99E385478DB7982056
:1010C000942295473307F70297D70100938787C784
:1010D000BA97B6979C23A1B79C3081C79032E1475D
:1010E0001DFEBC205D8F118B69DB982095479422F3
:1010F0003307F70297D70100938787C6D1BFEF5018
:101100006F8361B722859306C4022686CA85EFF0F5
:101110002FB12285EF00702651F1C1470A203CB063
:101120008145EF503FE401459DBF13F7870151C74B
:10113000C18B930484004146B1CB8905268597F085
:10114000FA1FE7802021814513058401414697F06D
:10115000FA1FE780A0267C201309C403C14593E74A
:1011600047007CA09737FB1F83A787F34A8595C765
:101170009C4F85C78297832704089DC32285EF0073
:10118000102609FD930720053CB071BF81452685D7
:1011900097F0FA1FE78080227DB7EF40BFF9E1BFEB
:1011A0009306C4024A86A6852285EFF06FA72285A2
:1011B000EF00B01CCD4769D9D5B50947854563888F
:1011C000E70093F7D70F11476396E70089450A2098
:1011D000EF505FD97C2093E747007CA08327040869
:1011E00081C7930710054DB7C54779BF3C2163857B
:1011F0000726397122DC06DE26DA4AD84ED652D4CA
:101200003C31130750052A846397E70803497500AA
:10121000173AFB1F130ACAE89309C503935739000D
:10122000AA97842783270A00C1454E85B5C39C4FE2
:10123000A5C3829783270A00A1C79C47B1C3032592
:10124000040813797900B3D62441858A93050504EF
:10125000180893E606084E8613050508829713754D
:10126000F50F19ED41460C081305C40297F0FA1F5B
:10127000E780400E2285EF005010930760053CB0D8
:10128000F2506254D2544259B259225A216182809A
:10129000EF405FEA45B7130710026392E7021C555F
:1012A00003270508DE2361EB13F7071069C778559C
:1012B0005A2B1377071061C3930770023CB03C3080
:1012C00013077002639FE70C3C5885E393053005D4
:1012D000714597F0FA1FE78060D828D819C5714684
:1012E000814597F0FA1FE780600D2458A1C8BC2CF7
:1012F00089E72285EFF00F9EA8AC2858814541462A
:1013000097F0FA1FE780800B28583D472C2D9387D4
:10131000F5FF93F7F70F6364F700EF40BFE1EF20AD
:101320005FFD3C58A1458AAB13852701EF409FE044
:101330002C580A20EF003034631A051093078002FE
:101340003CB00A209720FB1FE7802082414609C558
:101350007E2513D617003E966254F250D25442595D
:10136000B259225A1735FB1F0345350F060685452E
:1013700021616F30AF9313F7072009CB78545A2BB4
:101380001377072001C7930790020DBF93F707401B
:101390009DD77C54DE2B93F7074095D39307B0027B
:1013A00031BF130780026397E7023C5899C78E2B21
:1013B0000A2013862701EF0070311C54DE2313F737
:1013C000072029CF78545A2B1377072021CB930776
:1013D0009002BDB713079002639BE700EF50AF8404
:1013E000AA850A20EF00902D9307A00291BF130752
:1013F000A0026390E704EF506F82AA8585470145FC
:101400006384F500814505452EC6EF40BFFE2A8660
:10141000B2450A20EF0030271C54DE2393F7074023
:101420009DC37C54DE2B93F7074091CF9307B00206
:1014300001BF1307B0026398E700EF407FFFAA8562
:101440000A20EF00102C9307F00215BD38309307E7
:10145000F002E318F7EE2DB58280411122C4405905
:1014600026C206C67C54AA84DE2B13F7071011C7C8
:1014700018545A23137707100DE313F7072011C7E9
:1014800018545A231377072009EB93F707408DCBA5
:101490001C54DE2393F7074085C7930710023CB026
:1014A0002285EFF0BFD438309307F002631EF700B7
:1014B0002244AA20B2409244814541016FE05FC3BB
:1014C0009307F0023CB0EDB7B24022449244410190
:1014D0008280397122DC405926DA4AD84ED606DE9F
:1014E0002A89AE84B289630604382A211E206391BA
:1014F000A7123C20638A07389387E5FF93F7F70F1D
:101500002D476363F73817D7010013072787B3C741
:10151000E7209C43BA97828722856254F250D254C6
:101520004259B259B28521616FF0BFA74146CE85BD
:101530001305C40497F0FA1FE780C0E12285BD259A
:10154000383093074005631AF70093079005333549
:10155000A000931435003CB06DA893066005D147F8
:10156000E317D7FE9307A005DDB71309C4054A8525
:101570004146CE8597F0FA1FE780C0DD03250408B9
:101580005DC53C30130790056397E7002285452D24
:101590009307E005A5A81307A0056394E7087C302E
:1015A00013D73700229714279D8BB3D6F640858A30
:1015B0009737FB1F83A7C7AE93E60608B1CB9C47BE
:1015C000A1CB9305050818084A86130505048297E0
:1015D0001375F50F15ED41460C081305C40497F07B
:1015E000FA1FE780A0E87C304D47850793F7F70F97
:1015F0007CB0E36DF7F885451735FB1F0345F5E52E
:101600009710FB1FE780A03F930750053CB031A81F
:10161000A144F25062544259B2592685D2542161F4
:1016200082801307C005E383E7F68144DDB79309A1
:1016300084004A86CE8522851408EFE07FDE41468D
:101640009305C404080897F0FA1FE78020E271D1DF
:101650008A861306C403CA854E85EF10A06DA14487
:101660000DE12285EFE01FE72A870A209737FB1F4D
:1016700083A747DE814601468A858297B334A0005E
:101680008E0493072002C1BD0C22EFE07FA671BF3C
:101690003830930720026319F71E7C5889EB9305B5
:1016A0003005714597F0FA1FE780409B68D868586D
:1016B000630C051C4146CE8597F0FA1FE78080C970
:1016C00064582285EFE01FE1A8AC930730023DBFCC
:1016D0003830930730026319F71A1E2268582146E2
:1016E000938529001EA9490597F0FA1FE78080C657
:1016F0007C54DE2B13F727002DC718545A23098B6F
:101700002DC39307400219B7383093074002631D79
:10171000F7163C5C81EB85455D4597F0FA1FE78045
:10172000E09328DC285CE30205F083C7090041460A
:10173000CE857CA997F0FA1FE780C0C193075002BD
:10174000F1B53830930750026310F714285C19463E
:1017500093851900410597F0FA1FE780A0BF7C54DC
:10176000DE2B918B95CF1C54DE23918B95CB930769
:10177000600269BD7C5C89EB93053005514597F0AB
:10178000FA1FE780A08D68DC685CE30305E841464A
:10179000CE8597F0FA1FE780E0BB7C5C7D5798CB45
:1017A0004A85EFF09FCB51B50325040813060004CA
:1017B000CE851305050497F0FA1FE780A0B92285AE
:1017C000EFE05FC23C30130700056395E700930725
:1017D00040052DBD13071005E38FE7E01307200533
:1017E000E395E7E49737FB1F83A7878BE38207E244
:1017F0009C47E38F07E083250408930484001808BE
:1018000093850508814626862E8582970A20100832
:10181000A685EF500FFE9307B005CDBB3830930778
:10182000E0056313F7068325040841464E8597F0CB
:10183000FA1FE780A0C3AD44E30D05DC03250408CF
:101840004146CE8597F0FA1FE780C0B02285EFE0D1
:101850007FC82A872C580A209737FB1F83A787BF8A
:10186000814601468297B334A0008E04930710028C
:10187000DDB1AD47E39BF5DA14222E211306650096
:101880000821EF40BFF255B39D4461B3AA870945D3
:1018900041C6D9C11CA29C211CB29C313CA2BC21D6
:1018A0003CB2BC31A30206005CA2DE2193D787487C
:1018B0005CB2DA211377072001C793E727005CB2F7
:1018C000DE2193F7074089C75C3293E747005CB29B
:1018D000DE211317B028F98F89C75C3293E78700A0
:1018E0005CB223030600DE21858B7CA2DA21098B02
:1018F00001C793E727007CA2DE21918B89C77C2258
:1019000093E747007CA2DE21A18B89C77C2293E765
:1019100087007CA20145828082802E86AA850545AB
:101920006FF0DFF62E86AA8509456FF03FF68DC56C
:101930002A87094505C7411106C6AE878D4694A181
:10194000138517004146BA8597F0FA1FE78080A0FB
:10195000B2400145410182800945828082808DC567
:101960002A87094505C7411106C6AE87914694A14D
:10197000138517004146BA8597F0FA1FE780809DCE
:10198000B2400145410182800945828082808DC537
:101990002A87094505C7411106C6AE87994694A115
:1019A000138517004146BA8597F0FA1FE780809AA1
:1019B000B2400145410182800945828082809DC9F3
:1019C0002A87094515CB411106C69D4694A11623C9
:1019D000AE871385370094B116232146A182B4A1A6
:1019E0009305270097F0FA1FE780C096B2400145A3
:1019F000410182800945828082808DC52A87094500
:101A000005C7411106C6AE87A14694A113851700EC
:101A10004146BA8597F0FA1FE780C093B24001456E
:101A20004101828009458280828085C92A870945D3
:101A30001DC7411106C6A54694A11423AE87138580
:101A4000270094B119469305170097F0FA1FE78015
:101A50006090B240014541018280094582808280C8
:101A60008DC52A87094505C7411106C6AE87A94617
:101A700094A1138517004146BA8597F0FA1FE780B5
:101A8000608DB2400145410182800945828082809B
:101A900095C52A8709450DC7411106C6AE87B146CF
:101AA00094A11385170013060004BA8597F0FA1F56
:101AB000E780408AB2400145410182800945828029
:101AC00082808DC52A87094505C7411106C6AE87A4
:101AD000B54694A1138517004146BA8597F0FA1FC1
:101AE000E7804087B24001454101828009458280FC
:101AF0008280AA87094581C999C7154798A19C2367
:101B000001459CB182808280AA87094581C999C715
:101B10002D4798A19C2301459CB1828082800DC5F0
:101B20005D718A8586C6A2C42A84EFE0BF870A2039
:101B30000A8697060000938686DE9D45EFE0EFF962
:101B4000B640264461618280054582800DC55D7185
:101B50008A8586C6A2C42A84EFE0DF840A200A862A
:101B600097060000938646DC9D45EFE00FF7B640F0
:101B7000264461618280054582805D71A2C493051F
:101B8000C5022A8441460A8586C697E0FA1FE78087
:101B9000607C0A200A8697060000938686D9C54590
:101BA000EFE0AFF3B6402644616182805D71A2C46C
:101BB0009305C5032A8441460A8586C697E0FA1F25
:101BC000E78040790A200A8697060000938666D946
:101BD000C545EFE08FF0B6402644616182809727CB
:101BE000FB1F83A7E74BA9CB9C435D71A2C486C6AC
:101BF0002A841305E00F8DCF032504089305050CF7
